:020000040800F2
:100000000000012019760008EB330008ED330008EA
:10001000EF330008F1330008F3330008000000005C
:10002000000000000000000000000000F5330008A0
:10003000F733000800000000F9330008FB33000824
:100040006976000869760008FD33000869760008C3
:100050006976000869760008093400081934000838
:1000600069760008293400086976000831340008F0
:100070003D340008493400086976000869760008B4
:10008000553400085934000869760008697600087C
:1000900000000000697600086534000869760008F1
:1000A00069760008697600086976000869760008B4
:1000B00069760008697600086976000869760008A4
:1000C00069760008697600086934000869760008D6
:1000D00069760008753400086976000869760008BA
:1000E000697600086976000881340008697600089E
:1000F0006976000800000000000000006976000832
:1001000069760008697600088D3400086976000871
:100110006976000869760008697600086976000843
:100120006976000869760008697600086976000833
:080130006976000869760008F9
:1001400010B5054C237833B9044B13B10448AFF311
:1001500000800123237010BDC008002000000000B3
:10016000942B030808B5034B1BB103490348AFF3B5
:10017000008008BD00000000C4080020942B030884
:1001800014214160704714207047406A7047000096
:1001900081010008870100088B010008A101000807
:1001A00010B5044604F1100000F05CFCC4F8F8003F
:1001B0000148C4F87C0110BD90010008F8B5E6B014
:1001C00004460D4616461F460A4906A800F0CAFE18
:1001D00070996F9A05910492009733466E996D9AC3
:1001E000039102922A466C990191214600F060F831
:1001F00067B0F0BD9C010008F8B5E6B004460D46B6
:1002000016461F46094906A800F0ACFE6F996E9A83
:100210000491039200976D996C9A02910192334672
:100220002A46214600F087F867B0F0BD9C0100081F
:1002300038B500281CBF01680029184A23D1184B83
:100240001C684FF6F0710C404CF24025AC421FBFC9
:100250001B6819404CF27024A14212D1114D29683B
:1002600079B911490B68C3F30B03B3F58A6F1FBF4C
:100270000968C1F30B0140F28343994204BF012195
:10028000117028B905E0094B994204BF0121117092
:100290004068BDE8324002F071BC00BFDC080020BD
:1002A00000ED00E0002004E00010005C0000374892
:1002B0002DE9F04104460D46216816464A681F465E
:1002C00090478046B8F5403F2ED122680A9993683E
:1002D000204698478046B8F5403F25D12368089AC4
:1002E0000799D3F80CC02046E0478046B8F5403F58
:1002F0001AD12368069A39461F692046B8478046B6
:10030000B8F5403F10D1236829465D693246204642
:10031000A8478046B8F5403F06D123680B9A099953
:100320009D692046A847804621680A682046904774
:100330004046BDE8F0812DE9F04104460D462168B4
:1003400016464A681F4690478046B8F5403F2ED172
:1003500022680A999368204698478046B8F5403F3E
:1003600025D12368089A0799D3F80CC02046E047A6
:100370008046B8F5403F1AD12368069A39461F696E
:100380002046B8478046B8F5403F10D1236829463B
:100390005D6932462046A8478046B8F5403F06D101
:1003A00023680999DD6900222046A8478046216814
:1003B0000A68204690474046BDE8F0814FF440303F
:1003C00070470000F0B50C4685B0114600281A466B
:1003D0001CBF0568002D0B4B11D082B104B971B957
:1003E0000D9860B10F9E0E9F0A9B02900496039792
:1003F0000B980C9E009001962046A847034618468D
:1004000005B0F0BD020003002DE9F04F0646D0B064
:100410000868F56DD6F860E0726EB76EF36E00BADC
:1004200000906C46486800BA60600DF1400888682A
:1004300000BAA060C86800BAE060086900BA20612C
:10044000486900BA6061886900BAA061C86900BAE9
:10045000E061086A00BA2062486A00BA6062886A8D
:1004600000BAA062C86A00BAE062086B00BA2063F2
:10047000486B00BA6063886B00BAA063C86B00BAAF
:10048000E063402058F80C1C58F820CC58F838ACE1
:100490008CEA010158F840CC8AEA01018CEA010992
:1004A0004FEAF979401E48F8049BEBD187EA020035
:1004B00000EA0E00784010EBF5610098DFF824C4E4
:1004C00041186144C81882EABE032B404FEAF0612C
:1004D00053405918636859186144CF194FEAB5035E
:1004E00083EABE01014081EABE0111EBF765A16814
:1004F0004D196544A91883EAB0023A404FEAF16504
:100500005A405519E26855194FEAB70282EAB00716
:1005100065440F4005EBBE0E97EAB00717EBFE658A
:1005200027697D194FEAB10782EA0701654401EAAC
:100530000E01EB18514011EBF36561694D194FEA5B
:10054000BE0187EA010E65440EEA030E15EBB0000A
:100550008EEA070E0EEBF065D4F818E0754465449A
:10056000AA1881EAB30505404FEAF26E4D40AE4449
:10057000E569AE44E64477444FEAB00080EAB30E42
:100580000EEA020E8EEAB30E0EEBF765D4F820E009
:1005900075446544691880EAB2053D404FEAF16E42
:1005A0004540AE44656AAE44E6440EEBB3034FEA01
:1005B000B70787EAB20E0EEA010E8EEAB20E0EEB14
:1005C000F365D4F828E075446544281887EAB10536
:1005D0001D404FEAF06E7D40AE44E56AAE44E6440D
:1005E0000EEBB2024FEAB30383EAB10E0EEA000E3D
:1005F0008EEAB10E0EEBF265D4F830E07544654436
:10060000EF1983EAB00515404FEAF76E5D40AE443E
:10061000656BAE44E6440EEBB1014FEAB20282EAEA
:10062000B00E0EEA070E8EEAB00E0EEBF165D4F8AE
:1006300038E075446544EB1882EAB7050D404FEA8F
:10064000F36E5540AE44E56BAE44E6440EEBB000AD
:100650004FEAB10181EAB70E0EEA030E8EEAB70E39
:100660000EEBF065D4F840E07544654481EAB30EC2
:10067000AA180EEA000E4FEAF2658EEA010E7544E2
:10068000DDF844E04FEAB000754480EAB30E6544FB
:100690000EEA020E15EBB7078EEAB30E0EEBF76506
:1006A000DDF848E04FEAB202754480EA020E654484
:1006B0000EEA070E69188EEA000E0EEBF165DDF802
:1006C0004CE07544654405EBB3034FEAB70E1427BD
:1006D0000DF1500CDFF810528EEA010B82EA0B0B81
:1006E0000BEBF36A5CF804BBDA44AA44504483EA97
:1006F000B10B4FEAF06A8EEA0B0BDA445CF804BBEC
:10070000DA44AA44524480EAB30B4FEAF26A8BEA15
:10071000B10BDA445CF804BBDA444FEAB000AA44F7
:1007200080EA020BD6448BEAB30B0BEBFE6A5CF853
:1007300004BBDA444FEAB202AA4482EA0E0B0AEB87
:10074000B10180EA0B0B0BEBF16A5CF804BBDA44F5
:100750007F1DAA44282F0AEBB3034FEABE0EBBD37A
:100760003C2F61D3502F4DD204EB870CC7F15407B7
:100770005E4CA7FB04A504465D4FA8088EEA010A5B
:1007800082EA0A0A5CF804BB0AEBF3655D447D1952
:100790002C1983EAB10A4FEAF4658EEA0A0A554435
:1007A0005CF804AB5CF804BB55447D19AA1884EAD4
:1007B000B30A4FEAF2658AEAB10A55445D444FEA4A
:1007C000B4047D1984EA020AAE448AEAB30A0AEB49
:1007D000FE655CF804AB55444FEAB2027D1982EA2B
:1007E0000E0A15EBB10184EA0A0A5CF804BB0AEBB5
:1007F000F1655D447D1915EBB303401E4FEABE0E53
:10080000BCD12046F46D1B19F365336EC9183166EF
:10081000716E71447166B36ED218B266F16E401893
:10082000F06650B0BDE8F08F4EEA010B0EEA010A07
:100830000BEA020B4BEA0A0A0AEBF36554F827A00D
:10084000DFF8B0C0554443EAB10B654403EAB10A8E
:100850000BEA0E0B28184BEA0A0A7F1C0AEBF0651C
:1008600054F827A0554440EAB30B654400EAB30AA4
:100870000BEAB10BAA184BEA0A0A7F1C0AEBF265D5
:1008800054F827A055444FEAB00040EA020B6544F3
:1008900000EA020A0BEAB30BAE444BEA0A0A7F1CD9
:1008A0000AEBFE6554F827A055444FEAB20242EA2B
:1008B0000E0B654402EA0E0A0BEA000B15EBB101C0
:1008C0004BEA0A0A7F1C0AEBF16554F827A055444D
:1008D0007F1C65443C2F05EBB3034FEABE0EA3D348
:1008E00040E700BF9979825AA1EBD96ECDCCCCCC30
:1008F000D6C162CADCBC1B8F00B581B00168074A53
:10090000914200D110B9064801B000BD7C212EF003
:10091000F2FE4FF4003001B000BD00BF040A000831
:10092000030002002DE9F0410B4A92E8F85188B02B
:10093000694681E8F8510268084B9A4200D118B91B
:10094000074808B0BDE8F0811422083000F04FFBE2
:1009500008B0BDE8F08100BFE4090008040A0008FF
:1009600003000200152904D20268044B9A4200D108
:1009700008B903487047083000F048BB040A000873
:100980000300020010B481B013460268074CA24273
:1009900000D118B901B010BC0548704701B000F192
:1009A000240210BC083000F035BB00BF040A000868
:1009B0000300020010B481B013460268074CA24243
:1009C00000D118B901B010BC054870470A4601B003
:1009D00000F1240110BC083000F070BB040A0008CC
:1009E000030002000123456789ABCDEFFEDCBA9816
:1009F00076543210F0E1D2C3000000000000000085
:100A000000000000F9080008250900086509000831
:100A100085090008B509000809040008810F0008CD
:100A2000CD0F0008890F0008F0B5A3B004460B48AD
:100A300002900D4616461F46094B0822402104A885
:100A400000F0D1FA28980190009733462A462146B3
:100A500002A800F01BF823B0F0BD00BF040A000894
:100A6000180A000810B5040008BF002408D0054883
:100A7000054B20600822402104F1080000F0B3FA81
:100A8000204610BD040A0008180A00082DE9F041AC
:100A900004460E46216817464A681D469047804620
:100AA000B8F5003F19D12268069993682046984707
:100AB0008046B8F5003F10D123683146DE683A46DB
:100AC0002046B0478046B8F5003F06D12368079A14
:100AD00029461D692046A847804621680A682046A5
:100AE00090474046BDE8F08110B500F033FA4FF46E
:100AF000403400280EBF034C4FF4C0712EF0FBFDB4
:100B0000204610BD0200030010B5044600F022FA92
:100B100008B9054810BD0021A160D0F87C211168FA
:100B200088474FF4403010BD0200030070B5044602
:100B30000D4600F00FFA064E40B1D0F87C01416836
:100B40008847A84224BF65604FF44036304670BDE8
:100B5000020003002DE9FF4715000C4600D02CB120
:100B6000064600F0F7F95FEA000801D16448C3E0E7
:100B7000D8F8F80001684A689047B0F5003F17D1EF
:100B8000D8F87C118A68404690478146B9F1810FB8
:100B900080F09E80A94508F1FC0A17D2D8F8F80029
:100BA0000368D3F80CC02A462146E047B0F5003F61
:100BB00040F08E80D8F8F8000368D3F810C06A4679
:100BC0005146E047B0F5003F76D10AE0002004E04E
:100BD000215C0AF800100098401C00900098A84280
:100BE000F6D34FF0000C4749474A484B01AC0098F8
:100BF000844558D2D3E9007001ADC5E90070107882
:100C000000281ABF042086464FF0000E085854F8FA
:100C10000E5028443E4D05600127D0F800E0876063
:100C2000019D4F681AF80C007D408EEA050585F09D
:100C3000040E65680F687D4085F0FC05754485F0FD
:100C4000A30568400AF80C000CF1010CCFE7D3E9CA
:100C5000004501A8C0E9004510782E4D002814BFBA
:100C60004FF0040E4FF0000E01A8744651F80EE04C
:100C70000459A6440127CEF80050DEF80040CEF813
:100C800008704D68019F40687D406C400D68684069
:100C900084F0040480F0FC00041984F057040AF87E
:100CA0000C400CF1010CCC45D1D3D8F8F800016808
:100CB0004A689047B0F5003F0AD1D8F8F8000368B9
:100CC000D3F80C804A465146C047B0F5003F01D0EA
:100CD000114811E0002006E05AF8201081F06A3136
:100CE0004AF82010401CB0EB990FF5D3B06840F0E3
:100CF0000100B0604FF4403004B0BDE8F08700BFA1
:100D000002000300DC6C0308DC0800202C0F000844
:100D1000ADBE4ED70DBE75A10100030038B50C461F
:100D2000017A1546CA0702D500F014F908B9084837
:100D300032BDD0F8F80003682146DC682A46A04797
:100D4000B0F5003F01D0034832BD4FF4403032BD12
:100D500002000300010003002DE9F84191B00546AF
:100D60000E461746402101A82EF0C5FC297AC80777
:100D700004D5284600F0EEF8040002D1DFF8A48084
:100D80004BE0D4F8F800DFF8A0800368D3F810C077
:100D90006A4601A9E047B0F5003F3ED1D4F8F8001B
:100DA00001684A689047B0F5003F36D1D4F87C110D
:100DB0008A6820469047D4F8F830024618461B68E7
:100DC000D3F80CC004F1FC01E047B0F5003F24D19A
:100DD000D4F87C0141688847D4F8F83002461846B8
:100DE0001B68D3F80CC001A9E047B0F5003F14D14F
:100DF000D4F8F8000268696893689847B0F5003F36
:100E00000BD1D4F8F80003681C693A463146A04774
:100E1000B0F5003F08BF4FF44038404612B0BDE87F
:100E2000F08100BF02000300010003002DE9F8413A
:100E3000A5B0074688461646402115A82EF05BFC53
:100E400000220492402105A82EF055FC387AC107F3
:100E50005ED5384600F07EF8050059D0D5F8F80088
:100E60002D4C0368D3F810C06A4605A9E047B0F5D9
:100E7000003F3CD1D5F8F80001684A689047B0F5CA
:100E8000003F34D1D5F87C118A6828469047D5F8C0
:100E9000F830024618461B68D3F80CC005F1FC0177
:100EA000E047B0F5003F22D1D5F87C014168884782
:100EB000D5F8F830024618461B68D3F80CC005A9CF
:100EC000E047B0F5003F12D1D5F8F8000268796824
:100ED00093689847B0F5003F09D1D5F8F80003684A
:100EE0001D6904AA15A9A847B0F5003F01D0204606
:100EF0000FE00A4B0A490B4A0396029101924046C1
:100F00001C68049B009415AA796800F0E5F900E0DC
:100F1000054826B0BDE8F08101000300E46C030839
:100F2000936E030026C703000200030004B0010112
:100F300000170145E90A0008090B00082D0B0008FD
:100F4000BD030008550B00081D0D0008590D0008D1
:100F50002D0E00080168024A914218BF0020704718
:100F6000340F000810B5040008BF002404D0034863
:100F70002060204609688847204610BD340F0008CD
:100F800020225C302EF0B3BBF0B58468A3080022A9
:100F900004F0030407E000F15C0555F8226035BA5F
:100FA00041F82250521C9A42F5D300220BE000F186
:100FB0005C0502EB830755F82360D500C5F11805E1
:100FC000EE40CE55521CA242F1D3F0BD30B5C468FC
:100FD00003690022E31AD5188C5C0544521C082AC8
:100FE0002C77F8D330BD0360C1600261704738B51B
:100FF000044615460022626023685A689047002024
:101000006061A061A5604FF4003032BD81604FF493
:10101000003070472DE9F84304462079D4F80C805D
:10102000450748BF244845D466691D46A8F101001C
:1010300000EAD60306EBC506B6EBC50F666102D221
:10104000A669761CA6611746A66906EB5576A661C9
:101050000E46E918884225D2A8EB03094A463146D4
:10106000F8182EF044FB2268136839460FE0424618
:1010700038462EF03CFB23681A68394620469047D4
:1010800007E0311811F00300F1D1226813682046FF
:101090009847484600EB0809A9F10101A942F0D39D
:1010A000002300E000202A1A3118F8182EF01FFB48
:1010B0004FF40030BDE8F283040002002DE9FC4F3C
:1010C000024685B0D0681369DFF86CC1DFF86C8127
:1010D000A0EB030A506840F004005060002703A80A
:1010E00002900DF10C0ED8E9003403A8544DC0E96C
:1010F00000342878534D00280CBF00230423994660
:101100005CF803305EF80940234401261D601C682A
:101110009E60DCF80430039DDCF80090DEF804608B
:101120005D406540484C654089EA0606474C66408C
:101130007519474C6540D8E9006B03AC0028C4E939
:10114000006B0EBF002404200424029E5CF8000003
:10115000345920183F4C04600126046886600398C7
:10116000029E43406340384C7068634089EA000047
:10117000364C6040034438484340280018BF0120E3
:101180005B1E9B41042F2CBFC0B2D80F02F1140389
:1011900053F8200007F00303C3F10303DB00D8403A
:1011A0000DF807007F1C082F9DD315460C466A6971
:1011B000AB69E868D20842EA4372401E00EA0207BF
:1011C000002302409B420AD8524508D28020E055B5
:1011D0007F1C574516D2AAEB0701E01910E08020CA
:1011E000E05500E0E355E8687F1C8742FAD32A689F
:1011F000136828469847BAF1000F03D0514620469D
:101200002EF079FA2A68069E059F9368694628465B
:1012100098472A68D2F8009021462846C8472B688C
:10122000DA683946284690470EB1A86830604FF416
:10123000003007B0BDE8F08FDC6C03085C120008DA
:10124000DC0800205FC5109304850012FC68017A59
:10125000C0F524FF24AF33D426AF698B04B001015D
:1012600000170145F8B501240094002300240DE087
:10127000009D065D0F5D7E40F643761CF60F86F0FE
:10128000010635400095641C009DEB189442EFD395
:101290001846F2BDF8B5002301240094002A11E09D
:1012A000009C85188F1815F8016C17F8015C6E40CA
:1012B000F643761CF60F86F0010634400094009C3D
:1012C000E318521EECD11846F2BD0000651200086A
:1012D00095120008010000002DE9F84F1D46DDF8C9
:1012E00028900B9F0D9C4FF0FF3300930E469246C3
:1012F000D9F800B0804632465146D847834664B399
:10130000D9F8043032465146404698476FEA0B02FE
:10131000521C42EA0B0200996FEAD2735B1C19401F
:10132000C2430091521C024300996FEAD2735B1CC6
:101330001940009186F05531484087EA000181F05C
:101340005531216080F05531C943491C0843009A4A
:101350006FEAD070401C82430092D9F8080001283F
:1013600009D17540E943491C0D4300986FEAD572D5
:10137000521C90430AE0F11C85EA9102D243521CB0
:10138000154300986FEAD5735B1C984386F0AA3624
:10139000009086EA0B0686F0AA33F243DB430C98F2
:1013A000C2F3C0725B1C42EAD3720099D243521C52
:1013B00091430091774000998843009987F0AA37BC
:1013C0000F403843BDE8F28F00000000000000002D
:1013D00001F0FF01102A2BDB10F0070F08D010F8E6
:1013E000013B013A8B422DD010F0070F42B3F6D1EA
:1013F000F0B441EA012141EA014122F007047FF003
:1014000000070023F0E80256083C85EA010586EA59
:10141000010685FA47F5A3FA87F586FA47F6A5FA95
:1014200087F68EB9EED1F0BC01F0FF0102F00702A1
:1014300032B110F8013B013A83EA010313B1F8D14C
:101440000020704701387047002D06BF354603382D
:10145000073815F0010F07D1013015F4807F02BF66
:10146000013015F4C03F0130F0BC0138704700BFB7
:10147000034613F8012B002AFBD1181A01387047D4
:1014800081F0004102E000BF83F0004330B54FEA35
:1014900041044FEA430594EA050F08BF90EA020FA2
:1014A0001FBF54EA000C55EA020C7FEA645C7FEA35
:1014B000655C00F0E2804FEA5454D4EB5555B8BF58
:1014C0006D420CDD2C4480EA020281EA030382EAC9
:1014D000000083EA010180EA020281EA0303362D5B
:1014E00088BF30BD11F0004F4FEA01314FF4801C2E
:1014F0004CEA113102D0404261EB410113F0004F40
:101500004FEA03334CEA133302D0524263EB4303F6
:1015100094EA050F00F0A780A4F10104D5F1200E94
:101520000DDB02FA0EFC22FA05F2801841F10001EF
:1015300003FA0EF2801843FA05F359410EE0A5F1C3
:1015400020050EF1200E012A03FA0EFC28BF4CF0F4
:10155000020C43FA05F3C01851EBE37101F00045AA
:1015600007D54FF0000EDCF1000C7EEB00006EEBB7
:101570000101B1F5801F1BD3B1F5001F0CD3490841
:101580005FEA30004FEA3C0C04F101044FEA445298
:1015900012F5800F80F09A80BCF1004F08BF5FEA1F
:1015A000500C50F1000041EB045141EA050130BDFF
:1015B0005FEA4C0C404141EB0101013C28BFB1F511
:1015C000801FE9D291F0000F04BF01460020B1FA5C
:1015D00081F308BF2033A3F10B03B3F120020CDA2F
:1015E0000C3208DD02F1140CC2F10C0201FA0CF00D
:1015F00021FA02F10CE002F11402D8BFC2F1200C72
:1016000001FA02F120FA0CFCDCBF41EA0C01904027
:10161000E41AA2BF01EB0451294330BD6FEA040470
:101620001F3C1CDA0C340EDC04F11404C4F120025B
:1016300020FA04F001FA02F340EA030021FA04F36D
:1016400045EA030130BDC4F10C04C4F1200220FAC4
:1016500002F001FA04F340EA0300294630BD21FA02
:1016600004F0294630BD94F0000F83F4801306BFC8
:1016700081F480110134013D4EE77FEA645C18BFBC
:101680007FEA655C29D094EA050F08BF90EA020F53
:1016900005D054EA000C04BF1946104630BD91EA4B
:1016A000030F1EBF0021002030BD5FEA545C05D14E
:1016B0004000494128BF41F0004130BD14F580048D
:1016C0003CBF01F5801130BD01F0004545F0FE4101
:1016D00041F470014FF0000030BD7FEA645C1ABF36
:1016E000194610467FEA655C1CBF0B46024650EA6D
:1016F000013406BF52EA033591EA030F41F4002199
:1017000030BD00BF90F0000F04BF0021704730B51E
:101710004FF4806404F132044FF000054FF00001F3
:1017200050E700BF90F0000F04BF0021704730B5B4
:101730004FF4806404F1320410F0004548BF404289
:101740004FF000013EE700BF42004FEAE2014FEADE
:1017500031014FEA02701FBF12F07F4393F07F4FB9
:1017600081F06051704732F07F4208BF704793F0BC
:101770007F4F04BF41F40021704730B54FF46074CF
:1017800001F0004521F000411CE700BF50EA0102D2
:1017900008BF704730B54FF000050AE050EA01027B
:1017A00008BF704730B511F0004502D5404261EBEB
:1017B00041014FF4806404F132045FEA915C3FF42C
:1017C000D8AE4FF003025FEADC0C18BF03325FEAC9
:1017D000DC0C18BF033202EBDC02C2F1200300FA7A
:1017E00003FC20FA02F001FA03FE40EA0E0021FA9F
:1017F00002F11444BDE600BF70B54FF0FF0C4CF48D
:10180000E06C1CEA11541DBF1CEA135594EA0C0F3E
:1018100095EA0C0F00F0DEF82C4481EA030621EA79
:101820004C5123EA4C5350EA013518BF52EA0335B4
:1018300041F4801143F4801338D0A0FB02CE4FF066
:101840000005E1FB02E506F00042E0FB03E54FF096
:101850000006E1FB03569CF0000F18BF4EF0010E8E
:10186000A4F1FF04B6F5007F64F5407404D25FEA8A
:101870004E0E6D4146EB060642EAC62141EA55513D
:101880004FEAC52040EA5E504FEACE2EB4F1FD0C7F
:1018900088BFBCF5E06F1ED8BEF1004F08BF5FEAFD
:1018A000500E50F1000041EB045170BD06F00046AF
:1018B00046EA010140EA020081EA0301B4EB5C045C
:1018C000C2BFD4EB0C0541EA045170BD41F4801154
:1018D0004FF0000E013C00F3AB8014F1360FDEBF79
:1018E000002001F0004170BDC4F10004203C35DA55
:1018F0000C341BDC04F11404C4F1200500FA05F3D8
:1019000020FA04F001FA05F240EA020001F0004278
:1019100021F0004110EBD37021FA04F642EB0601EE
:101920005EEA430E08BF20EAD37070BDC4F10C0418
:10193000C4F1200500FA04F320FA05F001FA04F2DC
:1019400040EA020001F0004110EBD37041F10001C8
:101950005EEA430E08BF20EAD37070BDC4F12005D3
:1019600000FA05F24EEA020E20FA04F301FA05F23B
:1019700043EA020321FA04F001F0004121FA04F2E3
:1019800020EA020000EBD3705EEA430E08BF20EAB3
:10199000D37070BD94F0000F0FD101F000464000ED
:1019A00041EB010111F4801F08BF013CF7D041EA6F
:1019B000060195F0000F18BF704703F00046520073
:1019C00043EB030313F4801F08BF013DF7D043EA44
:1019D0000603704794EA0C0F0CEA135518BF95EAFA
:1019E0000C0F0CD050EA410618BF52EA4306D1D181
:1019F00081EA030101F000414FF0000070BD50EAA0
:101A0000410606BF1046194652EA430619D094EA29
:101A10000C0F02D150EA013613D195EA0C0F05D113
:101A200052EA03361CBF104619460AD181EA030167
:101A300001F0004141F0FE4141F470014FF000001F
:101A400070BD41F0FE4141F4780170BD70B54FF0BA
:101A5000FF0C4CF4E06C1CEA11541DBF1CEA13553A
:101A600094EA0C0F95EA0C0F00F0A7F8A4EB05041C
:101A700081EA030E52EA03354FEA013100F0888013
:101A80004FEA03334FF0805545EA131343EA1263DC
:101A90004FEA022245EA111545EA10654FEA002691
:101AA0000EF000419D4208BF964244F1FD0404F54A
:101AB000407402D25B084FEA3202B61A65EB0305A6
:101AC0005B084FEA32024FF480104FF4002CB6EB63
:101AD000020E75EB030E22BFB61A754640EA0C00E3
:101AE0005B084FEA3202B6EB020E75EB030E22BF23
:101AF000B61A754640EA5C005B084FEA3202B6EB64
:101B0000020E75EB030E22BFB61A754640EA9C0022
:101B10005B084FEA3202B6EB020E75EB030E22BFF2
:101B2000B61A754640EADC0055EA060E18D04FEAB0
:101B3000051545EA16754FEA06164FEAC30343EA50
:101B400052734FEAC2025FEA1C1CC0D111F4801F1D
:101B50000BD141EA00014FF000004FF0004CB6E716
:101B600011F4801F04BF01430020B4F1FD0C88BFB5
:101B7000BCF5E06F3FF6AFAEB5EB030C04BFB6EBC0
:101B8000020C5FEA500C50F1000041EB045170BDB3
:101B90000EF0004E4EEA113114EB5C04C2BFD4EBE0
:101BA0000C0541EA045170BD41F480114FF0000E64
:101BB000013C90E645EA060E8DE60CEA135594EAE0
:101BC0000C0F08BF95EA0C0F3FF43BAF94EA0C0FE3
:101BD0000AD150EA01347FF434AF95EA0C0F7FF458
:101BE00025AF104619462CE795EA0C0F06D152EAAC
:101BF00003353FF4FDAE1046194622E750EA410690
:101C000018BF52EA43067FF4C5AE50EA41047FF4A0
:101C10000DAF52EA43057FF4EBAE12E74FF0FF3C05
:101C200006E000BF4FF0010C02E000BF4FF0010CD6
:101C30004DF804CD4FEA410C7FEA6C5C4FEA430C4F
:101C400018BF7FEA6C5C1BD001B050EA410C0CBF9E
:101C500052EA430C91EA030F02BF90EA020F002000
:101C6000704710F1000F91EA030F58BF994208BF67
:101C700090422CBFD8176FEAE37040F00100704724
:101C80004FEA410C7FEA6C5C02D150EA013C07D17B
:101C90004FEA430C7FEA6C5CD6D152EA033CD3D0C6
:101CA0005DF8040B704700BF8446104662468C46C0
:101CB0001946634600E000BF01B5FFF7B7FF0028F3
:101CC00048BF10F1000F01BD4DF808EDFFF7F4FF1C
:101CD0000CBF012000205DF808FB00BF4DF808EDA7
:101CE000FFF7EAFF34BF012000205DF808FB00BFCA
:101CF0004DF808EDFFF7E0FF94BF012000205DF8EC
:101D000008FB00BF4DF808EDFFF7CEFF94BF0120A0
:101D100000205DF808FB00BF4DF808EDFFF7C4FF99
:101D200034BF012000205DF808FB00BF4FEA410CE2
:101D30007FEA6C5C02D150EA013C0AD14FEA430CC5
:101D40007FEA6C5C02D152EA033C02D14FF0000002
:101D500070474FF0010070474FEA410212F5001240
:101D600015D211D56FF47873B3EB625212D94FEAE2
:101D7000C12343F0004343EA505311F0004F23FACC
:101D800002F018BF404270474FF00000704750EA21
:101D9000013005D111F0004008BF6FF000407047DE
:101DA0004FF00000704700BF4FEA4102B2F1E0433C
:101DB00024BFB3F5001CDCF1FE5C0DD901F0004C32
:101DC0004FEAC0024CEA5070B2F1004F40EB830082
:101DD00008BF20F00100704711F0804F21D113F1AE
:101DE0003872BCBF01F00040704741F480114FEAE7
:101DF0005252C2F11802C2F1200C10FA0CF320FA70
:101E000002F018BF40F001004FEAC1234FEAD3238C
:101E100003FA0CFC40EA0C0023FA02F34FEA4303F6
:101E2000CCE77FEA625307D150EA01331EBF4FF07F
:101E3000FE4040F44000704701F0004040F0FE409A
:101E400040F40000704700BF80F0004002E000BF97
:101E500081F0004142001FBF5FEA410392EA030F95
:101E60007FEA226C7FEA236C6AD04FEA1262D2EBDF
:101E70001363C1BFD218414048404140B8BF5B42E4
:101E8000192B88BF704710F0004F40F4000020F07D
:101E90007F4018BF404211F0004F41F4000121F093
:101EA0007F4118BF494292EA030F3FD0A2F10102DD
:101EB00041FA03FC10EB0C00C3F1200301FA03F11B
:101EC00000F0004302D5494260EB4000B0F5000F3E
:101ED00013D3B0F1807F06D340084FEA310102F1FD
:101EE0000102FE2A51D2B1F1004F40EBC25008BFAF
:101EF00020F0010040EA03007047490040EB000079
:101F0000013A28BFB0F5000FEDD2B0FA80FCACF179
:101F1000080CB2EB0C0200FA0CF0AABF00EBC250A6
:101F200052421843BCBFD0401843704792F0000F94
:101F300081F4000106BF80F400000132013BB5E7E7
:101F40004FEA41037FEA226C18BF7FEA236C21D05D
:101F500092EA030F04D092F0000F08BF08467047C2
:101F600090EA010F1CBF0020704712F07F4F04D190
:101F7000400028BF40F00040704712F100723CBFA3
:101F800000F50000704700F0004343F0FE4040F4CD
:101F9000000070477FEA226216BF08467FEA23638B
:101FA0000146420206BF5FEA412390EA010F40F476
:101FB000800070474FF0000304E000BF10F00043C2
:101FC00048BF40425FEA000C08BF704743F09643A9
:101FD00001464FF000001CE050EA010208BF7047C4
:101FE0004FF000030AE000BF50EA010208BF70474B
:101FF00011F0004302D5404261EB41015FEA010C60
:1020000002BF84460146002043F0B64308BFA3F157
:102010008053A3F50003BCFA8CF2083AA3EBC25339
:1020200010DB01FA02FC634400FA02FCC2F1200258
:10203000BCF1004F20FA02F243EB020008BF20F08F
:102040000100704702F1200201FA02FCC2F12002F5
:1020500050EA4C0021FA02F243EB020008BF20EAEA
:10206000DC7070474FF0FF0C1CEAD0521EBF1CEA18
:10207000D15392EA0C0F93EA0C0F6FD01A4480EA06
:10208000010C400218BF5FEA41211ED04FF00063EF
:1020900043EA501043EA5111A0FB01310CF000401B
:1020A000B1F5000F3EBF490041EAD3715B0040EA41
:1020B000010062F17F02FD2A1DD8B3F1004F40EB11
:1020C000C25008BF20F00100704790F0000F0CF0E4
:1020D000004C08BF49024CEA502040EA51207F3AA8
:1020E000C2BFD2F1FF0340EAC250704740F4000083
:1020F0004FF00003013A5DDC12F1190FDCBF00F074
:1021000000407047C2F10002410021FA02F1C2F121
:10211000200200FA02FC5FEA310040F1000053EABD
:102120004C0308BF20EADC70704792F0000F00F00B
:10213000004C02BF400010F4000F013AF9D040EA11
:102140000C0093F0000F01F0004C02BF490011F4A5
:10215000000F013BF9D041EA0C018FE70CEAD153A3
:1021600092EA0C0F18BF93EA0C0F0AD030F0004C23
:1021700018BF31F0004CD8D180EA010000F00040D7
:10218000704790F0000F17BF90F0004F084691F095
:10219000000F91F0004F14D092EA0C0F01D14202CF
:1021A0000FD193EA0C0F03D14B0218BF084608D198
:1021B00080EA010000F0004040F0FE4040F40000E2
:1021C000704740F0FE4040F4400070474FF0FF0C75
:1021D0001CEAD0521EBF1CEAD15392EA0C0F93EABC
:1021E0000C0F69D0A2EB030280EA010C49024FEA0E
:1021F000402037D04FF0805343EA111143EA1013C7
:102200000CF000408B4238BF5B0042F17D024FF47E
:10221000000C8B4224BF5B1A40EA0C00B3EB510F59
:1022200024BFA3EB510340EA5C00B3EB910F24BF42
:10223000A3EB910340EA9C00B3EBD10F24BFA3EBC7
:10224000D10340EADC001B0118BF5FEA1C1CE0D18F
:10225000FD2A3FF650AF8B4240EBC25008BF20F042
:10226000010070470CF0004C4CEA50207F32C2BF96
:10227000D2F1FF0340EAC250704740F400004FF033
:102280000003013A37E792F0000F00F0004C02BF64
:10229000400010F4000F013AF9D040EA0C0093F02E
:1022A000000F01F0004C02BF490011F4000F013B88
:1022B000F9D041EA0C0195E70CEAD15392EA0C0FF0
:1022C00008D142027FF47DAF93EA0C0F7FF470AF28
:1022D000084676E793EA0C0F04D14B023FF44CAF6B
:1022E00008466EE730F0004C18BF31F0004CCAD100
:1022F00030F000427FF45CAF31F000437FF43CAF3C
:102300005FE700BF4FF0FF3C06E000BF4FF0010C5D
:1023100002E000BF4FF0010C4DF804CD4FEA40023F
:102320004FEA41037FEA226C18BF7FEA236C11D089
:1023300001B052EA530C18BF90EA010F58BFB2EB3C
:10234000030088BFC81738BF6FEAE17018BF40F0BC
:10235000010070477FEA226C02D15FEA402C05D170
:102360007FEA236CE4D15FEA412CE1D05DF8040BF5
:10237000704700BF844608466146FFE70FB5FFF788
:10238000C9FF002848BF10F1000F0FBD4DF808ED40
:10239000FFF7F4FF0CBF012000205DF808FB00BF31
:1023A0004DF808EDFFF7EAFF34BF012000205DF88B
:1023B00008FB00BF4DF808EDFFF7E0FF94BF0120D8
:1023C00000205DF808FB00BF4DF808EDFFF7D2FFD5
:1023D00094BF012000205DF808FB00BF4DF808ED18
:1023E000FFF7C8FF34BF012000205DF808FB00BFE5
:1023F0004FEA40024FEA41037FEA226C02D15FEAD2
:10240000402C08D17FEA236C02D15FEA412C02D133
:102410004FF0000070474FF0010070474FEA400254
:10242000B2F1FE4F0FD34FF09E03B3EB12620DD902
:102430004FEA002343F0004310F0004F23FA02F06C
:1024400018BF404270474FF00000704712F1610F13
:1024500001D1420205D110F0004008BF6FF00040EA
:1024600070474FF00000704742000ED2B2F1FE4FAD
:102470000BD34FF09E03B3EB126209D44FEA002353
:1024800043F0004323FA02F070474FF0000070471A
:1024900012F1610F01D1420202D14FF0FF307047BB
:1024A0004FF00000704700BF53B94AB9002908BF78
:1024B00000281CBF4FF0FF314FF0FF3000F06AB929
:1024C000ADF1080C6DE904CE00F006F8DDF804E08B
:1024D000DDE9022304B070472DE9F047089D0C4662
:1024E000002B4ED194468C458646B2FA82F262D9D0
:1024F0004AB1C2F12003914020FA03F30CFA02FC26
:10250000194300FA02FE4FEA1C471FFA8CF6B1FB92
:10251000F7F44FEA1E4307FB141143EA014304FB9F
:1025200006F199420AD91CEB030304F1FF3080F055
:102530001281994240F20F81023C6344591A1FFAFA
:102540008EF3B1FBF7F007FB101143EA014300FBE8
:1025500006F69E420AD91CEB030300F1FF3180F01E
:10256000FC809E4240F2F980634402389B1B40EAA3
:10257000044000211DB1D3400022C5E90032BDE86E
:10258000F0878B4205D90DB1C5E90001002108464D
:10259000F5E7B3FA83F1002946D1A34202D3904272
:1025A000C0F0F080861A64EB03030120002DE6D012
:1025B000C5E90063E3E7002A40F09080A1EB0C043A
:1025C0004FEA1C481FFA8CF70121B4FBF8F64FEADA
:1025D0001E4308FB164443EA044307FB06F09842F7
:1025E00008D91CEB030306F1FF3402D2984200F233
:1025F000CD8026461C1A1FFA8EF3B4FBF8F008FBB8
:10260000104443EA044300FB07F79F4208D91CEB40
:10261000030300F1FF3402D29F4200F2B080204653
:10262000DB1B40EA0640A5E7C1F120068B4022FAF9
:1026300006F71F4320FA06FC04FA01F343EA0C03F1
:10264000F44000FA01F8380C4FEA1349B4FBF0FEED
:102650001FFA87FC00FB1E4449EA04440EFB0CF9F8
:10266000A14502FA01F20AD93C190EF1FF3A80F0B5
:102670008480A14540F28180AEF1020E3C44A4EB7F
:1026800009041FFA83F9B4FBF0F300FB134449EA91
:10269000044403FB0CFCA44507D93C1903F1FF30AB
:1026A00067D2A44565D9023B3C4443EA0E40A0FBF7
:1026B0000293A4EB0C049C42CE469C4651D34ED0D0
:1026C00055B1B8EB0E0364EB0C0404FA06F6CB40EC
:1026D0001E43CC40C5E90064002150E7C2F120034D
:1026E00020FA03F10CFA02FC24FA03F394400C43A1
:1026F0004FEA1C4800FA02FE1FFA8CF7B3FBF8F011
:1027000008FB1031230C43EA014300FB07F1994217
:1027100008D91CEB030300F1FF362CD299422AD9C9
:10272000023863445B1AA4B2B3FBF8F108FB11331F
:1027300044EA034401FB07F3A34208D91CEB040459
:1027400001F1FF3613D2A34211D902396444E41ACD
:1027500041EA004139E70446F0E6084606E7C84585
:10276000AED2B9EB020E63EB070C0138A8E7314695
:10277000EDE7034699E73046D4E7D6467FE7634462
:1027800002384DE70646234608460FE7023E6344FB
:1027900030E700BF704700BF00487047001BB74BD1
:1027A00070B50C4601F0F2F9104E0546082130468E
:1027B00006F056F8012804D001F0E8F9431BA342C3
:1027C00007D30821094806F04BF8431E58425841E8
:1027D00070BD72B60821304606F042F8012800D0DC
:1027E00030BF62B6BFF36F8FE0E700BF0004004860
:1027F00008B5002210214FF0904006F037F8054848
:102800000022202106F032F8BDE80840022001F045
:10281000C5B900BF0004004810B50C4C01221021BE
:10282000204606F023F8052001F0B8F920460122E1
:10283000202106F01BF84FF090400122102106F0F5
:1028400015F8BDE81040022001F0A8B900040048C6
:1028500070B54FF090400C46164610210022144DE2
:1028600006F004F800232B701248B3B2224621462A
:1028700007F0F0F9D8B901F089F941F2873604463A
:102880002B783BB1BDE87040012210214FF0904001
:1028900005F0ECBF01F07AF9031BB342F2D872B62F
:1028A0002B7803B930BF62B6BFF36F8FE8E770BD16
:1028B000DD080020400A0020014B01221A707047F9
:1028C000DD08002000487047E86C030813B5114B81
:1028D0000446186800909B88ADF804300120FFF78B
:1028E0009BFF062269460120FFF7B2FF0120FFF798
:1028F0007FFF9DF80430112B08D19DF80520122A86
:1029000004D101202370627002B010BD00231A466A
:102910001846F7E7B02B03080CB4F0B5ADB032ABF6
:1029200006AF53F8042B059305460E46384696210C
:102930002CF028FE9528C1BF42F62E63ADF8AA30D0
:102940002E23ADF8AC3000F035F83C24042D4FF4C4
:102950007A7E1449B0FBFEFCB0FBF1F14EF6602329
:10296000B0FBF3F3B3FBF4F204FB1232BCFBF4F361
:1029700004FB13C30EFB1C049ABF0B48405D3F20B1
:10298000CDE90040CDE9026708482CF07BFD084BFB
:102990001B6898682CF0A0FC2DB0BDE8F04002B098
:1029A000704700BF80EE3600466D0308246D0308B3
:1029B000EC06002001F0EAB81348144A08B54FF0BD
:1029C0000043C0E900230422426101220023C261C6
:1029D0004FF480510722C0E90233C0E90933C0E94E
:1029E0000C1203610383837680F8203080F82C304A
:1029F000826380F83C30C36404F08AFE18B1BDE8FD
:102A0000084000F099BB08BDE00800200024014008
:102A10000268084B9A4282B00AD14FF0B0431A6E56
:102A200042F400721A661B6E03F400730193019B5B
:102A300002B07047002401400268054B9A4201BF72
:102A40004FF0B042136E23F400731366704700BF5B
:102A50000024014030B585B000240546CDE901448D
:102A60000394FFF7A9FF144805F0E6F908B100F058
:102A700063FB1148039401A9CDE9015404F0A6FFBA
:102A800008B100F059FB0C4805F000F908B100F05E
:102A900053FB4FF0FF31084804F03AFF064805F0B9
:102AA000ADF9054804F08EFF0446034805F050F9DF
:102AB000204605B030BD00BFE0080020014B024AAF
:102AC0001A607047E00800200024014008B509485A
:102AD000FFF7C0FF68B1084BB3F8AA304FF6FF729A
:102AE000934216BF40F6E442044B5343B3FBF0F36A
:102AF00098B208BD002000B40075FF1FD8084C0034
:102B000013B50023ADF80630FFF7E0FF044619487F
:102B1000FFF7A0FF184BB3F8C820B3F8A8108A42FB
:102B200004FB00F018D040F6E443B0FBF3F364205C
:102B30005B1A4343521A93FBF2F31E331BB2ADF8F8
:102B40000630BDF806305BB21B02ADF80630BDF8AA
:102B5000060000B202B010BD4FF47A7240F6FF7367
:102B6000B0FBF3F35343A3F53923A3F50C6340F60D
:102B7000C412E0E7001000B00075FF1F4FF0B04333
:102B800082B09A6A22F480529A629A6C42F480521D
:102B90009A649B6C03F480530193019B002002B064
:102BA00070474FF0B04307B59A6C42F004029A6444
:102BB0009A6C02F004020192019A9A6C42F00102AE
:102BC0009A649B6C002203F00103114600930B20D2
:102BD000009B05F0CFF90B2005F0FEF9002211460D
:102BE0000C2005F0C7F90C2005F0F6F9002211467B
:102BF0000D2005F0BFF90D2005F0EEF900220221AD
:102C00000F2005F0B7F90F2005F0E6F90022114674
:102C1000102005F0AFF9102005F0DEF90022114672
:102C2000112005F0A7F9112003B05DF804EB05F0C1
:102C3000D3B9000008B505F013FC10B16FF0040023
:102C400008BD064B9A6942F040429A614CF2FA3252
:102C50001A6105F017FC0028F2D0EFE70040005899
:102C6000F0B585B000230D4600930646A8B3FFF7E4
:102C7000E1FF044670BB05F0F3FB88BB1A481B4A12
:102C800002230193D0F8E01506F1784302EA81218E
:102C9000B3FBF1F701FB1733DB0A0293D0F8E00531
:102CA00005F178410139314402EA8022B1FBF2F0AA
:102CB00002FB1011C3EBD1230133694601A8039332
:102CC00005F060FC20B1022814BF6FF0010401245C
:102CD00005F0D8FB204605B0F0BD6FF00504F9E71C
:102CE0006FF00404F6E700BF0070FF1F00FCFF0355
:102CF000014B186000207047440900202DE9F04F77
:102D0000B0F1006F89B006460F469046C0F0C08013
:102D1000DFF89091644DD9F8E03505EA832303F19B
:102D20000063013B984200F2B380002900F0B380B9
:102D300040EA02035B0740F0AE80FFF77BFF0446EA
:102D400090BB05F08DFB002840F0A880D9F8E01575
:102D5000009705EA812106F17842B2FBF1F301FB0D
:102D6000132208F17843013B3344B3FBF1F001FB3C
:102D70001033DB0A01334FEAD22AA3EBD222012A15
:102D8000039388BFC6F30A050AF58037C6F1080326
:102D90008CBFC5F500654546FF02B3460693039B0D
:102DA0009A4505D305F06EFB204609B0BDE8F08FCB
:102DB000A6F10803069A1A4495421CD8009B049574
:102DC0000193CDF814B04FF00009059B09EB030106
:102DD000049B99453DD3009BAB442B44A8EB0505D0
:102DE000B5F5006F009328BF4FF400650AF1010AA2
:102DF00007F50067D3E753F8081F5A68B2F1FF3FA1
:102E000008BFB1F1FF3FD5D0284B186810B96FF05B
:102E10000504C7E727B14FF40062394612F0B4FD4C
:102E2000DFF888900099D9F80030CBF30A001844F5
:102E3000AAB212F0A9FD4FF400613846FFF710FF67
:102E400000BBD9F8003001934FF400630597049359
:102E5000B9E7019B07914B4402930120D3E900237A
:102E600005F04AFB88B90799019BD1E9000259F89E
:102E70000310029B5B689A4208BF884205D109F1A2
:102E80000809A2E76FF001048CE76FF0030489E7FB
:102E90004FF0FF3488E76FF0050485E76FF0040416
:102EA00082E700BF0070FF1F00FCFF034409002001
:102EB000B1F1006F70B510D30B4BD3F8E0650B4B3D
:102EC00003EA862303F10063013B994205D838B138
:102ED00092B212F059FD002070BD4FF0FF30FBE7B9
:102EE0006FF00500F8E700BF0070FF1F00FCFF0354
:102EF000B0F1006F10B40DD3084BD3F8E045084B88
:102F000003EA842303F10063013B984202D810BC1A
:102F1000FFF7A6BE4FF0FF3010BC70470070FF1FD8
:102F200000FCFF034FF0B04382B0DA6C0243DA6476
:102F3000DB6C03400193019B02B070472DE9F04127
:102F400086B01422002101A82CF03AFB0220464E44
:102F5000FFF7E8FF0420FFF7E5FF0120FFF7E2FF9E
:102F600004213046002205F081FC002210214FF0A0
:102F7000904005F07BFC04230024012502270DEB83
:102F800003013046CDE901354FF01008CDE9034784
:102F900005F046FB01A93046CDE90185CDE9037472
:102FA00005F03EFB202301A93046CDE90135CDE9EE
:102FB000037405F035FB01A94FF09040CDE9018580
:102FC000CDE9034405F02CFB08224FF4881301A936
:102FD0003046CDE901234FF00308CDE9034705F062
:102FE0001FFB4FF4441301A94FF09040CDE901833A
:102FF000CDE9035705F014FB4FF4405301A93046C7
:10300000CDE90135CDE9034805F00AFB4FF404137F
:103010004021CDE901131548039501A905F000FBF6
:1030200022460F21062004F0A5FF062004F0D4FF5D
:1030300022460F21072004F09DFF072004F0CCFF5B
:1030400022462146092004F095FF092004F0C4FF20
:1030500022462146092004F08DFF092004F0BCFF20
:1030600006B0BDE8F08100BF000400480008004839
:1030700000B59BB04822002108A82CF0A1FA182224
:10308000002102A82CF09CFA05F00AFC4FF0B04297
:103090000120D2F8903023F01803C2F89030D2F813
:1030A000003423F4C06343F40073C2F80034D2F850
:1030B000003403F4C0630193019B2423089381230C
:1030C0000B930023CDE91003B02208A8CDE9122309
:1030D00005F05EFD08B172B6FEE74F23CDE9023080
:1030E000CDE90400CDE90600022102A805F0EAFFBF
:1030F00008B172B6FEE71BB05DF804FB08B504F03A
:10310000B5FAFFF7B5FFFFF719FFFFF74AFD00F02B
:10311000E3FF00F075FE00F089F806480122042163
:1031200005F0A4FB02F0D8FB00F010FC02F0DBFB82
:10313000FCE700BF0004004872B6FEE700B58DB0A2
:103140002C22002101A82CF03BFA1748174B0360F2
:103150001F2383604FF080420023C0E90433C0E99D
:10316000072383614FF48073436206F051FA08B17C
:10317000FFF7E2FF0C4806F077FB08B1FFF7DCFF32
:103180004FF0005300220793074808924FF48073D2
:1031900001A9029206920B9306F09AFA08B1FFF782
:1031A000CBFF0DB05DF804FB48090020002800406B
:1031B00010B5044690B03822002102A82CF000FA85
:1031C0002268194B9A422CD14FF48033029302A803
:1031D0004FF480730F9306F099F808B1FFF7ACFF36
:1031E0004FF0B0430220D3F8902042F40042C3F8DD
:1031F00090209A6D42F480629A659B6D002203F4E0
:10320000806311460193019B04F0B4FE022004F098
:10321000E3FE00222A20114604F0ACFE2A2004F02E
:10322000DBFE10B010BD00BF002800401148124A5C
:1032300008B54FF48273C0E9002300234FF4E06225
:10324000C0E902324FF400712822C0E906120722B9
:10325000C0E90433C0E90833C0E90B2383620823C3
:10326000436306F071FC18B1BDE80840FFF764BF86
:1032700008BD00BF400A002000300140F0B50546FF
:1032800089B01422002103A82CF09AF92A68374B40
:103290009A4269D14FF0B04302261A6E42F480522E
:1032A0001A661A6E02F480520292029ADA6C42F0A6
:1032B0000102DA64DA6C02F001020192019ADA6C1E
:1032C00042F00202DA64DB6C03F00203009305248F
:1032D000009B0327D02303A94FF09040CDE903368C
:1032E000CDE9067405F09CF92023CDE903364FF0B3
:1032F0009040002603A90794CDE905671C4C05F012
:103300008FF91C4826620723C4E900038023204666
:10331000C4E90266C4E90436C4E9066604F0BCFEEA
:1033200008B1FFF709FF144AAC65A562134C0823E6
:10333000C4E900231021002380222046C4E902139F
:10334000C4E90423C4E90633236204F0A5FE08B1EE
:10335000FFF7F2FE002222206C651146A56204F000
:1033600009FE222004F038FE09B0F0BD0030014013
:10337000E00900201C0002403000024080090020CB
:103380007047000008B504F087F9044B0120C3F82A
:103390008800BDE8084005F0DBBA00BF0004005813
:1033A00008B504F080F900F0A7FFFFF7C7FDFFF7AD
:1033B000F8FB00F025FDBDE80840FFF737BF08B572
:1033C00004F071F9FFF7BAFDFFF7EBFBBDE8084029
:1033D000FFF72CBF08B504F05FF9BDE808400121F4
:1033E000002005F065BA70477047FEE7FEE7FEE78C
:1033F000FEE7FEE77047704770477047014806F0E8
:1034000059BA00BF48090020024B0120187005F08E
:103410003BBA00BF921F0020024B012202201A700B
:1034200005F032BA911F0020082005F02DBA0000E7
:10343000014804F0A7BF00BF4C140020014804F06D
:10344000A1BF00BFE0090020014804F09BBF00BFFE
:103450008009002070470000014804F093BF00BFBE
:103460000015002070470000014806F0E1BD00BFD4
:10347000400A0020014807F05FBF00BF6015002030
:10348000014806F04BB800BF48090020014807F08A
:1034900060B800BF381400202DE9F04389B08046A1
:1034A0000020109E0790894615461F46FCF7C0FE77
:1034B000F0B9104CCDE90090CDE9020407AB0E48FD
:1034C0000593142304933A46434629460068FCF7C3
:1034D00079FF2346324604F1140153F8044B42F8B5
:1034E000044B8B42F9D1079B337509B0BDE8F083DB
:1034F0000120FAE7BA0A0020D86C03087FB5124C05
:1035000000253C2302A86375CDE90255257500F01E
:10351000E7FA042303AA009412210C48FFF7BCFF2A
:103520000B49142220462CF03BF80646B0FA80F0F6
:1035300040096075074B00902A462946022012F088
:103540001DF9304604B070BDA40A0020826D030846
:1035500056220020646D0308034A044840F21B53BE
:10356000002107F019BD00BFCE0A0020AC140020D6
:10357000312BF0B52DD81825102415FB0343194D18
:1035800000244FF0800C4CFA04F6A3F110073142EE
:1035900005EB470714BF4FF0240E4FF0140EA7F8A9
:1035A00006E0A3F10807304205EB470714BF4FF0D0
:1035B000240E4FF0140E0134324205EB4306A7F8F7
:1035C00006E00CBF14272427082CF78003F1010321
:1035D000D9D1054B1B781BB9BDE8F040FFF7BCBF44
:1035E000F0BD00BFCE0A0020FC1F002010B5002453
:1035F0000022E3B2114610460134FFF7B9FF322C26
:10360000F6D1BDE81040FFF7A7BF000070B5044633
:103610000D46FFF7EBFF0F4B04EB440400261C4460
:10362000142000F0BBFAA2786178207812FB05F232
:1036300011FB05F110FB05F0F3B2D2B2C9B2C0B272
:103640000136FFF795FF322EEAD1BDE870400A201F
:1036500000F0A4BA080000202DE9F04106460F460C
:103660002048904600214FF416622BF0A9FF1E4A15
:1036700010254FF0800C2B4600244CFA04F1A3F1E6
:1036800010000F4202EB400014BF4FF0240E4FF029
:10369000140EA0F806E0A3F108000E4202EB400071
:1036A00014BF4FF0240E4FF0140E013418EA010F2E
:1036B00002EB4301A0F806E00CBF14202420082CE4
:1036C000C88003F10103D8D11835B5F5986FD2D170
:1036D000064B1B781BB9BDE8F041FFF73DBFBDE8C5
:1036E000F08100BFD40A0020CE0A0020FC1F002079
:1036F00000F00F000B4607281ED8DFE800F0040793
:103700000A0F1316191B0022114600E00022104672
:1037100002E0002211461846FFF79EBF0A4600212C
:103720000020F9E700220846F6E70A460021EEE706
:103730000A46F5E70A46E7E770470000024B1878AB
:10374000024B1978FFF7D4BF0600002000000020CC
:1037500070B56A496A4B0A78D2B20B2A2ED8DFE8D4
:1037600012F00C0011001300190020005600810017
:103770009400A300B200B200B200624A1278D2B242
:103780001A701BE00022FBE75F480078012808BFA1
:103790000122F5E75D4A1078002840F0818001227F
:1037A000EEE75A485A4A04780CBB5A4C2478012C4C
:1037B0001DD11478012CE5B219D11D700A78564D2F
:1037C000012A05D0554E317801F0FF0200297FD043
:1037D00000221A70524B1A702A70FFF707FF514BE4
:1037E0001B781BB9504B1A7802B91B7870BD007852
:1037F000012805D04748007810B110780028DDD1A5
:10380000022018701278002AD8D12322B8E73F4846
:103810003F4A04789CB93F4C2478012C0FD114788E
:10382000012CE5B20BD11D70404A1278012AD0B2AA
:1038300016D00328C2D1042239480270A0E70078CC
:10384000012805D03348007810B110780028EBD15A
:10385000022018701278002AE6D123221A70E3E7BA
:103860002322E9E7294A107830B92748007801284F
:10387000C4B201D11C70A1E71278012A03D0224AF8
:103880001278002A9AD102227AE7204A107818B9D1
:1038900027480078002882D01278012AF3D0244AE1
:1038A0001278012A8AD1EEE7184A107820B9214807
:1038B000007804283FF473AF1278012AE3D01D4A40
:1038C0001278052AEEE71B4A10780428F8D166E73B
:1038D00028781978884282D0317809B91A78D2B21A
:1038E0000F4C154B227020781978FFF701FF3378C1
:1038F00003B123782378DBB22B7070E70601002038
:10390000070000200400002055220020831F002013
:10391000090100200A01002001000020FC1F0020F6
:1039200006000020841F0020851F00200A160020AA
:10393000821F0020811F0020000000200248036831
:103940000021596307F0A2BBAC140020002270B51F
:103950000F4B1146032011F011FF01240A252946BF
:1039600020461435FFF7C4FEEDB2322000F016F900
:103970006E2DF4D10134E4B2FFF738FE082CEDD1FE
:103980000022BDE87040034B1146032011F0F6BE43
:10399000946D0308C76D0308054808B50823036044
:1039A00006F0F4FB18B1BDE80840FFF7C5BB08BD41
:1039B000381400204FF0B04307B55A6E42F00102B0
:1039C0005A665B6E002203F0010301931146322018
:1039D000019B04F0CFFA322003B05DF804EB04F051
:1039E000FBBA00000CB407B5054A05AB10210193E2
:1039F00012F096FB03B05DF804EB02B0704700BF15
:103A0000FD6D030830B585B0044602A80D4612F0DE
:103A10001FF9BDF90C30064A00931021029B204685
:103A2000FFF7E0FF2046FDF723FD288005B030BDFD
:103A3000FD6D03084FF0B04210B5936823F40043C6
:103A4000936012F021FA104B01241C7000F0ACF8C6
:103A500011F02AFE0D4811F041FE0D4B4FF40042CB
:103A60001A61022011F040FEFFF728F800F002F979
:103A700011F034FF2146204611F050FF2146204628
:103A8000BDE8104011F034BF44140020053A00088E
:103A90000040005811F058BF08B5FFF717F840F67E
:103AA000B83398420CD8B0F5E16F0BD3FE23A0F5E4
:103AB000E16058434FF49663B0FBF3F0C0B208BD29
:103AC000FE20FCE70020FAE77FB5684600F0B6F874
:103AD0000198FEF7A3FC00B207B05DF804FB0000FC
:103AE000194A38B5D2F88035591C044619D103F06B
:103AF000E1FD054603F0EAFD054403F0E1FD2B0E70
:103B0000E3712B0CA3712B0A6371030EE370C0F3F6
:103B10000742C0F307232571C0B2A2706370207002
:103B200038BD190AC3718171190C1B0E41710371E3
:103B3000D2F88435C370D2F88405C0F30722C0F3ED
:103B40000743000EE9E700BF0070FF1F38B5094BBF
:103B5000D3F8803503600133054609D103F0AAFD8F
:103B6000044603F0ADFD444003F0B0FD44402C603A
:103B700038BD00BF0070FF1F0121022011F0B8BE48
:103B80000021022011F0B4BE00207047024B1878CB
:103B900008B100F0DDB970474414002082B00190F4
:103BA000019802B000F070BAF0B5224A224CD2F867
:103BB000903043F4804389B0C2F8903003F08CFD1C
:103BC00003F092FD03F098FD012304930323069371
:103BD00000254FF0B04305950795DA6C42F00202DC
:103BE000DA64DA6C02F002020292029ADA6C42F0B3
:103BF0000202DA64DB6C03F0020301934FF4805796
:103C000003A92046019B03974FF4005604F008FDDA
:103C100003A92046039604F003FD2A4639462046B0
:103C200004F024FE2A463146204604F01FFE09B067
:103C3000F0BD00BF000800580004004810B504465D
:103C4000FEF75EFF074BA36040F30F20FEF7B6F9C7
:103C5000054B064A2360064B6060C4E9032300203D
:103C600010BD00BF0000484200007A440D093E002C
:103C7000AB030500002070470120704708B52BF00A
:103C800001FD162303604FF0FF3008BD08B52BF08F
:103C9000F9FC16230360FEE770B50D4614460E4688
:103CA000731B9C4201DC204670BDAFF3008006F818
:103CB000010BF5E730B5104600234FF06042834218
:103CC00000DB30BDD2F8804EE50707D5D2F8004EB4
:103CD000E40703D5CC5C156815B114700133EEE729
:103CE00000BFF8E74FF0FF3070474FF400534B60D0
:103CF0000020704701207047002070470B4A116870
:103D000010B5034609B90A491160106809490A4CFF
:103D10000344091B8B4206D92BF0B4FC0C2303602F
:103D20004FF0FF3010BD1360FCE700BF48140020C7
:103D300098420020000001200008000037B5184B11
:103D400002689A42054628D14FF0B043154C1A6ECE
:103D500042F400621A661B6E134A03F40063019377
:103D6000019B1723C4E90023102100238020C4E90C
:103D700002134FF48073C4E904034FF4806C2023D2
:103D8000C4E906C320464FF40053236204F084F9CB
:103D900008B1FFF7D1F96C62A56203B030BD00BF76
:103DA000002C01404C1400200800024010B50446CD
:103DB00086B01422002101A82BF002FC22680F4BD0
:103DC0009A4218D14FF0B04301A9DA6C42F00102D7
:103DD000DA64DB6C03F0010300930222009B4FF4D2
:103DE0008073CDE901324FF090400123CDE90332D9
:103DF000059304F015FC06B010BD00BF002C014077
:103E000010B510229CB0002400210DEB02002BF015
:103E1000D7FB1C22214608A8CDE9014403942BF0CE
:103E2000CFFB342221460FA82BF0CAFB2B482C4B8A
:103E30008460C0E900343B23C0E90334C0E9054491
:103E400006F0F0FD08B1FFF777F94FF480532348EF
:103E5000049304A906F004FF08B1FFF76DF91F48A9
:103E600006F010FE08B1FFF767F900241B48039421
:103E700001A9CDE9014407F00BF908B1FFF75CF99E
:103E8000602316480E94002208A9CDE90834CDE934
:103E90000A44CDE90C4406F05DFE08B1FFF74CF989
:103EA00000234FF40052CDE914230C4813934FF034
:103EB00000720FA9CDE90F33CDE91133CDE91633E7
:103EC000CDE91823CDE91A3307F00EF908B1FFF751
:103ED00033F90248FFF76AFF1CB010BDAC14002094
:103EE000002C0140014B1868704700BFF8140020F7
:103EF0000320704708B501464FF47A720023800210
:103F0000890DFEF7D1FA08BD4FF47A73A0FB0303C5
:103F1000800A40EA83507047034B98689A68904241
:103F2000FBD1C043704700BF0028004008B5FFF731
:103F3000F3FF014B186008BDF814002008B5FFF727
:103F4000EBFF024B1B68C01A08BD00BFF81400202D
:103F5000024B187808B1FFF7DFBF7047FC14002050
:103F600010B5074B074C0122DA654FF480712046EB
:103F700005F09AFA4FF0FF332363002010BD00BF15
:103F8000002800404809002002460021014805F0B1
:103F9000A2BC00BF4809002002460121014805F0EB
:103FA0009ABC00BF4809002010B58CB02C2200211B
:103FB000044601A82BF004FBFFF7D2FF0C4B0D4881
:103FC0001B681C440023089306934FF00053E443FE
:103FD000079301224FF4807301A902940B9305F01B
:103FE00077FB08B1FFF7A8F800200CB010BD00BFA8
:103FF000F81400204809002038B50546FFF78CFF6B
:1040000002210446074805F06DFCC4F309024FF491
:104010007A71A2FB0121920AA30A2A8043EA805006
:1040200038BD00BF480900200148002105F05ABCF6
:10403000480900200148012105F054BC480900202E
:10404000F8B50F4D2E78CEB90E4C4FF0FF372763E1
:10405000FFF774F8FFF784FF4FF48071204605F0F6
:1040600023FA2046276305F0E1FB32462046022171
:1040700005F031FCFFF75AFF01232B700020F8BD3B
:10408000FC14002048090020014610B54FF47A7254
:1040900000238002890DFEF707FA0146FFF73CFF77
:1040A0000446FFF739FF031B8B4200D310BD00BF4E
:1040B000F7E711F0F1BF000010B5064C02212046D1
:1040C00005F010FC0221421C2046BDE8104005F01E
:1040D00002BC00BF480900201648174A08B54FF433
:1040E000E133C0E9002300230C22C0E90233C0E918
:1040F0000523C0E90733C0E90933036107F001FF75
:1041000008B1FFF719F80B48002108F072F808B160
:10411000FFF712F80748002108F08BF808B1FFF705
:104120000BF8044808F045F818B1BDE80840FFF75F
:1041300003B808BD601500200044004070B596B07B
:1041400006461422002103A82BF03AFA3822002157
:1041500008A82BF035FA3268274B9A424AD102233D
:10416000089308A84FF440230A9305F0CFF808B14C
:10417000FEF7E2FF4FF0B04300259A6D1F4C42F46A
:1041800000329A659A6D02F400320292029ADA6C59
:1041900042F00102DA64DB6C03F001030193019B3E
:1041A0000C220223CDE9032303A907234FF09040FB
:1041B0000793CDE9055504F033FA1149256214231C
:1041C000C4E900131023C4E9023520468023C4E962
:1041D0000435C4E9065503F05FFF08B1FEF7ACFFF4
:1041E0002520F46700220221A66203F0C3FE2520E9
:1041F00003F0F2FE16B070BD004400400015002030
:104200008000024002680C4B9A4210B5044612D15D
:104210004FF0B0420C21936D23F4003393654FF0BF
:10422000904004F0A9FAE06F03F0A8FFBDE8104049
:10423000252003F0DFBE10BD0044004008B50A464B
:104240000146024806F0DCFF002008BD6015002092
:1042500013B5114B114C18604FF40013009302ABCF
:1042600013E90600204607F048FF2368DA69D10306
:10427000FCD4DA695202FCD59A68084842F48002FC
:104280009A6007F080FF06490448012207F0EEFE1D
:10429000002002B010BD00BFF41500206015002002
:1042A000FC15002008B5074B1860FEF77AFCFFF7F5
:1042B00013FF054AD2F8803043F00063C2F8803023
:1042C000002008BDF81500200008005808B54FF080
:1042D000B04308489A6B42F400329A639A6B22F416
:1042E00000329A63FFF78EFF112003F083FE002057
:1042F00008BD00BF6015002008B5074807F001FEA3
:1043000008B1FEF719FF054803F0C6FE18B1BDE875
:104310000840FEF711BF08BD601500200015002001
:104320000268044B9A4203D1034B00201B681847D4
:10433000704700BF00440040F815002002680B4B96
:104340009A4210B504460FD1094B1B682BB1D0F827
:10435000902012B907480121984720460549BDE839
:104360001040012207F082BE10BD00BF0044004093
:10437000F4150020FC1500202DE9F04F9DB0FEF74C
:10438000A1FA14F031FB024640B90146644B022009
:1043900011F0F4F901201DB0BDE8F08F012014F0F8
:1043A000CBFB13F0C7F80446039040B90246014620
:1043B0005C4B022011F0E2F914F08AFBEAE75A4D57
:1043C000296813F007FD6968204613F01DFD297A5E
:1043D000204613F04DFD697A204613F07DFD696992
:1043E000204613F009FEE868FEF73EF881B2204649
:1043F00013F08CFD2969204613F054FDA97A20465C
:1044000013F01CFD0221204613F0CEFD10212046A2
:1044100013F00CFE039813F015F90246049040B90E
:104420000146424B022011F0A9F903A813F0E2F86B
:10443000C2E703A813F0DEF8049813F06BFC024601
:1044400040B901463A4B022011F098F904A813F044
:1044500017FAB1E7374EDFF8E0A0DFF8E0B000234D
:1044600033604FF00208049805AB0A2208A913F044
:1044700043FA054628BB02460146314B022011F0A3
:104480007DF930682C49FDF7EDFD4FF07C51FDF7CB
:10449000E9FD3060049813F06DFC044604A813F0A5
:1044A000EFF914F015FB002C3FF474AF002D3FF42E
:1044B00071AF0022234B1146032011F05FF9002059
:1044C00069E731680998FDF7C5FCBDF818903060C0
:1044D00000221D4BCDF800901146022011F04EF93C
:1044E00008AC0027BBB2994504F1080405D8B8F11F
:1044F000010FC6D04FF00108B5E754F8040C51463F
:10450000FDF7B0FDFDF7B0FF019034F8083C0093D3
:1045100000225B461146022011F030F90137E1E735
:10452000586E0308706E030820000020A56E030873
:10453000CC6E0308941F002000007A442F6F0308FC
:10454000F56E0308466F03081E6F030830B5044676
:1045500085B0084614491546FDF784FDFDF75EFF5A
:10456000CCB1114902902846FDF77CFDFDF756FFBE
:104570000E4901902846FDF76BFC0D49FDF726FE1C
:10458000FDF772FF002200900A4B1146032011F044
:10459000F5F805B030BD0090074B224621460320B8
:1045A00011F0ECF8F5E700BF00007A44CDCC4C3FA9
:1045B000CDCCCC3E5F6F03088C6F03082DE9F04F24
:1045C000ADF21C4D4FF40072002106A82AF0F8FF4E
:1045D0004FF40072002186A8B74F2AF0F1FF0024A3
:1045E0003E464FF000082546B1682846FDF732FCEC
:1045F000716805462046FDF72DFC08F10408B8F562
:10460000007F044606F11006EED14FF070512846A7
:10461000FDF728FD4FF0705106462046FDF722FDBC
:104620000024DFF8948282464FF000092546D8F82E
:1046300008003146FDF70CFC0146FDF713FD01466D
:104640002846FDF707FC51460546D8F80400FDF75B
:10465000FFFB0146FDF706FD01462046FDF7FAFB8C
:1046600009F10409B9F5007F044608F11008DED10C
:104670004FF070512846FDF7F5FC8346FDF764F8CE
:104680008E4B00222CF018FFCDE900014FF0705145
:104690002046FDF7E7FCFDF757F8884B00222CF089
:1046A0000BFFFDF781FB06AD82462C464FF000095B
:1046B0004FF00008B968B869FDF7CAFBFDF7AEFE18
:1046C0000028B8BF4042FDF779FC44F8040B0146CE
:1046D0004046FDF7BFFB09F10409B9F5FE7F8046AE
:1046E00007F11007E6D17649FDF770FD06AC0746E5
:1046F0004FF000094FF00008394654F8040BFDF75D
:10470000A7FB0146FDF7AEFC01464846FDF7A2FBBC
:1047100008F101081FFA88F8B8F17F0F8146EBD144
:104720006749FDF753FDFDF70FF8644B00222CF0AD
:10473000C3FECDE9020186ACA04600234FF000097C
:104740002A46296850680493FDF782FBFDF766FE50
:104750000028B8BF4042FDF731FC049B48F8040B29
:1047600001461846FDF776FB09F101091FFA89F9A0
:10477000B9F17E0F05F104050346E1D15149FDF77A
:1047800025FD4FF0000905464FF00008294654F872
:10479000040BFDF75DFB0146FDF764FC014648464E
:1047A000FDF758FB08F101081FFA88F8B8F17E0FF1
:1047B0008146EBD14349FDF709FDFCF7C5FF3F4BAF
:1047C00000222CF079FE404A13889BB2FA2BCDE9E7
:1047D000040100F2D480108880B2FDF7EFFB51464F
:1047E000FDF7F2FD394C08B105232370384B1A78D8
:1047F000384B1B889BB29A4280F08C80364B1A78DB
:10480000364B1B889BB29A4206D235493046FDF79B
:10481000E5FD08B101232370324C334D2388013369
:104820009BB2238023889BB20A2B04BF00232380E2
:1048300022884FF01C0892B208FB02F2DDE9000169
:10484000AE50228892B208FB0252C2F804B0FDF7C3
:10485000ABFAB4F800B0228892B208FB02521FFAF9
:104860008BFB08FB0B5BC2F80CA0B4F800A0CBF8E4
:1048700008004FF086413846FDF7F4FB1FFA8AFA2C
:1048800008FB0A5A2788CAF81000DDE90201FDF783
:104890008BFA4FF08641FDF7E5FB22880B4C92B274
:1048A000BFB208FB075708FB0255217878612976CB
:1048B000DDE904011AE000BF241700200000E03FFA
:1048C0000000FE420000FC423C0000200A160020CE
:1048D00023040020021600202204002000160020DD
:1048E000CDCC4C3F241F00200C160020FDF75CFAB5
:1048F0004FF08641FDF7B6FBFDF7B6FD2B4BC0B27E
:1049000018802378012B05D10022294B1146022063
:1049100010F034FF274F284C3B78DFF8A080012BA4
:1049200024D1DFF89C90274DB9F80030B9F8002069
:104930004FF01C0A9BB292B20AFB03F30AFB02522D
:10494000E8589168FDF786FA3146FDF747FDC0B19A
:10495000022323702378022BD8B204D100221A4BF1
:10496000114610F00BFF2378DBB23B702378DBB2EB
:104970003B70C8F800600DF21C4DBDE8F08F134885
:104980002DE7B9F80030D8F800909BB20AFB035528
:104990003046A968FDF75EFA4946FDF71FFD10B1E4
:1049A00003232370E2E72070E0E700BFFE1500203C
:1049B000A26F0308081600200A1600200416002023
:1049C000241F00200C160020E76F030800007A4324
:1049D0002DE9F04F99B0FDF775FF14F005F8024688
:1049E00040B901469E4B032010F0C8FE012019B0CB
:1049F000BDE8F08F012014F09FF811F0B3FC0446DD
:104A00000C9040B902460146964B032010F0B6FECA
:104A100014F05EF8EAE7944F3B78012BDDB252D0F8
:104A2000022D6FD0002D39D1042112F061F801213F
:104A3000204611F08BFF8D49204611F0BBFF8C49B9
:104A4000204611F09DFF8B49204611F04BFF8A490B
:104A5000204611F061FF0221204612F07DF88749BF
:104A6000204612F05FF8214606A811F0BDFF844AE7
:104A70001392844A14924FF07C53002212A92046CC
:104A8000129315921692179311F0DAFF29462046D9
:104A900011F0FAFF0321204612F010F80C980024C0
:104AA0003C7011F0F5FC02460D9000286DD1764B5C
:104AB0000146032010F062FE0CA811F0C1FC0DA805
:104AC00011F074FDA4E7714E294611F03FFF6749CC
:104AD000204611F06FFFB168204611F003FFF16826
:104AE000204611F019FF716A204611F049FFF16C60
:104AF000204612F017F8664B00221146012010F0F4
:104B00003DFECBE7614D012111F020FFE969204610
:104B100011F050FF696A204611F032FFA968204663
:104B200011F0E0FEE968204611F0F6FEA86CFDF7F2
:104B30009BFC81B2204612F00FF8E96C204611F080
:104B4000F1FF214606A811F04FFF2B6B12936B6B00
:104B50001393AB6B1493EB6B15932B6C169312A9F9
:104B60006B6C1793204611F06BFFA86AFDF77CFC75
:104B7000C1B2204611F088FF286AFDF775FCC1B26A
:104B8000204612F003F8434BB6E711F0A5FD38B903
:104B90000022414B1146032010F0F0FD002026E7D3
:104BA0000026DFF8F8A03E4DDFF8F8904FF04208FD
:104BB00037460D980EA911F0E7FD0246002879D17D
:104BC0000146394B032010F0D9FD0D9811F0A4FDDA
:104BD0000C9D0121284611F0B9FE0421284611F050
:104BE00087FF2249284611F0E5FE2149284611F0A9
:104BF000C7FE2049284611F075FE1F49284611F0CE
:104C00008BFE0221284611F0A7FF1C49284611F00F
:104C100089FF294606A811F0E7FE194A1392234A94
:104C200015924FF07C534FF07E5212A928461692EF
:104C300012931493179311F003FF0021284611F0EB
:104C400023FF0321284611F039FF0C990DA811F01C
:104C5000D7FC0246002862D10146154B022029E705
:104C6000586E03082C700308901F00200000824239
:104C70009A99993FCDCC4C3F000020406666263F74
:104C8000000020410AD7233CAE700308281F0020F3
:104C90004C7003087C700308C970030820040020CE
:104CA000261F002024170020E7700308CDCC4C3EBF
:104CB00010710308109A0F999DF83800FFF746FC11
:104CC0009DF838305BB110993846FDF7C3F80F995D
:104CD00007463046FDF7BEF80134E4B206469AF8BE
:104CE0000030012B16D12B88109A9BB209EB0313CD
:104CF0009A602B880F9A9BB209EB03135A602B889A
:104D00009BB25A1C92B2802B2A8003D1FFF756FC2B
:104D100000232B80B8F101087FF44BAF55E70D98C5
:104D200011F0DAFC00283FF433AF0CA811F088FB37
:104D3000DFF850B1DFF85081DFF850A14FF02109C2
:104D40000D980EA911F020FD054600285CD1024601
:104D500001464F4B032010F011FDDFF83891012C74
:104D600094BF0023012389F8003099F8003003F044
:104D7000FF0203B101224848042103F077FD4749AF
:104D80003846FDF76FF907462046FDF717F98046CC
:104D900001463846FDF71AFA404907463046FDF706
:104DA00061F94146FDF712FA3D4B1F603D4B002172
:104DB00018608046FDF7EAFA0646A8B94223404645
:104DC00099F80090CDE90343FDF728FB029038469F
:104DD000FDF724FB5FFA89F9CDE90090324B3246AA
:104DE0003146032010F0CAFC0D9811F095FC0446E2
:104DF0000DA811F0DBFB13F06BFE002C3FF4F6ADB9
:104E000085F00100C0B2F2E5109A0F999DF83800C4
:104E1000FFF79CFB9DF8453073BB9DF838305BB1C4
:104E200010993846FDF716F80F9907463046FDF7FA
:104E300011F80134E4B206469BF80030012B1BD177
:104E4000B8F80030109A9BB20AEB03139A60B8F8D6
:104E500000300F9A9BB20AEB03135A60B8F8003087
:104E60009BB25A1C92B2802BA8F8002004D1FFF705
:104E7000A5FB0023A8F80030B9F101097FF460AF69
:104E80006BE700BF20040020261F0020241700200D
:104E9000E7700308831F00200004004800007A44E4
:104EA0007C1F0020781F0020307103082DE9F0439B
:104EB000ADB014230DF10E0204A9ADF80E3014F0BC
:104EC0001BF8044648B902460146194B032010F06E
:104ED00055FC20462DB0BDE8F0830022154B164F3F
:104EE000DFF85880DFF858901146032010F046FC98
:104EF0000025BDF80E30AAB29342EAD9AAB22CAB73
:104F000003EBC202032012F89C6C52F8A03C002E66
:104F100014BF3A464246CDE9003200224B461146C4
:104F200010F02CFC002E05F1010508BF3446E0E727
:104F30008A710308AD710308807103088571030845
:104F4000D171030830B5102289B0002529460446E6
:104F50000DEB020003952AF033FB15F077FB2A4690
:104F6000A34B00902946032010F008FCFDF7AAFC93
:104F700013F03AFD8DF80C0013F0E0FD431B18BF51
:104F8000012301218DF80D30029013F0F5FD0298F8
:104F900013F094FF029813F009FE0298FFF786FFC2
:104FA000002840F0008102A813F0D8FD13F090FD16
:104FB000029813F017FE029813F030FE0298FFF7E4
:104FC00075FF002840F0F38002A813F0C7FD13F02E
:104FD0007FFD029813F03EFE0022864B114603200F
:104FE00010F0CCFB029813F051FE0298FFF75EFF21
:104FF000002840F0E08002A813F0B0FD13F068FD37
:10500000029813F05FFE002211467B4B032010F044
:10501000B5FB0022794B1146032010F0AFFB02983C
:1050200013F0DCFE0298FFF741FF002840F0C78034
:1050300002A813F093FD13F04BFD029813F0EAFE63
:10504000002211466E4B032010F098FB00226D4B9E
:105050001146032010F092FB029813F0F7FE02981D
:10506000FFF724FF002840F0AE8002A813F076FD81
:1050700013F02EFD029813F005FF00221146624B3B
:10508000032010F07BFB0022604B1146032010F040
:1050900075FB029813F032FE0298FFF707FF002815
:1050A00040F0958002A813F059FD13F011FD02980D
:1050B00013F040FE00221146554B032010F05EFB1A
:1050C0000022544B1146032010F058FB029813F0B5
:1050D0004DFE0298FFF7EAFE00287CD102A813F0EB
:1050E0003DFD13F0F5FC029813F05CFE0022114622
:1050F000494B032010F042FB0022404B1146032095
:1051000010F03CFB029813F069FE0298FFF7CEFE08
:10511000002864D102A813F021FD13F0D9FC0298F5
:1051200013F078FE00221146354B032010F026FBC9
:105130000022344B1146032010F020FB029813F09C
:1051400085FE0298FFF7B2FE00284CD102A813F0AA
:1051500005FD13F0BDFC029813F094FE00221146E9
:10516000294B032010F00AFB002211462B4B032091
:1051700010F004FB01238DF8173003AB03CB0022A2
:105180002060186861600C23A06011460093032022
:10519000234B10F0F3FA02A813F0E0FC13F098FC94
:1051A000002009B030BD01238DF80E3000E7012347
:1051B0008DF80F300DE701238DF8103020E7012323
:1051C0008DF8113039E701238DF8123052E70123B1
:1051D0008DF813306BE701238DF8143083E701233A
:1051E0008DF815309BE701238DF81630B3E700BF2B
:1051F000E77103081072030843720308747203080E
:10520000A3720308D07203080573030838730308F8
:105210006B7303089C730308CC730308FA730308C9
:105220002774030802480122102103F01FBB00BFAE
:105230000004004802480022102103F017BB00BF01
:105240000004004813B5134C23785BB9E37C03F0EA
:10525000FF023BB9104B1146022002B0BDE81040DE
:1052600010F08CBAFEF74AF900380C4B18BF012039
:10527000400018701A78022A02BF00222270E274DD
:105280001B7800930022064B1146032010F076FA9B
:1052900002B010BD5622002046740308FC1F0020F7
:1052A0006274030838B5184C23785BBBE37C03F0C9
:1052B000FF023BBB154D2B68012B0CD92B68042B2F
:1052C00009D81146124B022010F058FA114A042155
:1052D000012000F0EBFF2B68042B13D900220E4BAA
:1052E0001146022010F04AFAFEF708F900380B4B7D
:1052F00018BF0120400018701B78022B02BF00234A
:105300002370E37438BD00BF56220020F81F002030
:10531000797403089E740308A3740308FC1F00201B
:1053200010B5124C237863B101214FF0904003F087
:1053300097FA0F4B0022187022701B780D4ADBB2CF
:1053400013700D4C237863B102214FF0904003F0AD
:1053500087FA0A4B0022187022701B78084ADBB2C9
:105360001370BDE81040FEF7F3B900BF921F002094
:105370000A01002008010020911F002009010020DF
:105380000701002070B5174D174B00242C701A78B8
:10539000022A23D91B78082B20D8FFF719FB1348C2
:1053A000134A037811785B1A124918BF01230B7056
:1053B00003781148DBB21370104B114A1E78037842
:1053C000F31A18BF012313700E4B06701B781BB124
:1053D0000D4B0C701C701470FEF7BAF901232B7082
:1053E00070BD00BF1604002006010020831F0020AE
:1053F000801F0020841F0020081600200A160020AD
:1054000009160020FC1F0020851F002008B501217F
:105410004FF0904003F024FA064B012816BF0222F9
:1054200018701A701878044B1978BDE80840FEF718
:10543000EDB800BF060000200000002038B5324D56
:10544000324C287BFCF7B6FD3149FCF70BFEA0601F
:10545000687BFCF7AFFD2E49FCF704FEE060A87BFB
:10546000FCF7A8FD2A49FCF7FDFD6062E87BFCF72C
:10547000A1FD2849FCF7F6FD274BE0642361287C59
:10548000FCF798FD6060687CFCF794FDA061A87C47
:10549000FCF790FDE061E87CFCF78CFD2062287D44
:1054A000FCF788FDA062687DFCF788FD1849FCF7D1
:1054B000D9FD2063A87DFCF77DFD6063E87DFCF7E6
:1054C0007DFD1449FCF7CEFDA063287EFCF772FD3C
:1054D000E063687EFCF772FD0D49FCF7C3FD2064B4
:1054E000A87EFCF76BFD0A49FCF7BCFD6064E87E12
:1054F000FCF760FDA064287FFCF75CFD074BE062D1
:1055000002221A7038BD00BFD5030020281F0020DA
:10551000CDCCCC3D0AD7233CCDCCCC3E901F002037
:1055200038B5114D114C287BFCF748FD1049FCF7AC
:1055300099FDA060687BFCF741FD0D49FCF792FDE9
:10554000E060A87BFCF73AFD0949FCF78BFD60623F
:10555000E87BFCF733FD0749FCF784FD064BE0646C
:1055600001221A7038BD00BFD5030020281F00207B
:10557000CDCCCC3D0AD7233C901F002073B52F4DD6
:105580002F4E2B7803702F4B1B784370044601215C
:105590004FF0904003F064F93378A070E37002217B
:1055A0004FF0904003F05CF9274B20711B7863713A
:1055B0003378012B3ED1254B1868FCF755FF244B5F
:1055C000E0801868FCF750FF80B2224BA0831B7864
:1055D000191F4A424A41A2771F4A92F82B1084F8B9
:1055E0002B10D26AE262012B84F828300FD11B4BBA
:1055F000009300221A4B1146022010F0BFF8194BFD
:105600001B8884F82930184B1B8884F82A30174BE4
:105610001B7853B1164B1B683BB1164B1B78012B03
:1056200001BF154A232313702B70144B01221A70EB
:1056300002B070BD0020E080C7E700BF0600002078
:10564000831F002006010020821F00207C1F0020F5
:10565000781F00200A160020981F0020520000200A
:10566000D674030802160020FE1500202104002035
:105670008C1F00205322002007000020F41F002070
:10568000024B01220021032010F078B804750308B2
:1056900008B50122074B0021032010F06FF8FFF737
:1056A000C1FDFFF7CBFE044A00231370034A1370B9
:1056B00008BD00BF4A750308901F0020512200203A
:1056C00010B5144B01220021022010F057F8124BA4
:1056D0001A78124BD2B25A700024012263211A7038
:1056E00083F8331083F834209C63DC631C645C64AF
:1056F0009C64DC641C655C6583F82B40DC625C6246
:105700009C77FFF78FFDFFF7BBFFFFF7C1FF044B4F
:105710001C7010BD8075030806010020981F002032
:10572000512200201FB5114B11491C6858681A7A84
:105730005B7ACDE90223FCF795FCFCF795FE0C495A
:1057400001902046FCF78EFCFCF78EFE0022094BF0
:1057500000901146032010F011F8FEF70DFE6420B2
:1057600004B0BDE81040FEF719BA00BF20000020C9
:1057700000007A44B77503082DE9F04186B00D4664
:105780000446FFF74FFD01F071FFFDF7D7FB9620B0
:10579000FEF704FA154F00264FF00508AE420FD170
:1057A0004FF47A70FEF7FAF901AB03CB1B88238123
:1057B0000F4B2060002261601A7006B0BDE8F081D6
:1057C000FEF7C4F887F80080FDF7B8FF4FF47A7051
:1057D000FEF7E4F901A8FFF7B5FB41F28830FEF7C8
:1057E000DDF90136FFF79EFFD8E700BF0600002075
:1057F0005122002030B585B00446002503A8ADF83D
:105800000C50FDF763F870B19DF80C309DF80D2039
:10581000237062702946CDE900320320034B2A46EB
:105820000FF0ACFF012005B030BD00BFEC750308E0
:10583000022801D8FFF7F6BC7047022801D8FFF70D
:10584000F9BC7047022803D80248102103F013B8AE
:10585000704700BF0004004807B5684610F01EFA04
:10586000054B1B7803F0FF021BB9044B00999963A9
:10587000DA6303B05DF804FB03000020981F0020EA
:1058800007B5684610F00AFA054B1B7803F0FF02D3
:105890001BB9044B009919645A6403B05DF804FB0A
:1058A00002000020981F002007B5684610F0F6F9A6
:1058B000064A009B1278012A01BF054A0021936421
:1058C000D164044A136003B05DF804FB831F002019
:1058D000981F0020881F002008B5FEF7ABF8BDE830
:1058E000084000F037BF4FF0FF3010F091B870471C
:1058F000014B01221A70704760200020014BD870C4
:10590000704700BF18010020014B1874704700BF9A
:105910001801002007B5064B00221B5C00931146BE
:10592000044B03200FF02AFF03B05DF804FB00BF17
:105930002B760308117603080021012010F030B8FF
:1059400013B5104A104C42F21073002818BF0346DA
:105950000E482360136010F0FFFA21680B4810F026
:1059600083FB0A4810F046FB23684FF47A72B3FBBE
:10597000F2F3002200931146054B03200FF0FEFEC8
:1059800002B010BD1804002014010020B82100202E
:105990002F76030813B50D4C206023680BB90C4B10
:1059A00023600C4810F0D8FA21680A4810F05CFB1C
:1059B000084810F01FFB236800930022064B114695
:1059C00003200FF0DBFE02B010BD00BF1804002062
:1059D000A0860100002000205B76030813B50F4C61
:1059E0002060236813B942F2107323600C4810F052
:1059F000B3FA21680A4810F037FB094810F0FAFAA8
:105A000023684FF47A72B3FBF2F30022009311463D
:105A1000044B01200FF0B2FE02B010BD1C040020A8
:105A2000182000209776030837B5044600283BD09D
:105A300090F90650002D48D1274810F08DFA274BD9
:105A400001221A70FDF788FD2A462946244B0220C0
:105A50000FF094FEE379012B0CBF224B224B2A4618
:105A600029460220214D0FF089FEE3792B70204B4F
:105A70001868FFF78FFF29781E4A1F4B012908BFBE
:105A800013460022009311461C4B01200FF076FEB6
:105A900094F90530019394F9043000930022184BD7
:105AA000114603200FF06AFE164B0122002102204E
:105AB0001A700FF075FF40F6B830FEF76FF8124815
:105AC00003B0BDE8304010F095BA00220F4B1146EC
:105AD00002200FF053FEDBE76420002006000020C8
:105AE000D9760308EE7603080B77030852220020CC
:105AF00018040020D0760308D4760308287703081A
:105B000060770308502200204820002047770308D0
:105B10000A460149FDF7CCB900F0030870B51648F4
:105B200010F01AFA06F0E6FF044650B10022134BBB
:105B3000114602200FF022FEBDE87040104810F020
:105B400059BA104D104B0246014602200FF016FEC6
:105B500001260E4B2E702246214602200FF00EFE2B
:105B60000B4806F05BFE2878314606F0AFFB024892
:105B700010F040FAE0E700BFB82100208977030861
:105B8000A02100207C010020A7770308BB77030831
:105B9000180100202DE9F047AAB0FDF77DFF05466A
:105BA00006F08EFC002846D1954F964C13A8FFF7BF
:105BB000E5FC3B78042B41D111232370924B1A78DA
:105BC00002F0FF01002A43D000221A703B78042B18
:105BD00039D1122323708D4B62681B7863F07F03E9
:105BE0001370636828B200EB400000EB4010FE2207
:105BF0000226B0FBF2F05870854B1B78012B88BF52
:105C000000266670834C637A33B106F045FC0128A8
:105C100002D1204610F0A0F97F4B7A48D9780022B3
:105C200006F064FC0146002840F0D5807B4B012241
:105C300002200FF0A3FD2AB0BDE8F0873B78052BCA
:105C4000BCD11323B9E73B78052BC4D11423C1E79A
:105C5000734B1A7802F0FF06002ACDD019706B4BF7
:105C600062681B7863F07F03137063689DF84C20B3
:105C70005A7063689DF84D509D703B78042B5FD13E
:105C800063689DF84E20DA7063689DF84F201A71A2
:105C900063689DF850205A710626624BDFF888A190
:105CA00093F8009093F8008000211A220CA84FEA84
:105CB00019190B9108F00F0829F082FCB9F1000FB7
:105CC00073D0C9EB09190AEB09010BAB184629F08F
:105CD00006FD05EB8505554A554B05EB8505C8EBDB
:105CE000081815440AEB0802CDE9000200220295CB
:105CF000114601200FF042FD3B78052B57D19DF84E
:105D0000743008931C9B07939DF86A300693BDF886
:105D100068300593BDF8523004939DF851300393D9
:105D20009DF8503002939DF84F30019300229DF86A
:105D30004E30009311463F4B03200FF01FFD5BE7F1
:105D40003B78052B2FD163689DF84E20DA7063688D
:105D50009DF84F201A7163689DF850205A7163684E
:105D60009DF851209A71BDF8523062681B0AD371B8
:105D70006368BDF852201A72BDF86820120A5A7280
:105D8000BDF868209A729DF86A20DA729DF8742036
:105D90001A739DF877205A731E9A120A9A731E9AE4
:105DA000DA73102679E7032677E723498DE73B78F6
:105DB000042B7FF421AF9DF8503002939DF84F30B3
:105DC000019300229DF84E30009311461B4B012099
:105DD0000FF0D4FC10E706317FF42DAF06F056FB30
:105DE00000283FF428AF4FF47A730122B0FBF3F0A0
:105DF00000210090124B03200FF0C0FC1BE700BFF6
:105E0000060100200C01002050220020AC200020C0
:105E1000FC1F002064200020180100207E79030868
:105E2000F41F002006000020F40200207D01002065
:105E3000DA77030803780308917C030810790308D4
:105E40008E79030813B568460FF028FF1A4B009AA5
:105E500019781A4B11B9996B511AD9631849DC6B2F
:105E60000878844281BF012083F82B00D86BD86268
:105E70001448007810B9186C101A58645C6C0878D3
:105E8000844281BF012083F82B00586CD8620E48F1
:105E90000078012802BF986C121ADA64D86C0A786C
:105EA000904205D9012283F83220DA6C92B21A8628
:105EB000064B1B7802B010BD03000020981F002085
:105EC0002104002002000020831F00200A16002069
:105ED00000B503468DB000282CD0407802280AD0A7
:105EE00003282AD0164B0022114602200DB05DF87F
:105EF00004EB0FF043BC1A7F0B92DA7E0A929A7E73
:105F000009925A7E08921A7E0792DA7D06929A7D4D
:105F100005925A680492DA68039293F91420029267
:105F2000B3F9122001921B7C00930022054B11460D
:105F30000FF024FC0DB05DF804FB034BD3E700BF6A
:105F4000AC790308C3790308357A030801284FF0B8
:105F500000020CBF024B034B114602200FF00EBC97
:105F6000547A0308667A03081FB50446002831D026
:105F70000378002B2ED01D4810F03CF8002211466B
:105F80001B4B02200FF0FAFB94F91830039394F99D
:105F90000A300293237C0193E368009300221146A8
:105FA000144B03200FF0EAFB0022134B1146032091
:105FB0000FF0E4FB237A012B0ED1617A0F4A104BCC
:105FC000002918BF13460022009311460D4B0320F1
:105FD0000FF0D4FB04B010BD00220B4B1146032080
:105FE00004B0BDE810400FF0C9BB00BF94200020F2
:105FF0007F7A0308B07A0308E17A03087B7A030802
:106000007A7A0308EE7A0308FF7A030808B5104B82
:106010000122002102201A700FF0C2FC0D480FF07F
:10602000E9FF0D4B1B788BB10C4B1A7872B9DB7CF6
:1060300063B90B4B1A68042A9EBF1A6801321A60B2
:106040000021BDE8084010200FF0AABC08BD00BF29
:106050005022002000200020522200205622002042
:10606000F81F0020044B1B78022B03D100210820CD
:106070000FF096BC704700BF7C010020044B1B78DA
:10608000012B03D0002180200FF08ABC704700BF95
:106090000601002008B50C4B1B789BB10021402065
:1060A0000FF07EFC094B1B7863B1094B1A78012A6B
:1060B00008D10021022019700FF072FCBDE80840E1
:1060C000FFF7F2BB08BD00BF1604002052220020DB
:1060D000841F002008B506F016FD80B906F0DCF933
:1060E00001280CD1BFF34F8F0549064BCA6802F453
:1060F000E0621343CB60BFF34F8F00BFFDE708BDE5
:1061000000ED00E00400FA0538B504460D460748E6
:106110004FF40061FCF7ECFE30B92A4621460348F3
:10612000BDE83840FCF7EABD38BD00BF00F0030809
:1061300010B506F093FD10F1080F07D1064B0022B1
:10614000BDE81040114602200FF018BB013001D10C
:10615000024BF4E710BD00BF0D7B0308237B03084F
:1061600038B5104C237822781809D2B20CD10E4DD4
:106170002A7823789A4206D020781E21FDF7B8FAB3
:106180002378DBB22B7038BD084C23781E2133B145
:10619000FDF7AEFA237883F001032370F3E702F0F2
:1061A0000F00F5E70600002054220020150400200F
:1061B00070470000022837B5044636D040285CD02E
:1061C00001285DD12F4B1B78002B59D0FA20FDF709
:1061D000E5FC21464FF0904002F042FB2A4B21465D
:1061E00018704FF0904002F03BFB214605464FF0FF
:1061F000904002F035FB254A254B002808BF134686
:106200000022CDE900531146224B02200FF0B6FACE
:10621000FFF722FB002120200FF0C2FB002102200B
:1062200003B0BDE830400FF0BBBB1B4B1B783BB34A
:10623000FA20FDF7B3FC21464FF0904002F010FB2E
:10624000164B214618704FF0904002F009FB214692
:1062500005464FF0904002F003FB114A114B002815
:1062600008BF13460022CDE9005311460E4B2046CD
:106270000FF084FAFFF704FBCCE700210420CFE7FE
:1062800003B030BD921F0020030000203B7B0308B9
:10629000477B03086D7B0308911F0020020000204C
:1062A000537B0308607B0308937B030873B50546A3
:1062B0000C46164606F004F90346002832D002B018
:1062C00070BD4A68F05CD0540133DAB2A242F8D310
:1062D0001E4B0D701A781B78012A88BF00244C7061
:1062E0000022CDE900341A4C1A4B114601200FF060
:1062F00045FA637A33B106F0CFF8012802D120467F
:106300000FF02AFE144B1548D978002206F0EEF85B
:10631000014648B9124B0122032002B0BDE870408B
:106320000FF02CBA0D49D0E70631C8D106F0AEF80F
:106330000028C4D04FF47A730122B0FBF3F000219F
:106340000090084B03200FF019FAB8E7FC1F00205B
:1063500064200020B87B0308180100200C010020F5
:10636000E97B03088E790308044B1B7823B9044AA0
:1063700005210120FFF79ABF704700BFFC1F0020D6
:10638000F87B030810B5002490B03C22214601A8F8
:10639000009429F015F9454B2022DA7219788DF80E
:1063A000001059788DF8011099788DF80210D9787D
:1063B0008DF8031019798DF8041059798DF80510AE
:1063C00099798DF80610D9798DF80710197A8DF81A
:1063D0000810597A8DF80910997A8DF80A108DF8FD
:1063E0000B2021460DF10B0258180131007B02F8F9
:1063F000010F1429F8D193F820208DF8202093F86C
:1064000021208DF8212093F822208DF8222093F866
:1064100023208DF8232093F824208DF8242093F84E
:1064200025208DF8252093F826208DF8262093F836
:1064300027208DF8272093F828208DF8282093F81E
:1064400029208DF8292093F82A208DF82A2093F806
:106450002B2093F828108DF82B20154A19BB93F8A0
:10646000291001F0FF00F1B9107093F82C206AB1E7
:1064700093F83F2052B10DF12B0100229818013200
:1064800090F82C0001F8010F142AF7D109484FF4B5
:106490000061FCF72DFD20B9064840226946FCF753
:1064A0002DFC10B010BD01211170DEE7D5030020D6
:1064B0002004002000F8030810B50022044611460D
:1064C000054B02200FF05AF920460449BDE8104060
:1064D00040220FF059BA00BFFE7B030800F8030802
:1064E00038B5454C207963794D2BC0B26AD1C0EBE9
:1064F00000108000A379E2790A2838BF0A204D2ACB
:10650000DBB267D1C3EB03139B004FF47A7202FB3B
:1065100003F594F82C30002B64D194F83F30002B15
:1065200060D142F21070FFF70BFA344B1868FFF796
:1065300031FA237A32493348DBB20B70324B0122F5
:106540001A70637ADBB2037094F827302F48DBB2FD
:1065500003700B782E49052B2E4B18BF00221A70A2
:1065600094F828302C4A03EB83035B00DBB21370F2
:1065700094F82930294A03EB83035B00DBB21370E4
:1065800094F82A30264A0133DBB2DB01138094F8F9
:106590002B30244A03EB83035B00DBB21370002330
:1065A000E21892F82C20D2B2CA540133142BF7D13E
:1065B000A378012B1FD1E37A202B1CD1BDE83840F2
:1065C000FFF77EB86379482B0ABF4FF461636379A4
:1065D00058438FE7E279482A0ABF4FF46162E279B3
:1065E000534392E74FF47A735843FFF7D3F92846A1
:1065F000FFF7F4F99DE738BDD5030020180400200B
:1066000006010020FC1F00200600002005000020DD
:106610005622002020040020230400202204002011
:106620003C0000202104002010B590B000213C2245
:1066300001A8009128F0C4FF4022434968460FF0AA
:10664000A3F99DF800203AB99DF80100072803D16D
:106650009DF8021001290FD000223C4B1146022068
:106660000FF08CF8FFF78EFE4FF47A70FDF796FA74
:10667000FFF736FF10B010BD354B1A705870997087
:106680009DF80310D9709DF8041019719DF805103C
:1066900059719DF8061099719DF80710D9719DF8F0
:1066A000081019729DF8091059729DF80A10997214
:1066B0009DF80B1001F03F01D9720DF10B019818F4
:1066C000013211F8014F0473142AF8D19DF82020EB
:1066D00083F820209DF8212083F821209DF8222096
:1066E00083F822209DF8232083F823209DF824207E
:1066F00083F824209DF8252083F825209DF8262066
:1067000083F826209DF8272083F8262083F8272069
:106710009DF8282083F828209DF8292083F8292037
:106720009DF82A2083F82A209DF82B2083F82B201F
:106730000DF12B0100229818013211F8014F80F859
:106740002C40142AF7D193E700F80308127C0308C1
:10675000D5030020F0B507238BB0062200240125C5
:10676000CDE905231822CDE9033221466B4B029473
:1067700022460327CDE90055022009940EF0FEFFC2
:10678000674B029422462146CDE9005702200EF0C5
:10679000F5FF02260523CDE900632246614B0294F2
:1067A000214630460EF0EAFF5F4B00952246214617
:1067B000CDE9017430460EF0E1FF09A9204606F04C
:1067C00087F9099BC3F307220292C3F307421B0E0A
:1067D000019200932246554B214630460EF0CEFFE3
:1067E00009A9284606F074F9099BDAB20392C3F3AB
:1067F00007220292C3F307421B0E01920093224626
:106800004B4B214630460EF0B9FF4A4B4A480094A4
:1068100022464FF4FA710FF041FB484B4848009470
:1068200022464FF4FA710FF039FB464B464800946C
:106830002A464FF4FA710FF031FB444B4448009460
:106840002A464FF4FA710FF029FB424B424800945C
:106850002A4642F210710FF021FB2046FCF748FA5D
:1068600008B1FCF769FC3D4B009400224FF4FA613B
:106870003B480FF013FB3B4A002101200FF04CF97D
:10688000394A002102200FF047F9384A002104203C
:106890000FF042F9364A002108200FF03DF900F0D0
:1068A0003FFE3449344806F0C9F8344805F0B6FFD5
:1068B00025480FF09FFB324B0021187805F006FDAC
:1068C000FFF7B2FE2F4A002110200FF025F92E4AC3
:1068D000002120200FF020F92C4A002140200FF049
:1068E0001BF92B4A002180200FF016F9294B2A486A
:1068F00019682A4B009401220FF0D0FA26480FF0B5
:1069000079FB274B27481968274B009401220FF089
:10691000C5FA24480FF06EFB0BB0F0BD527C0308A3
:10692000927C0308B37C0308D47C0308F57C03083D
:10693000167D0308EF58000894200020B16100087C
:106940007C2000207D600008642000206161000838
:1069500048200020455E00083020002065600008C7
:10696000A021002021C60008955B000831610008C5
:106970001D5B000800000301300100201801002009
:106980007C010020A552000821530008855300080F
:106990000D5400081C0400201820002095600008F9
:1069A00018040020002000200D60000873B50D4D74
:1069B00000262E60FEF7B6FEC820FDF7EFF8286827
:1069C0003146FBF7E3FC04460028F3D12868FBF7C7
:1069D00025FD054B00902246214601200EF0CEFEFB
:1069E00002B070BD941F00203A7D030830B500242A
:1069F000A5B07C22214605A8049428F0E1FD53238C
:106A00008DF81030012540F20713ADF81230ADF8C3
:106A100000408DF81450FDF73FF8FE23B0FBF3F073
:106A200000EB400000EB40103A4B8DF81500224679
:106A3000214603200EF0A2FE6846FEF7DBFE9DF81D
:106A400000309DF80120134314D158238DF81630DF
:106A5000072480220021304828F0B2FD224604A9F4
:106A60002D4828F04BFE2C4A21460120FFF71EFC42
:106A700025B030BD0E23294601A8CDE901448DF88B
:106A80001630ADF80C40FEF777FE01AB03CB234C7C
:106A90001B88CDF81B10ADF81F30CDF81700FEF79E
:106AA00041FE2068FBF7E0FC0A254FF47A7380B2C0
:106AB000B0FBF3F0B0FBF5F305FB130030308DF8BD
:106AC00021002068FBF7D0FC642380B2B0FBF3F018
:106AD000B0FBF5F305FB130030308DF82200206881
:106AE000FBF7C2FC80B2B0FBF5F0B0FBF5F305FBA1
:106AF000130030308DF823002068FBF7B5FC80B21E
:106B0000B0FBF5F305FB130030308DF8240015249D
:106B10009FE700BF6D7D0308D0210020941F002057
:106B20002DE9F047044698B0C0480D468022002168
:106B30000EF034FF2378592B40F06782052D5ED884
:106B40006378443B162B5AD8DFE813F0A9015900AB
:106B500099015900A1015900590059005900BD007F
:106B60005900840159005900590004025900590084
:106B7000E7005900590059001700A678482E17D190
:106B8000AB4A14210120FFF791FB41F28830FDF759
:106B900005F80022A74B114603200EF0EFFD40F64A
:106BA000B830FCF7FBFF18B0BDE8F047FFF792BA2A
:106BB000532E0DD1FFF71AFF41F28830FCF7EEFF9C
:106BC0009A4A1521012018B0BDE8F047FFF76EBBC7
:106BD000432E17D1002408A88DF8204005F096FD1B
:106BE000924A4C231370072393709DF82030547001
:106BF00001204133D07013710521FFF757FB18B006
:106C0000BDE8F087442EFAD1884C8B4DA6705923ED
:106C100023705A236370FFF7C9FE2868FBF7FEFB59
:106C20000022864B0090114603200EF0A7FD7F2224
:106C30000021601C28F0C4FC072326700126A370E5
:106C4000E6702671FCF728FFFE23B0FBF3F000EBA3
:106C50004000042300EB40106071A3712868FBF72B
:106C600003FC0A274FF47A7380B2B0FBF3F0B0FB59
:106C7000F7F307FB13003030E0712868FBF7F4FBF3
:106C8000642380B2B0FBF3F0B0FBF7F307FB130013
:106C9000303020722868FBF7E7FB80B2B0FBF7F0DA
:106CA000B0FBF7F307FB1300303060722868FBF786
:106CB000DBFB80B2B0FBF7F307FB13003030A072B0
:106CC00022460B217EE7A378303BDBB2092B96D816
:106CD0005B4C5C4A23702378DBB25372534A5923CE
:106CE00013704D23537023780321303301209370A8
:106CF000FFF7DCFA237800930022534B1146012062
:106D00000EF03CFDFFF73EFB2378002B3FF477AFFE
:106D100018B0BDE8F047FCF769BCA578482D47D10D
:106D2000424C562318220025012623706271072346
:106D3000062206A8A370A271E3716570E670267141
:106D40000EF086FF069808A912380FF009F80D9B7F
:106D500003F26C7305930C9B334404930B9B0393D6
:106D6000089B0293099B01930A9B00932A46374B89
:106D7000294602200EF002FD0D9B25726C336372D2
:106D80000C9B3344A3720B9BE3720A9B2373099BF6
:106D900063732246089BA3730F213046FFF786FAE0
:106DA0002B4B00942A46114602200EF0E7FC26E702
:106DB000432D7FF424AF00213C2209A81B4C0891ED
:106DC00028F0FEFB08A8FFF777FB9DF820306370E2
:106DD0009DF82130A3709DF82230E3709DF8233098
:106DE00023719DF8243063719DF82530A3719DF8BF
:106DF0002630E3719DF82730257023729DF82B50C3
:106E00009DF8283063729DF82930A3722A469DF8B8
:106E10002A30E3720BA904F10D00257328F06EFCF3
:106E200005F10D012246C9B20120E6E6D02100207D
:106E3000867D03089B7D0308941F0020BD7D030809
:106E4000FC1F0020D5030020E07D0308097E030815
:106E5000337E0308A07839280CD83038C0B2FEF74A
:106E6000E7FC8E4A2378137063785370A37893708D
:106E70000321A7E618B0BDE8F047FFF775BAA07880
:106E80003928F7D83038C0B2FEF7D7FCE9E7A07848
:106E90003928EFD83038C0B2FEF7D4FCE1E7A37848
:106EA000303BDAB2092AE5D8E578303DEAB2092A62
:106EB000E0D82179A1F14802D2B20B2ADAD8784879
:106EC00040FA02F2D007D5D40A224D2902FB03551D
:106ED0003BD13C235D43734B4FF47A706843186099
:106EE000714B1860FEF756FD6C4A23781370637877
:106EF0005370A3789370E378D370052123791371CD
:106F00000120FFF7D3F9694B002607221E705A7043
:106F100001229A70DA70A178303901EB8100E178B2
:106F2000303901EB4001C9B2197122795A71604AB6
:106F30001278D2B21A725F4A1278D2B25A72FFF73E
:106F400021FA5D4B009532462DE74829C3D14FF415
:106F50006163BFE7A278303AD3B2092B8AD8E378CD
:106F6000303BD9B2092985D82079A0F14801C9B2AE
:106F70000B293FF67FAF4A4D45FA01F1C9073FF5AE
:106F800079AF0A214D2801FB023339D13C2253430A
:106F90004FF47A725343494A13601068FEF71EFD9E
:106FA0003E4A2378137063785370A3789370E37824
:106FB000D3700521237913710120FFF777F93B4B3B
:106FC00000221A7007225A7001229A70DA70A27891
:106FD000303A02EB8201E278303A02EB4102D2B25F
:106FE0009A712279DA71324A1278D2B21A72314A1F
:106FF0001278D2B25A7218B0BDE8F047FFF7C2B9A2
:107000004828C5D14FF46162C1E7502B40F0B381ED
:10701000022D7FF6F4AD6178A1F13003012B3FF62C
:10702000EEADA378312B7FF4EAAD052D4ED1E37898
:10703000302B40F0C1801E4D214E00232B702B7849
:1070400003F0FF0253B92379303BDBB2337033785E
:10705000009311461B4B02200EF090FB15491A4A73
:1070600000230B703378DBB213702B780F4ADBB23E
:1070700013720B78DBB25372FFF784F9074B227857
:107080001A7062785A70A2789A70E278DA7022796F
:107090001A71FCF75DFB0521004A93E5D021002021
:1070A000DEF7FFFF1401002018040020D5030020A4
:1070B00006010020FC1F00205D7E03081C04002048
:1070C00004000020947E030806000020082D67D1EC
:1070D000E378462B40F0F8802179A1F13000C0B26E
:1070E000092800F246816279A2F13003092B00F2EF
:1070F0004081A679A6F13003092B00F23A81E379A9
:10710000A3F13005092D00F2348101EB8101490022
:10711000B74D203102EB8202C9B2520029702032F1
:10712000B449D2B22F3E0A70F6B2B34A03EB8303DE
:10713000F6015B0016802033B04ADBB21370B04A10
:1071400082F828006379303BDBB282F82930A379DA
:107150002F3BDBB282F82A30E379303BDBB282F896
:107160002B302B782BB90B7803F0FF020BB9A54B12
:107170001A70FFF707F9A44B22781A7062785A70D8
:10718000A2789A70E278DA7022791A7162795A716B
:10719000A2799A71E279DA71FCF7DAFA08217BE7D1
:1071A000042D3CD1E278A2F13003DBB2092B11D9D6
:1071B000A2F14103192B0AD9FFF7D6F80022934B0D
:1071C0001146012018B0BDE8F0470EF0D7BAA2F181
:1071D0003703DBB28E4803708B4B20785970312116
:1071E00099708B491870DA700B78854ADBB213728C
:1071F0000B78052B834B0CBF012100211970854BA7
:107200001B78DBB25372FFF7BDF8FCF7A1FA4FF41D
:10721000FA60FCF7C3FCFEF75DFF04213CE71D2D7F
:107220004FD9A61C0025DFF8D891DFF8ECA137462E
:10723000A84617F8012F303AD2B2092A3ED809EBF6
:10724000050303201A731B7BCDE902533B78002210
:10725000CDE90053114653460EF090FA01351E2D2C
:10726000E7D1B8F1000FA7D1FEF7E8F8664B50223E
:107270001A7000225A7007229A700122DA7003F8FD
:10728000042F203416F8012F03F8012FB442F9D14E
:107290005B4B00221A7007225A7001229A70DA7032
:1072A0005B4A1278D2B21A725A4A1278D2B25A7221
:1072B0001E22DA72FFF766F82321EDE64FF001088F
:1072C000CCE7072D7FF678AF00254D4FDFF84881DA
:1072D00002342E4614F8012F303AD2B2092A46D889
:1072E000791903200A730B7BCDE90253237800221E
:1072F000CDE90053114643460EF040FA0135082D02
:10730000E8D1002E7FF458AFFEF70AF93E4B3C4C13
:1073100050221A7007229A701A460121002502F89D
:10732000041F5D70D97061190135097B082D01F1C9
:10733000300102F8011FF6D100221146009301200E
:10734000364B0EF01BFA00232370072363700123D2
:10735000A370E3702E4B1B78DBB223722D4B1B788E
:10736000DBB26372E572FFF70DF80D2194E601269A
:10737000C4E7002190E6412B7FF441AC6378432BB6
:107380007FF43DAC162D7FF43AAC254D621C0023F2
:1073900012F8011FE9540133142BF9D1FDF752FF04
:1073A000204B5B7D012B1ED115490023EA5CC818D8
:1073B0000133D2B2142B80F82C20F7D1154B0022C8
:1073C0001A701B78DBB24B72FEF7DCFF0E4A631EAD
:1073D000153413F8011F02F8011BA342F9D10A4A20
:1073E0001621FFF7EFBB0B4B02221A70EEE700BF2E
:1073F00023040020220400203C000020210400205F
:10740000D503002020040020D0210020F37E0308B3
:1074100006010020FC1F0020B07E0308D87E030870
:1074200056220020A40A002070B5054688B00C46FC
:10743000002951D033480EF0DDFD26789EB3002D93
:107440005ED068682E7870B3032E0BD0112E45D015
:10745000022E28D16978012925D00B0623D4FFF705
:107460005FFB20E06B78012B07D10078012802D068
:10747000022800D008B905F003F900250DF11F001E
:107480008DF81F5005F042F91F4A4C231370072353
:1074900093709DF81F305570012041330521D07045
:1074A0001371FEF703FF237C052B15D894F90A20EE
:1074B000059294F909200492144A52F82330039358
:1074C00094F90830CDE901630022E3680093114686
:1074D0000F4B03200EF052F908B070BD6B78012BF2
:1074E000E1D102780B4B02F001021A702AB90A4B63
:1074F000114603200EF042F9D5E7084B0022F7E7CA
:107500002E46D0E77C200020D02100207C7F03087D
:107510002B7F0308AC200020187F0308227F03087C
:10752000034B0022C3E902220122C3E90022704773
:107530006C220020004870476C2200204FF0B043BE
:1075400082B0DA6C0243DA64DB6C03400193019B86
:1075500002B070472DE9F04186B000240220154D9D
:107560000594FFF7EBFF0420FFF7E8FF124F0394A9
:107570004FF4807601230DEB0001CDE9016328462D
:10758000032304934FF4005801F04AF801A9384648
:10759000CDF8048001F044F822464146384601F017
:1075A00065F928462246314601F060F9204606B0CA
:1075B000BDE8F0810004004800080048032810B529
:1075C0000ED8012810D868B902460B484FF48071D4
:1075D00001F04CF9002209484FF4005101F046F93E
:1075E000002010BD0122F0E7002203484FF4807113
:1075F00001F03CF90122EEE70004004800080048D1
:10760000022070470020704701207047002814BFF7
:1076100016200F20704700000D48854600F025F821
:107620000C480D490D4A002302E0D458C4500433DD
:10763000C4188C42F9D30A4A0A4C002301E01360B3
:107640000432A242FBD328F023F8FBF757FDFEE7F4
:107650000000012000000020C008002040E60308D0
:10766000C008002098420020FEE7704710B50320B4
:1076700000F06EFC01F07CFA064B18600F20FCF75E
:1076800083FA044618B9FBF7AFFE204610BD01246B
:10769000FBE700BF240400204FF0E022136923F031
:1076A0000203136170474FF0E022136943F00203B5
:1076B00013617047014BD3F8900570470070FF1FAE
:1076C000014BD3F8940570470070FF1F014BD3F8AE
:1076D000980570470070FF1F024A536843F001038A
:1076E00053607047002004E0024A536843F00203ED
:1076F00053607047002004E0024A536843F00403DB
:1077000053607047002004E08068C0F38000704739
:10771000F7B5002301930446002800F0E980856D49
:1077200025B9FBF775F9E56584F8545023689A6824
:10773000D00040F1A1809A68D10000F1B480A26D20
:1077400042F01002A265E26D42F00102E2650125FD
:107750001846FFF7D9FFA26D02F01002024340F075
:10776000C980A26D206922F4817242F00202A265F2
:107770009A68D2075DD4226BA67E94F82CC0003A9A
:1077800018BF01221703D4E902120A43217E42EAFC
:107790008132617E42EAC13242EA4632002842EA40
:1077A0004C02B4BF20F000414FF400113A430A43A9
:1077B00094F82010012903D1002E76D142F48032B2
:1077C000616A21B1A66A01F4E07131430A43D968C4
:1077D000E66C21F4FE3121F4FF711143D96094F875
:1077E0003C206168012A01F0404C4CEA060609D1B0
:1077F000D4E910273A433243A66C324342EA0C02E2
:1078000042F001061F693E4A3A4032431A6121F0B4
:107810000042B2F1804F0CD0B1F1004F09D0394E87
:10782000D6F8082701F4701122F470120A43C6F842
:1078300008275A69666BA16B22F0070232435A612E
:107840005A6922F0700242EA01125A61002835D1C9
:107850009A6A62F00F029A625B6903F007039E4224
:107860003CD10023E365A36D23F0030343F0010340
:10787000A365284603B0F0BD9A68234922F0104260
:1078800022F0170242F080529A60204A1268B2FB3E
:10789000F1F2013252000192019A002A3FF44BAFFB
:1078A000019A013AF7E7002552E7A16D41F0200166
:1078B000A165E16D41F00101E16581E7B0F5001FCF
:1078C000CAD19A6AE269013A92006FF00F0102F0A0
:1078D0001C0201FA02F2216E0A43BCE7A36D23F0F9
:1078E000120343F01003A365E36D43F00103E36566
:1078F0000125BEE7A36D43F01003A365F8E700BFC1
:1079000002FCFF1F00200140400D03002404002062
:10791000F8B54569082D04460E460AD00368DB68B1
:10792000D80705D5A36D43F02003A3650120F8BD5A
:107930000425FCF72BF9074623681A682A4220D051
:10794000A26D42F40072A265DA6812F4406F14D19D
:10795000A27E92B91A6812070FD51846FFF7D4FE17
:1079600020BB5A6822F00C025A60A26D22F4807289
:1079700022F0010242F00102A265227EFAB100204B
:10798000D5E7711CD9D0FCF701F9C01BB04201D872
:10799000002ED1D123681B682B40CDD1A26D84F875
:1079A000543042F00402A2650320C0E7A26D42F009
:1079B0002002A265E26D42F00102E265DDE70C22E1
:1079C0001A60DCE70368186C70470000F7B5002305
:1079D000019390F85430012B044600F0C0800568F4
:1079E0000269012380F854302846FFF78DFE0028F5
:1079F00040F0AF80D1E90030022822F004027ED0AE
:107A0000B2F1004FC3F3110E35D1AA6A42EA0E0259
:107A1000AA628A68686902EA032222F07C4222F0A4
:107A2000FF0220EA03210A43002B6A611DDA4D4A56
:107A30004D4DD2F80817AB4201F0E07043D10D0272
:107A400013D4D2F8083723F0E073034343F4000360
:107A5000C2F80837454B1A68454BB2FBF3F20C23CA
:107A600002FB03330193019B53BB0020002384F8E6
:107A7000543003B0F0BD226E00F01F074FF00F0C22
:107A80000CFA07FC6FEA0C0622EA0C0CBEF1000FA0
:107A900011D1C3F38462BA4042EA0C022266800824
:107AA000E26901309042B4D8A86AC3F38362BA4055
:107AB00006403243ACE793FAA3F2B2FA82F2EAE765
:107AC000019B013BCEE72B4DAB420BD1C901CCD47E
:107AD000D2F8083723F0E073034343F08073C2F811
:107AE0000837C2E7244DAB42BFD14B02BDD4D2F818
:107AF000083723F0E073034343F48003EFE7B2F168
:107B0000004F01BFAA6AC3F311018A43AA62002B86
:107B1000ABDA154813498342D1F8082709D1D1F8C7
:107B2000083702F0A07223F0E0731A43C1F8082767
:107B30009BE71048834204D1D1F8083702F4400291
:107B4000F1E70D48834290D1D1F8083702F0C072B6
:107B5000E9E7A26D42F02002A265184686E70220FE
:107B600087E700BF00200140001000B0240400207F
:107B7000400D0300004000B8002000B4026838B592
:107B800004461046FFF7C0FD08B9002038BD9368D1
:107B9000990707D4936823F0004323F0170343F0B9
:107BA00010039360FBF7F2FF054623689B685B07B1
:107BB000EBD5FBF7EBFF401B0228F6D923689B6847
:107BC0005A07F2D5A36D43F01003A365E36D43F0AC
:107BD0000103E3650120D9E773B50023026801932F
:107BE0009368DD07044602D5002002B070BD91689D
:107BF000214B194209D0A36D43F01003A365E36D37
:107C000043F00103E3650120EFE7936823F00043AD
:107C100023F0170343F001039360184BD3F80837A0
:107C200018021CD4637E012BDED0FBF7AFFF144E8D
:107C3000054622681368DB07D6D49368D9075FBF6F
:107C40009368334043F001039360FBF79FFF401BB1
:107C50000228EED923681B68DA07EAD4CBE7094B80
:107C6000094A1B68B3FBF2F301330193019B002B1C
:107C7000D8D0019B013BF8E71700008000200140AD
:107C8000E8FFFF7F24040020400D030038B50446C0
:107C90000068FFF739FD054620BB94F85430012BEE
:107CA00020D0012384F854302046FFF795FFB0B967
:107CB000A36D226823F4706323F0010343F48073FF
:107CC000A3651C23E065136084F85400936823F0D7
:107CD000004323F0170343F00403936038BD84F896
:107CE0005450FBE70220F9E7026838B593689168C1
:107CF0000446C80701D4002038BD9907FBD4936817
:107D000003F00503012B19D1936823F0004323F0FE
:107D1000170343F00203936003231360FBF736FF5E
:107D2000054623689B68DB07E5D5FBF72FFF401B63
:107D30000228F6D923689B68DA07F2D5A36D43F0D1
:107D40001003A365E36D43F00103E3650120D3E76E
:107D500070B5044600284BD0836D43F00203836561
:107D6000FFF70CFF054668B92046FFF7BDFF054643
:107D700008B90123A3652268936823F0104323F018
:107D80001703936023685A6822F4677222F0030293
:107D90005A6040F29F321A60D968164A0A40DA6087
:107DA0001A6922F040421A615A6922F007025A61A8
:107DB0001A6A02F0F0221A625A6A02F0F0225A623B
:107DC000DA6A02F0F022DA629A6A0B4A00269E62B0
:107DD000D2F8083723F0FE73C2F808372046FAF7C6
:107DE0002BFEE6652666A66584F85460284670BDBD
:107DF0000125FBE700023E830020014010B590F80A
:107E00005430012B044615D0012380F85430FFF77D
:107E1000B5FE58B92046FFF767FF38B9A36D23F4C4
:107E2000807323F0010343F00103A365002384F86A
:107E3000543010BD0220FCE7F7B50023019390F801
:107E40005430012B04467FD0012380F85430FFF7D3
:107E50004BFF23689A6812F00102054607D0A36D14
:107E600043F01003A365002384F854302DE0A16D86
:107E7000364F21F4817141F00201A165DE68D968B5
:107E800026F4FF4626F07C0621F40041360421F05A
:107E90000301360CD96008209968394041F000414F
:107EA00099609968002913DA0199013101910199CA
:107EB000B1F52E3FF5D3A36D23F0120343F0100369
:107EC000A365002384F854300125284603B0F0BD93
:107ED000D3F8B410013801F07F010A44DCD199686D
:107EE0001A48014041F001019960D3F8B41021F023
:107EF0007F0141EAD202C3F8B4209A68024042F0FE
:107F000002029A60FBF742FE074623689A68D2078E
:107F100008D4DA683243DA60A36D23F0030343F038
:107F200001039FE7FBF732FEC01B0228EDD923684F
:107F30009B68D907E9D5A36D43F01003A365E36DF2
:107F400043F00103E365BFE70225BEE7E8FFFF7FDB
:107F50000749CA6822F4E0620302120403F4E063F2
:107F6000120C134343F0BF6343F40033CB607047FC
:107F700000ED00E0164B30B5DC68C4F30224C4F118
:107F80000703251D042B28BF0423062D4FF0FF35C2
:107F90008CBF033C002405FA03F321EA0303A54048
:107FA00022EA0502A340002843EA0203ACBF00F125
:107FB0006040084A4FEA0313B8BF00F00F00DBB27D
:107FC000AABF00F56140135480F8003330BD00BFF4
:107FD00000ED00E014ED00E0002807DB044A410951
:107FE000012300F01F00834042F82130704700BF9A
:107FF00000E100E000280CDB4309064900F01F0007
:1080000020330122824041F82320BFF34F8FBFF37A
:108010006F8F704700E100E070B5D0E913456560EF
:10802000446D14B1D0E916456560D0E9105404F0F0
:108030001C060124B4406C60046863608368102BE4
:108040000BBFA260A160E160E26070BD0268416C9C
:10805000D3B210B5083B1424B3FBF4F30B4CA2428B
:1080600088BF0B4A21F0030199BF01F1804202F55C
:108070000232521807338264064AC26403F01F03B7
:10808000012202FA03F3036510BD00BF070402409A
:108090001C0802408008024038B500285CD0026805
:1080A0002E4B9A424FF014014AD82D4B1344B3FB88
:1080B000F1F32C499B00C0E91013022380F825300E
:1080C0001368056923F4FF4323F070031360D0E9BC
:1080D000024323432B43456911682B4385692B4396
:1080E000C5692B43056A2B430B431360FFF7AEFFB3
:1080F000B4F5804F04BF002343604368816C03F0F4
:108100007F020A60D0E91314013B032B4C601ED898
:10811000154B1649816513449B000121013A01FA70
:1081200002F200214365C2651960114B5A640023B5
:108130000122C36380F8243080F82520184638BD1A
:108140000C4B1344B3FBF1F30B499B00B3E7002343
:10815000C0E91533C365EAE70120F0E707040240F0
:10816000F8FFFDBF000002403F82001040090240BE
:1081700000090240F8FBFDBF0004024038B50028AA
:1081800041D00268136823F0010313601F4B9A4229
:108190004FF0140130D81E4B1344B3FBF1F31D49CB
:1081A0009B00C0E91013012403F01C0304FA03F33D
:1081B000002515604B60FFF749FF836C41681D6027
:1081C000D0E913325A604A1E032A06D8124B0B44D8
:1081D0009B0094401D60114B5C640023C363C0E9A5
:1081E0001533C0E90B33C0E90D33C36580F8253082
:1081F00080F82430184638BD094B1344B3FBF1F323
:1082000008499B00CDE70120F5E700BF07040240C5
:10821000F8FFFDBF000002403F820010000902404D
:10822000F8FBFDBF0004024070B590F82450012D0A
:1082300004463BD090F825600125AE4280F82450DA
:108240004FF000062CD1022580F825500568C66342
:108250002E6826F001062E60FFF7DEFE036BBBB131
:108260002B6843F00E032B60A36C1A68D20342BF45
:108270001A6842F480721A60636D1BB11A6842F486
:1082800080721A602B6843F001032B60002070BDE0
:108290002B6823F004032B602B6843F00A03E2E70A
:1082A0008023C36380F824602846F0E70220EEE7CD
:1082B000034640B190F82520022A06D00422C2636A
:1082C000002280F82420012070470268806C116829
:1082D00021F00E011160016821F4807101601168C4
:1082E00021F001011160D3E9100202F01C0101220A
:1082F0008A404260D3E9132151605A6D32B111684E
:1083000021F480711160D3E916215160012200200F
:1083100083F8252083F82400704708B590F82530AD
:10832000022B03D00423C363012008BD03681A682D
:1083300022F00E021A601A6822F001021A60826CA2
:10834000136823F480731360D0E9101303F01C0248
:10835000012393404B60D0E913325A60436D33B12F
:108360001A6822F480721A60D0E916325A6001232A
:1083700080F82530002380F82430836B03B19847C0
:108380000020D2E770B4426C046C036826681D6854
:1083900002F01C020421914031420FD015F0040F6D
:1083A0000CD01A6892065EBF1A6822F004021A60A6
:1083B000036B6160002B33D070BC184702219140E1
:1083C000314217D015F0020F14D01A68940606D463
:1083D0001A6822F00A021A60012280F82520114A48
:1083E00093428CBF104B114B5960002380F824300E
:1083F000C36ADFE708219140314211D029070FD528
:10840000196821F00E011960012303FA02F262607B
:10841000C36380F82530002380F82430436BC9E71C
:1084200070BC70478000024000040240000002401F
:108430000A4A536943F4802330B55361EFF3108443
:1084400072B60023CD58C5500433B3F5807FF9D1FF
:108450001369DB03FCD484F3108830BD004000585E
:10846000064B5A69002ABFBF054A9A6002F188325A
:108470009A60BABF5869C00F00207047004000588A
:1084800023016745044B5A6942F000425A6158691A
:10849000C043C00F704700BF0040005870B505468C
:1084A000FBF774FB124E04463369D90313D43369C6
:1084B000DA0744BF012232614CF2FA32134011D183
:1084C0000B4E306910F480200BD0FBF75FFB001BD4
:1084D000A842F6D304E0FBF759FB001BA842E3D304
:1084E000032070BD024A1361024A01205360F8E77D
:1084F000004000587C2200202DE9F041184D98469C
:108500002B78012B06460C46174626D001232B70EC
:108510004FF47A7000236B60FFF7C0FFA0B9012E03
:1085200016D1104A536943F0010353612760BFF32A
:108530006F8FC4F804804FF47A70FFF7AFFF094AD9
:10854000536923EA0603536100232B70BDE8F081D1
:1085500039462046FFF76CFFEDE70220F6E700BF43
:108560007C22002000400058054A536923F47E73A2
:1085700043EAC00040F4803040F002005061704790
:10858000004000582DE9F041234F3B78012B054670
:1085900088463FD001233B704FF47A7000237B6004
:1085A000FFF77CFF044688B92B68042B13D11B4AC4
:1085B000536943F4803343F0040353614FF47A70FA
:1085C000FFF76CFF0446154B1A681B6800233B70CD
:1085D0002046BDE8F0814FF0FF33C8F800306E68E8
:1085E000D5E901321344B3420AD93046FFF7BCFF44
:1085F0004FF47A70FFF752FF50B1C8F8006004469C
:10860000064A536923F47E7323F002035361DAE7C9
:108610000136E5E70224DBE77C2200200040005819
:108620002DE9F04F524C00234FF00F090A6832FA3F
:1086300003F501D1BDE8F08F012505FA03F818EA2A
:10864000020200F08E804E68032706F003054FEA11
:10865000430E07FA0EFC6F1E012F6FEA0C0C32D886
:10866000876807EA0C0ACF6807FA0EF747EA0A0795
:108670008760476827EA0808C6F300179F4047EA63
:1086800008074760C76807EA0C088F6807FA0EF703
:1086900047EA0807022DC76017D14FEAD30800EB5D
:1086A000880803F0070AD8F820704FEA8A0A09FA06
:1086B0000AFB27EA0B0B0F6907FA0AF747EA0B07D1
:1086C000C8F8207001E0032DDCD1076805FA0EF52B
:1086D00007EA0C073D4316F4403F056041D023F004
:1086E000030707F1804707F5803703F0030CBD68E7
:1086F0004FEA8C0C4FF0070E0EFA0CFEB0F1904FC3
:1087000025EA0E0E2FD01B4DA8422ED005F5806510
:10871000A84214BF0725022505FA0CF545EA0E0507
:10872000BD602568D74316F4801F0CBF3D4015433C
:108730002560656816F4001F0CBF3D401543656059
:10874000D4F8805016F4803F0CBF3D401543C4F868
:108750008050D4F88450B60354BF3D401543C4F84C
:108760008450013362E70025D6E70125D4E700BF36
:108770000008005800040048374A2DE9F04F002354
:108780004FF0010A4FF0070B4FF00F0931FA03F4D5
:1087900001D1BDE8F08F0AFA03FC1CEA010654D0AF
:1087A00023F0030404F1804404F5803403F003074C
:1087B000A568BF000BFA07F8B0F1904F08EA050E64
:1087C00045D0264DA84244D005F58065A8420CBF8F
:1087D00002250725BD40754517D1D2F8805025EAFE
:1087E0000605C2F88050D2F8845025EA0605C2F882
:1087F0008450156825EA06051560556825EA0605C2
:108800005560A56825EA0805A560056803265C0093
:1088100006FA04F423FA06F6254300EB8606056003
:1088200003F00705376AAD0009FA05F527EA0507E1
:108830003762856825EA04058560456825EA0C05E8
:108840004560C56825EA0404C46001339EE700253D
:10885000C0E70125BEE700BF00080058000400483B
:108860000369194214BF0120002070470AB18161D9
:10887000704781627047436901EA030221EA0301FC
:1088800041EA024181617047044AD168014208B55A
:1088900002D0D060FDF78EFC08BD00BF0008005874
:1088A000024A136843F48073136070470004005851
:1088B0000D4B10B55B690C4628B99A0507D500F039
:1088C00027F820B110BD9B0501D400F019F8074A24
:1088D0001369012C23F00403136101D130BFF1E7C8
:1088E00040BF20BF20BFEDE70004005800ED00E0CE
:1088F000024B186800F4C060704700BF00040058C5
:10890000024A136843F48043136070470004005820
:108910000C4A136823F4804313600B4B1B6832210D
:108920004B430A49B3FBF1F35169890500D533B9CB
:10893000536913F4007F14BF032000207047013BEC
:10894000F2E700BF000400582404002040420F005A
:108950000B4A136823F0070343F002031360094B2B
:108960001A69012842F004021A6105D130BF1A6960
:1089700022F004021A61704740BF20BF20BFF6E713
:108980000004005800ED00E04FF0B0431868C0F359
:10899000404070474FF0B0431868C0F34000704744
:1089A0004FF0B042536823F47F4343EA00235360FF
:1089B00070474FF0B0431868C0F340607047000044
:1089C0007FB54FF0B0432C4AD3F80831C0F3031001
:1089D00003F00F0352F82040284A52F82330B4FB2A
:1089E000F3F4FFF785FF264B054693E80700B5F53E
:1089F000007F04AB03E9070010D0224B9C4218D340
:108A000003F5B70303F67F539C4229D903F574138A
:108A100003F510639C4225D802230BE01A4B9C42BD
:108A200007D91A4B9C421BD903F5370303F5D853DA
:108A3000F0E7002304AA02EB830353F80C4C144D17
:108A40002B6823F0070323432B60FBF79FF80646B0
:108A50002B6803F007039C4206D1002004B070BDD0
:108A60000123E7E70024EAE7FBF790F8801B0228E0
:108A7000EED90320F2E700BF947F0308F47F0308D8
:108A8000B82B0308C0CF6A00BFEA21013F9334022C
:108A9000004000584FF0B04310B59A68D96812F002
:108AA0000C0205D00C2A4AD101F00303012B51D14D
:108AB0004FF0B0412B480B6813F0080306D00B6849
:108AC00013F0080337D1D1F8941007E00C6824079D
:108AD00056BFD1F894300968C3F3032350F823300C
:108AE000002A0CBF184600204FF0B0418A6802F0FF
:108AF0000C020C2A1ED1CA6802F00302022A2ED0F0
:108B0000032A06D10B68184A13F4801F174B18BFAD
:108B100013464FF0B042D068D168D268C0F3062047
:108B20005843C1F302130133B0FBF3F0530F013389
:108B3000B0FBF3F010BD0B68C3F30313CEE7042AB8
:108B400005D0082A06D11B6813F4801305D0064807
:108B50000023C9E700231846C6E70448C4E7024BD0
:108B6000D7E700BF947F03080024F4000048E80121
:108B700008B5FFF78FFF4FF0B043044A9B68C3F37B
:108B8000031352F82330B0FBF3F008BDF47F030861
:108B90002DE9F0410446002853D04FF0B0439D68C2
:108BA000DE6803689B0605F00C0506F0030668D531
:108BB000026A1DB10C2D46D1012E44D1002A40D0AD
:108BC0004FF0B043A16A1A68170756BFD3F8943024
:108BD0001B681B0903F0F00399421FD90846FFF7F1
:108BE000EFFE00282DD14FF0B042136843F0080388
:108BF00013601368A16A23F0F0030B431360606AEB
:108C0000FFF7CEFEFFF7B4FFAB4B1860AB4B186815
:108C1000FAF7BAFF002834D0BDE8F0814FF0B04237
:108C2000136843F008031360136823F0F0030B4349
:108C30001360606AFFF7B4FE0846FFF7C1FE002824
:108C4000E0D00120E8E74FF0B043002A54D01A6882
:108C500042F001021A60FAF799FF0746FFF79AFE01
:108C6000002842D04FF0B042136843F0080313606D
:108C70001368A16A23F0F0030B431360606AFFF7E7
:108C80008FFE2368D80748D42368990700F18C80A9
:108C900023681E0740F1FA80A3694FF0B046002B0D
:108CA00000F0E180D6F89430E16903F010029142BF
:108CB00000F0C48003F00302022AC2D0D80740F1BA
:108CC000B380D6F8943023F00103C6F89430FAF755
:108CD0005DFF0746D6F89430990740F1A580FAF772
:108CE00055FFC31B112BF5D904E0FAF74FFFC01B4A
:108CF0000228B3D903208FE71A6822F001021A6014
:108D0000FAF744FF0746FFF745FE0028B9D0FAF707
:108D10003DFFC01B0228F6D9ECE7082D03D00C2D2F
:108D200005D1032E03D16368002BADD189E74FF045
:108D3000B043A1681A6822F480120A431A6062687C
:108D4000B2F5803F10D11A6842F480321A60FAF707
:108D50001DFF0746FFF718FE002895D1FAF716FF0A
:108D6000C01B6428F6D9C5E7B2F5041F04D11A6800
:108D700042F400121A60E6E7196821F480311960A4
:108D8000196821F400111960002AE0D1FAF7FEFEFB
:108D90000746FFF7F9FD00283FF476AFFAF7F6FE35
:108DA000C01B6428F5D9A5E7042D236903D00C2D39
:108DB0000ED1022E0CD1002B3FF443AF4FF0B04246
:108DC0006169536823F0FE4343EA016353605FE740
:108DD0004FF0B046BBB1336843F480733360FAF7A9
:108DE000D5FE074633685A0505D4FAF7CFFEC31BF4
:108DF000022BF7D97EE77368626923F0FE4343EAEA
:108E00000263736044E7336823F480733360FAF7D6
:108E1000BDFE074633685B057FF53AAFFAF7B6FE4D
:108E2000C31B022BF6D965E74FF0B042E169D2F8D7
:108E3000943023F010030B43C2F894304FF0B04746
:108E4000D7F8943043F00103C7F89430FAF79EFE48
:108E50000646D7F894309A0718D4FAF797FE831B82
:108E6000112BF6D946E7D6F8943023F00103C6F863
:108E70009430FAF78BFE0746D6F894309B0705D559
:108E8000FAF784FEC31B112BF6D933E72368580782
:108E900054D50B4F3B68D90514D4FFF701FDFAF701
:108EA00075FE06463B68DA050CD4FAF76FFE831BA5
:108EB000022BF7D91EE700BF24040020280400205D
:108EC00000040058E3684FF0B046002B58D023F060
:108ED0008003052B02BFD6F8903043F00403C6F898
:108EE00090304FF0B046FAF751FED6F8903043F08C
:108EF00001030746C6F8903041F28838D6F8903022
:108F00009B0705D4FAF742FEC31B4345F6D9F1E6A9
:108F1000E36823F00403812B1BD1FAF737FED6F860
:108F2000903043F08003C6F8903007464FF0B046CB
:108F300041F28838D6F89030180504D5E36A002B42
:108F40004AD1002068E6FAF721FEC01B4045F1D95E
:108F5000D0E6FAF71BFED6F8903023F08003C6F86F
:108F6000903007464FF0B04641F28838D6F890303E
:108F70001905E3D5FAF70AFEC01B4045F6D9B9E654
:108F8000FAF704FED6F8903023F080030746C6F8BF
:108F9000903041F28838D6F890301A0516D4FAF796
:108FA000F5FDD6F8903023F00103C6F8903007465F
:108FB0004FF0B04841F28836D8F890309B07BDD5C5
:108FC000FAF7E4FDC31BB342F6D993E6FAF7DEFDE8
:108FD000C01B4045DFD98DE60C2D4ED0022B4FF043
:108FE000B0431A6822F080721A6033D1FAF7CEFDCE
:108FF0000546FFF7DEFC38BBD4E90C314FF0B04238
:109000000B43D0682D4901400B43E16B0B43216CAE
:109010000B43616C0B43A16B43EA0123D3601368DC
:1090200043F080731360D36843F08053D360FAF742
:10903000ADFD0446FFF7BDFC002882D1FAF7A6FD7E
:10904000001B0A28F6D955E6FAF7A0FD401B0A28AE
:10905000CFD94FE6FAF79AFD0446FFF7AAFC30B9DC
:109060004FF0B042164BD1680B40D36069E7FAF776
:109070008DFD001B0A28F0D93CE6012B3FF4E1AD41
:109080004FF0B043D868236B00F003029A427FF49C
:10909000D8AD626B00F0700393427FF4D2ADA26B47
:1090A00000F4FE43B3EB022F7FF4CBAD636C00F012
:1090B0006040C01A18BF0120AEE500BF8C80C1110E
:1090C000FCFFFEEE2DE9F0410D46044610B90120EB
:1090D000BDE8F081684E336803F007038B4216D376
:1090E00023689A0727D54FF0B047A268BB6823F0E2
:1090F000F0031343BB60FAF749FD0646BB68DB0388
:1091000019D4FAF743FD831B022BF7D911E033681A
:1091100023F007030B433360FAF738FD0746336843
:1091200003F00703AB42DBD0FAF730FDC01B022887
:10913000F5D90320CCE72368580617D54FF0B04780
:109140006269D7F8083123F00F0343EA1213C7F816
:109150000831FAF71BFD0646D7F80831D90305D4C4
:10916000FAF714FD831B022BF6D9E2E723685A07AE
:1091700013D54FF0B047E268BB6823F4E0631343B4
:10918000BB60FAF703FD0646BB689B0305D4FAF7FC
:10919000FDFC831B022BF7D9CBE72368180714D5F6
:1091A0004FF0B0472269BB6823F4605343EAC2031F
:1091B000BB60FAF7EBFC0646BB68590305D4FAF727
:1091C000E5FC831B022BF7D9B3E72368DA070FD43A
:1091D000294C236803F00703AB4239D8FFF7C8FCDA
:1091E000264B1860264BBDE8F0411868FAF7CCBC56
:1091F0006268022A1DD1FFF7C7FB00283FF467AF62
:109200004FF0B04641F28838B36823F003031343AC
:10921000B360FAF7BBFC0746B368626803F00C035F
:10922000B3EB820FD4D0FAF7B1FCC01B4045F3D9A1
:109230007FE7032A02D1FFF7BCFBDEE712B9FFF795
:10924000A9FBDAE74FF0B0431B685B05D8D43EE7D3
:10925000236823F007032B432360FAF797FC0646A5
:10926000236803F00703AB42B8D0FAF78FFC801BEA
:109270000228F5D95DE700BF004000582404002013
:109280002804002008B5FFF773FC4FF0B043044AF0
:109290009B68C3F3022352F82330D84008BD00BFB7
:1092A000D47F030808B5FFF763FC4FF0B043044ACE
:1092B0009B68C3F3C22352F82330D84008BD00BFD7
:1092C000D47F03084FF0B043D3F89000C0F34000C0
:1092D00070474FF0B0410209D1F8883002F47F2284
:1092E000000123EA020300F47F200343C1F8883021
:1092F00070474FF0B041020CD1F88830120423EAD5
:10930000020343EA0040C1F8880070470368DA03AB
:1093100070B5044639D5FFF7C3FAFAF737FC614E4A
:1093200005463368DB0532D54FF0B043616BD3F8A7
:10933000902002F4407291421DD0D3F89010D3F8DF
:10934000902042F48032C3F89020D3F8902021F48A
:10935000407022F480328D07C3F89020C3F890004B
:1093600009D5FAF713FC41F288360546FFF7AAFF44
:10937000012840F090804FF0B042616BD2F89030FD
:1093800023F440730B43C2F89030002605E0FAF74F
:10939000FDFB401B0228C4D903262568E8070AD52F
:1093A0004FF0B0416268D1F8883023EA124392B29C
:1093B0001343C1F88830A9070AD54FF0B041A2681D
:1093C000D1F8883023EA124392B21343C1F88830AF
:1093D000AA0609D54FF0B0422169D2F8883023F4AB
:1093E00040630B43C2F88830AB0502D5206AFFF713
:1093F00080FF680502D5606AFFF77BFF290502D56B
:10940000A06AFFF776FF6A0602D56069FFF761FF81
:109410002B0602D5A069FFF75CFFE80502D5E069DD
:10942000FFF757FFE90610D54FF0B042E168D2F8D8
:10943000883023F440730B43C2F88830B1F5807F45
:1094400002BFD36843F08073D3602A040ED54FF077
:10945000B042216BD2F8883023F040430B43C2F86E
:10946000883019B9D36843F08073D3606B0410D58A
:109470004FF0B042E16AD2F8883023F040530B43FA
:10948000B1F1005FC2F8883003D1D36843F4803370
:10949000D360304670BDFAF779FB401BB0427FF6CF
:1094A00065AF79E70004005830B590F82C30012BF7
:1094B00002464FF0020022D0174B82F82D00CA243A
:1094C000012582F82C505C6253245C62B1F5807FE8
:1094D000146B996914D121F488519961596C24F065
:1094E000010421F0004159641463DD650A4BFF213A
:1094F00059620020012382F82D3082F82C0030BD03
:1095000021F408519961D96C24F0020421F0004142
:10951000D9641463D865E9E70028004070B50B4EA4
:10952000036B756D1D40EA07044603D50123F365FF
:10953000FAF7BFFDAB0704D50223F365204600F020
:10954000C9F9012384F82D3070BD00BF0028004008
:1095500038B50A4CE36823F02003E360FAF716FB02
:109560000546E3689B0601D5002038BDFAF70EFBDF
:10957000401BB0F57A7FF4D90320F6E700280040BD
:10958000F8B5114DEC6814F0400406461AD1EB68AA
:1095900043F08003EB60FAF7F9FA23460746EC68DC
:1095A00014F0400401D1032B01D11846F8BDFAF79D
:1095B000EDFAC01BB0F57A7F234684BF032386F8FB
:1095C0002D30ECE70023F0E70028004038B50F4CC1
:1095D000E36823F08003E360A3699B06054606D495
:1095E000FFF7B6FF10B1032085F82D0038BDA36941
:1095F00023F02003A361FFF7ABFF10B1032085F830
:109600002D00A36943F02003A361EFE70028004089
:1096100038B5044600284BD090F82D3003F0FF02F7
:109620001BB980F82C20F9F7C3FD0223214D84F8E3
:109630002D30EB68DB0636D4CA236B6253236B6292
:109640002046FFF79DFF10B1FF236B6238BDAB6969
:1096500023F08E6323F04003AB6121696368AA693C
:109660000B431343A2691343AB61D4E9022343EADA
:1096700002432B61D4E90931EA680B4322F4F85222
:109680001343EB602046FFF7A1FF0028DCD1D4E9AB
:109690000713AA690B4322F0604213436269134324
:1096A000AB61FF236B62012384F82D300020CDE7EE
:1096B0000120CBE7002800400023092803D840EA16
:1096C0000310C0B270470A380133C0B2F5E700009A
:1096D0002DE9F04790F82C30012B05464FF00200A1
:1096E00069D0012385F82C304E4B85F82D00DE68BB
:1096F00006F44076B6F5807F78D04C69087891F80A
:10970000019091F802A091F82470002A55D19B692C
:1097100013F0400308BFCB70FFF7CEFF80464846EA
:10972000FFF7CAFF02465046FFF7C6FF814638469C
:10973000FFF7C2FF0B6ACF78234343EA875343EA1C
:10974000090343EA084343EA022343EA0063354A34
:10975000CA205062532050628C6A8869B4F5807FB9
:10976000946945D124F4885494610124D465B6F5F4
:10977000807F09BFCB6913640343536418BF5064EF
:10978000284B4A681A672A6B42F001022A639A69D9
:1097900042F488529A61244AD2F8803043F400336C
:1097A000C2F880301F4BFF225A620020012385F847
:1097B0002D3085F82C00BDE8F087B4F1803F07D04C
:1097C000B4F5000F04D09B6913F0400308BFCB70C1
:1097D0000B6ACA781C4344EA0A0444EA004343EA99
:1097E000092343EA825343EA0763B0E70023AEE765
:1097F00024F4085494610224D465B6F5807F09BF2F
:10980000CB6993640343D36418BFD064054B4A68A3
:109810005A672A6B42F002022A639A6942F408529C
:10982000B8E700BF002800400008005890F82C203E
:10983000012A03464FF0020012D00A4A83F82D0095
:10984000CA21516253215162916941F02001916115
:10985000FF2151620020012283F82D2083F82C0083
:10986000704700BF0028004090F82C20012A0346D2
:109870004FF0020019D00D4A83F82D00CA21516221
:109880005321516291690A4841F080019161D0F8F9
:10989000801041F48021C0F88010FF215162002027
:1098A000012283F82D2083F82C0070470028004007
:1098B00000080058064B5A6D520610B5044603D5F1
:1098C0004022DA65FAF7F8FB012384F82D3010BD49
:1098D000002800407047890001F1804101F53141C5
:1098E0000A607047890001F1804101F53141086843
:1098F000704700002DE9F3471F468946904604460D
:10990000FAF744F90A9D3D442D1AFAF73FF9264B20
:109910001E68C6F3CB366E43824601962268936872
:1099200039EA03030CBF01230023434501D1002082
:109930002EE07B1CF3D0FAF729F9A0EB0A00A8422D
:1099400029D323685A6822F0E0025A606268B2F5AF
:10995000827F0AD1A268B2F5004F02D0B2F5806FC3
:1099600003D11A6822F040021A60A26AB2F5005FC1
:1099700007D11A6822F400521A601A6842F40052A1
:109980001A60012384F85D30002384F85C300320E2
:1099900002B0BDE8F087019A019B002A03F1FF3372
:1099A000019308BF1546B9E7240400202DE9F74FBD
:1099B000994600238DF80330044688461746FAF787
:1099C000E5F80C9D4D442D1AFAF7E0F82C4BD4F82D
:1099D00000B01E6823235E43360D6E438246019617
:1099E0002268936803EA0803BB4201D100203AE0F1
:1099F000B8F5C06F07D137B99BF80C30DBB28DF8E2
:109A000003309DF80330B9F1FF3FEAD0FAF7BEF812
:109A1000A0EB0A00A84229D323685A6822F0E0028A
:109A20005A606268B2F5827F0AD1A268B2F5004F2F
:109A300002D0B2F5806F03D11A6822F040021A609A
:109A4000A26AB2F5005F07D11A6822F400521A60C8
:109A50001A6842F400521A60012384F85D30002332
:109A600084F85C30032003B0BDE8F08F019A019BBD
:109A7000002A03F1FF33019308BF1546B0E700BF8A
:109A80002404002073B50B4600920D4616464FF491
:109A9000C05100220446FFF789FF024630B1236E11
:109AA00043F020032366032002B070BD00962B46CE
:109AB00080212046FFF71EFF02460028EFD10096C6
:109AC0002B464FF4C0612046FFF770FF0028EBD013
:109AD000E5E74368B3F5827FF7B504460E461746BF
:109AE0000BD18368B3F5004F02D0B3F5806F04D17A
:109AF0002268136823F04003136000973346002266
:109B000080212046FFF7F6FE054628B1236E43F07C
:109B100020032366032514E06368B3F5827F10D128
:109B2000A368B3F5004F02D0B3F5806F09D1009759
:109B3000334600224FF4C0612046FFF737FF00286C
:109B4000E4D1284603B0F0BDF8B5044600287ED025
:109B5000436A002B50D14268B2F5827F00D0C361C6
:109B600094F85D3003F0FF0223B984F85C202046AE
:109B7000F9F784FB2268E068022384F85D301368FB
:109B8000B0F5E06F23F0400313604FF0000337D9C6
:109B90001D46B0F5706F18BFA362A7686368A1691E
:109BA000A66A07F4044703F482733B43276907F06E
:109BB00002073B43676907F001073B4301F4007765
:109BC0003B43E76907F038073B43276A07F0800704
:109BD0003B4306F400573B43B6F5005F136014D1D6
:109BE000236B8BBBB0F5E06F0DD9022323631368A1
:109BF00043F40063136008E00023C0E90433AFE7D7
:109C00004FF48055C7E701232363636A676B03F052
:109C1000100307F0080700F470603B43090C03438E
:109C200001F004010B432B43B6F5005F536004BF02
:109C3000A38D1361D36923F40063D3610020012352
:109C4000206684F85D30F8BD022BDED1CFE701201D
:109C5000F9E7000070B5044690F85C00012800F0B8
:109C6000CF80012084F85C0094F85D0066680128CC
:109C7000C5B20AD0B6F5827F40F0C080A068002847
:109C800040F0BC80042D40F0B980002951D0002A5A
:109C90004FD0002B4DD094F85D00A16304281CBF69
:109CA000052084F85D0000202066C4E91300A06A46
:109CB000E387B0F5005F2168A3872264A4F84430ED
:109CC000A4F8463007D1086820F4005008600868FE
:109CD00040F400500860486820F4C0404860E068E4
:109CE000B0F5E06FA06D29D94B6823F480534B6029
:109CF00094F85D30434E444D042B444B18BF1D4631
:109D0000434B18BF3346C0E90B35424B4363002336
:109D10008363B4F846300C319BB2FEF785FA0346F4
:109D2000002848D0236E43F010032366012384F8F3
:109D30005D300120002384F85C3070BD4D6845F42F
:109D400080554D60656DAD69B5F5806F0AD113F032
:109D5000010F4B681ED123F480434B60E38FC3F3A4
:109D60004E03E3878369B3F5806FC1D14B6823F459
:109D700080534B60B4F8463013F0010F4B6811D19B
:109D800023F400534B60B4F84630C3F34E03A4F8F9
:109D90004630ADE743F480434B60E38FC3F34E039B
:109DA0000133DEE743F400534B60B4F84630C3F3AD
:109DB0004E030133EBE72268606D516841F0010109
:109DC0005160C0E90B33C0E90D33E38FA16B9BB247
:109DD0000C32FEF729FA0028A4D123681A6852062B
:109DE0005EBF1A6842F040021A605A6842F02002D0
:109DF0005A605A6842F002025A609BE7022099E7D3
:109E000002209AE74D9F00081D9E0008299E000829
:109E1000579E0008359E00087047704708B5806A55
:109E2000FFF7FBFF08BD704708B5806AFFF7FBFF2F
:109E300008BD7047806A026808B5536823F00303C1
:109E40005360036E43F010030366012380F85D3016
:109E5000FFF7EFFF08BD7FB5064600230393846A32
:109E60008DF80B30F9F792FE33681B689A060546A9
:109E700068D42268536823F020035360A36AB3F5C3
:109E8000005F13D101220090642311462046FFF7A2
:109E900031FD18B1236E43F002032366E3682668A0
:109EA000B3F5E06F2ED9F3680393039BA268236890
:109EB000002A43D16268B2F5827F3FD15A6822F00E
:109EC00003025A6064212A462046FFF702FE08B1C9
:109ED000202323660023A4F846302268012384F857
:109EE0005D309368DB0606D5236E43F002032366DC
:109EF0004FF6EF739360236E23B32046FFF799FF6D
:109F000004B070BD337BDBB28DF80B309DF80B30A5
:109F1000236B022BCAD101220095642311462046EF
:109F2000FFF7E8FC18B1236E43F002032366337B8E
:109F3000DBB28DF80B309DF80B30B7E75A6822F092
:109F40000102BEE72046FFF767FFD9E77FB5064667
:109F500000230393846A8DF80B30F9F717FE3368FA
:109F60001B68990605465ED42268536823F02003D7
:109F70005360A36AB3F5005F1BD1E368B3F5E06FEC
:109F80003ED1236B012B3BD1009064234FF4007230
:109F90004FF4C0612046FFF709FD18B1236E43F06E
:109FA0000203236623681B7BDBB28DF80B309DF820
:109FB0000B302A4664212046FFF764FD18B1236E5A
:109FC00043F02003236623685A6822F003025A6094
:109FD0000022E287A4F84620012284F85D209A68D6
:109FE000D20606D5226E42F0020222664FF6EF72CA
:109FF0009A60236EBBB12046FFF71BFF04B070BD13
:10A00000009564234FF480624FF4C0612046FFF74F
:10A01000CDFC18B1236E43F0020323662368DB688E
:10A020000393039BC5E72046F8F746FCE6E70000EC
:10A03000036830B559689A6802F04105012D85B072
:10A04000044606D14D0604D5C36C05B0BDE83040CA
:10A050001847950704D5080602D5236D2046F4E776
:10A0600012F4B07F59D08D0657D550060FD594F80D
:10A070005D0003284FF0000549D0206E40F0040039
:10A0800020660095D8680090986800900098950622
:10A090000CD5206E40F001002066002002909868E8
:10A0A0000290186820F0400018600298D00508D58A
:10A0B000226E42F008022266002203929A680392FE
:10A0C000039A226E4AB35A6822F0E0025A600122D3
:10A0D00084F85D208A0722D05A68A06D22F003021E
:10A0E0005A6040B1104B8363FEF717F918B1236E25
:10A0F00043F040032366606D78B10B4B8363FEF73A
:10A100000CF950B1236E43F04003236605E001953E
:10A11000DA6801929B680193019B05B030BD20462F
:10A12000FFF787FEF9E700BF2DA1000808B5806A98
:10A130000023A0F84630C387FFF77BFE08BD000070
:10A14000034AD2F8903043F40043C2F8903070478D
:10A1500000040058034AD2F8903023F40043C2F8B8
:10A160009030704700040058074B1A6822F04002F4
:10A170001A6040F441704FF4B85218605A601A687F
:10A1800042F040021A6070470000015837B505469A
:10A1900000284ED0837903F0FF046BB1032C0BD061
:10A1A000254B4FF400629A612868FFF7DDFF002419
:10A1B00001232B71AC602FE000236B712846F9F767
:10A1C000F9FB1E4AD2F8903043F48053C2F8903025
:10A1D000002CE5D102234FF0B042AB71D2F894309D
:10A1E00023F40043C2F89430154B1B681C214B43E9
:10A1F000DB0C64214B430193019B93B90124AC60B8
:10A20000FFF79EFF0C4B9A6842F400629A604FF48D
:10A2100000629A61002CC7D00123AB71204603B0C5
:10A2200030BD019B013B0193D2F894305B04E3D431
:10A23000E6E70124F2E700BF0004005800080058D8
:10A240002404002037B5174D2B6802461C204343D9
:10A25000DB0C6420434314480193019B93B9012014
:10A260009060114C21732B681C214B43DB0C642143
:10A270004B430193019B6BB9012090600A4BDB6853
:10A2800003B030BD019B013B019383689C07E4D57B
:10A290000020E6E7019B013B0193A368DB07E9D5BA
:10A2A000ECE700BF240400200000015837B5184D2A
:10A2B0002B6802461C204343DB0C642043431548B3
:10A2C0000193019BA3B901209060124CFF232373DB
:10A2D0002B681C256B43DB0C64256B430193019BAE
:10A2E00073B9012090600B4BDB680B7003B030BD7D
:10A2F000019B013B019383689C07E2D50020E4E7C2
:10A30000019B013B0193A368DB07E8D5EBE700BFA6
:10A3100024040020000001580E4B0F491B6818222E
:10A32000534382B01B0D6422534301934B69019A3E
:10A33000C3F3800322B902238360012002B0704777
:10A34000019A013A01924A69920701D5002BEDD199
:10A350000020F3E7240400200004005807B5037927
:10A36000012B0FD10A4B1B68182253431B0C01937E
:10A37000FFF7F0FE019B013B0193019B002BF9D1FC
:10A38000FFF7DEFE03B05DF804EBFFF7C5BF00BFCB
:10A3900024040020F8B51E468379012B1546044697
:10A3A0000F46DAB22DD14379012B2AD00223427114
:10A3B0008371FFF7D3FF0D212046FFF7CBFEFFF798
:10A3C00041FF390A2046FFF73DFFF9B22046FFF76B
:10A3D00039FF2E44B5420ED12046FFF7B1FEFFF7FC
:10A3E0009BFFA06801230038A3714FF0000318BF42
:10A3F00001206371F8BD15F8011B2046FFF722FF0D
:10A40000E8E70220F6E7F8B51E468379012B1546EA
:10A4100004460F46DAB22FD14379012B2CD042717A
:10A42000FFF79CFF1D212046FFF794FEFFF70AFF70
:10A43000390A2046FFF706FFF9B22046FFF702FF70
:10A4400000212046FFF7FEFE2E44B5420ED12046E5
:10A45000FFF776FEFFF760FFA06801230038A371C5
:10A460004FF0000318BF01206371F8BD2946204654
:10A47000FFF71CFF0135E8E70220F6E7F8B51F46B5
:10A480008379012B154604460E46DAB22CD1437966
:10A49000012B29D04271FFF761FF06F0EF03A3F112
:10A4A000840253425341237131462046FFF752FE46
:10A4B000FFF7C8FE2F44AF4210D1FFF741FE842EB4
:10A4C00002D02046FFF728FFA06801230038A371BF
:10A4D0004FF0000318BF01206371F8BD15F8011B90
:10A4E0002046FFF7AFFEE6E70220F6E7F8B51E4686
:10A4F0008379012B154604460F46DAB227D14379FA
:10A50000012B24D04271FFF729FF39462046FFF77F
:10A5100021FEFFF797FE00212046FFF793FE2E4411
:10A52000B5420ED12046FFF70BFEFFF7F5FEA068FF
:10A5300001230038A3714FF0000318BF012063719D
:10A54000F8BD29462046FFF7B1FE0135E8E70220B5
:10A55000F6E737B50023ADF8043001AA0223122133
:10A560000546FFF7C3FFBDF80440022364BA01AA01
:10A57000A4B219462846FFF781FFE20702D5284614
:10A580000AF094FFA30702D528460AF095FF60075A
:10A5900002D528460AF0BAFF210702D528460AF05C
:10A5A000BBFFE20602D528460AF0BCFFA30602D58F
:10A5B00028460AF0A5FF600602D528460AF082FF69
:10A5C000210606D514F4807118BF012128460AF02F
:10A5D0007FFFA20502D528460AF08AFF630402D550
:10A5E00028460AF0A5FF03B030BDF8B51E468379B2
:10A5F000012B154604460F46DAB227D14379012BC9
:10A6000024D04271FFF7AAFE0E212046FFF7A2FDDB
:10A61000FFF718FE39462046FFF714FE2E44B542D8
:10A620000ED12046FFF78CFDFFF776FEA0680123D0
:10A630000038A3714FF0000318BF01206371F8BD0B
:10A6400015F8011B2046FFF7FDFDE8E70220F6E7BD
:10A65000F8B51E468379012B154604460F46DAB23B
:10A660002BD14379012B28D04271FFF777FE1E21B1
:10A670002046FFF76FFDFFF7E5FD39462046FFF75F
:10A68000E1FD00212046FFF7DDFD2E44B5420ED14D
:10A690002046FFF755FDFFF73FFEA0680123003875
:10A6A000A3714FF0000318BF01206371F8BD294664
:10A6B0002046FFF7FBFD0135E8E70220F6E7000042
:10A6C000036A23F001030362036A70B54468826978
:10A6D0000D6822F4803222F073022A438D6823F041
:10A6E00002032B43124DA84206D0124EB04203D0B3
:10A6F000A6F58066B04214D1CE6823F00803334338
:10A70000A84223F0040306D00B4DA84203D005F560
:10A710008065A84205D124F44075D1E9054634434B
:10A720002C43446082614A684263036270BD00BF8B
:10A73000002C01400048014000440140036A23F41A
:10A7400080730362036A426870B5C4690D6824F4BB
:10A75000803424F073042C438D6823F4007343EA9F
:10A7600005230F4DA8420ED1CD6823F4006343EAC0
:10A77000052323F48063D1E9055622F44052354382
:10A7800042EA051206E0074DA842F4D005F58065BF
:10A79000A842F0D042604A68C461C263036270BDDF
:10A7A000002C014000440140036A23F480530362FB
:10A7B000026A30B54468C3690D6823F0807323F4DE
:10A7C000E64343EA05238D6822F4005242EA05324B
:10A7D0000A4DA84207D005F5C055A84203D005F59B
:10A7E0008065A84204D14D6924F4804444EA85146C
:10A7F0004460C3614B680364026230BD002C0140B9
:10A80000036A23F480330362026A30B54468436DFF
:10A810000D6823F4803323F070032B438D6822F4FA
:10A82000003242EA05420B4DA84207D005F5C0555B
:10A83000A84203D005F58065A84204D14D6924F4EF
:10A84000803444EA0524446043654B6883650262B2
:10A8500030BD00BF002C0140036A23F48013036263
:10A86000026A30B54468436D0D6823F0807323F4A9
:10A87000E04343EA05238D6822F4001242EA0552C0
:10A880000A4DA84207D005F5C055A84203D005F5EA
:10A890008065A84204D14D6924F4802444EA8524CB
:10A8A000446043654B68C365026230BD002C0140C3
:10A8B000704710B5846A626A82420BD10123237704
:10A8C000D2690AB984F83E302046F9F737F80023F8
:10A8D000237710BDA36A834208D102222277DB6965
:10A8E000002BF1D1012384F83F30EDE7E36A834286
:10A8F00008D104222277DB69002BE5D1012384F8FB
:10A900004030E1E7236B8342DED108222277DB6906
:10A91000002BD9D1012384F84130D5E7704710B519
:10A92000846A636A834207D1012323772046FFF7B5
:10A93000F5FF0023237710BDA36A834201D10223D0
:10A94000F3E7E36A834201D10423EEE7236B8342FA
:10A95000ECD10823E9E7704710B5846A636A834243
:10A9600009D10123237784F83E302046FFF7F3FF17
:10A970000023237710BDA36A834205D102232377E6
:10A98000012384F83F30F0E7E36A83424FF001038C
:10A9900004D10422227784F84030E6E7226B824219
:10A9A00003BF0822227784F8413084F83D30DCE789
:10A9B0001A4A0368904210B502D0B0F1804F09D115
:10A9C0004C6823F07003904243EA040309D0B0F1CD
:10A9D000804F06D0124A904203D002F58062904226
:10A9E00003D1CA6823F4407313434A6923F08003F8
:10A9F000134303608B68C3620B688362074B984202
:10AA000007D003F5C053984203D003F58063984202
:10AA100001D10B6903630123436110BD002C014088
:10AA20000044014010B5044650B390F83D3003F0A7
:10AA3000FF021BB980F83C20F9F780F90223206857
:10AA400084F83D30211DFFF7B3FF012384F848301F
:10AA5000002084F83E3084F83F3084F8403084F899
:10AA6000413084F8423084F8433084F8443084F82C
:10AA7000453084F8463084F8473084F83D3010BDC6
:10AA80000120FCE710B5044650B390F83D3003F0C8
:10AA9000FF021BB980F83C20FFF70AFF0223206861
:10AAA00084F83D30211DFFF783FF012384F84830EF
:10AAB000002084F83E3084F83F3084F8403084F839
:10AAC000413084F8423084F8433084F8443084F8CC
:10AAD000453084F8463084F8473084F83D3010BD66
:10AAE0000120FCE7036A23F010030362036A426853
:10AAF00070B584690D6824F0807424F4E64444EA57
:10AB000005248D6823F0200343EA05130F4DA84266
:10AB10000ED1CD6823F0800343EA051323F04003F0
:10AB2000D1E9055622F44062354342EA850206E047
:10AB3000074DA842F4D005F58065A842F0D04260E8
:10AB40004A6884618263036270BD00BF002C0140CB
:10AB50000044014038B590F83C30012B044673D0D6
:10AB600001200C2A84F83C004ED008D8042A2BD0AF
:10AB7000082A39D0BAB1002384F83C3038BD102AF5
:10AB800052D0142AF7D12068FFF766FE436D0A6998
:10AB900043F400634365436D23F480634365436D71
:10ABA00043EA02234EE02068FFF78AFD83690A69C1
:10ABB00043F008038361836923F00403836183699D
:10ABC000134383610020D6E72068FFF78BFF83697A
:10ABD0000A6943F400638361836923F480638361BA
:10ABE000836943EA0223ECE72068FFF7A7FDC36906
:10ABF0000A6943F00803C361C36923F00403C36116
:10AC0000C3691343C361DDE72068FFF7CDFDC36966
:10AC10000A6943F40063C361C36923F48063C361B9
:10AC2000C36943EA0223EDE72068FFF7E9FD436DBE
:10AC30000A6943F008034365436D23F00403436549
:10AC4000436D13434365BDE7022097E710B5846861
:10AC50000A4324F47F4442EA03222243826010BD67
:10AC600038B590F83C30012B04464FF0020000F05C
:10AC7000958084F83D000122206884F83C20856896
:10AC8000474B2B4083600B68602B54D037D8402B48
:10AC90006BD019D8202B0DD00AD833F0100109D071
:10ACA000012384F83D30002384F83C30104638BD41
:10ACB000302BF5D1826822F4401222F070021A4340
:10ACC00042F0070282602BE0502BE9D14A68CD6840
:10ACD000016A036A23F001030362836921F00A0118
:10ACE00023F0F00343EA05130A4383610262836899
:10ACF00023F4401323F0700343F057030FE0B3F540
:10AD0000805F0DD0B3F5005F0CD0702BC8D1CB683D
:10AD1000D1E90121FFF79AFF836843F0770383604D
:10AD20000022BDE7CB68D1E90121FFF78FFF8368DF
:10AD300043F48043F3E7036A4D68C96823F01003C6
:10AD400003628269036A22F4704223F0A00343EA9B
:10AD5000051342EA013282610362836823F44013DF
:10AD600023F0700343F06703D9E74A68CD68016AAE
:10AD7000036A23F001030362836921F00A0123F0CF
:10AD8000F00343EA05130A4383610262836823F4F4
:10AD9000401323F0700343F04703C0E7024685E702
:10ADA0008800CEFF036A01F01F0110B501248C401A
:10ADB00023EA04030362036A8A401A43026210BD55
:10ADC00038B50D46082D044611461BD005D85DB197
:10ADD000042D14D094F8430008E00C2D15D0102D4C
:10ADE000F8D190F8420001E090F83E00A0F1020C8A
:10ADF000DCF1000040EB0C0050B1022076E090F84E
:10AE00003F00F3E790F84000F0E790F84100EDE7ED
:10AE1000082D1AD007D86DB1042D13D094F8432013
:10AE2000012A19D00CE00C2D27D0102DF6D194F862
:10AE300042000CE094F83E20501E424242415AB972
:10AE4000012053E094F83F20F6E794F84000421EBA
:10AE5000504250410028F3D00029F1D0002BEFD010
:10AE6000082D4FF0020256D00AD885B1042D3ED0ED
:10AE7000042D84F84320E3D13BE094F84100E6E759
:10AE80000C2D5CD0102DF3D184F84220D8E7606AF5
:10AE900084F83E203A4AC2623A4A02633A4A42631E
:10AEA00022683432FDF7C0F90028C9D12268D3687E
:10AEB00043F400732068D36029460122FFF772FF34
:10AEC000324A904250D0324B98424DD003F58063C5
:10AED000984249D0B0F1804F4DD182682D4B13403C
:10AEE000062B02D0B3F5803F45D1002038BD84F851
:10AEF0003F20A06A224AC262224A0263224A426377
:10AF000022683832FDF790F9002899D12268D36879
:10AF100043F48063CEE7E06A84F84020184AC262B6
:10AF2000184A0263184A426322683C32FDF77CF9F2
:10AF3000002885D12268D36843F40063BAE7206B08
:10AF400084F841200E4AC2620E4A02630E4A4263EE
:10AF500022684032FDF768F900287FF471AF22685B
:10AF6000D36843F48053A5E7436C904243F4004315
:10AF70004364B2D0AEE7036843F001030360B4E773
:10AF8000B3A800081FA9000859A90008002C014017
:10AF90000044014007000100FFF712BF082938B53F
:10AFA00004460D464FD004D861B1042944D0012095
:10AFB00038BD0C29FBD10268006BD36823F48053A1
:10AFC000D36005E00268406AD36823F40073D3605D
:10AFD000FDF7A3F9206800222946FFF7E3FE2A4B7C
:10AFE000984207D003F5C053984203D003F580631D
:10AFF00098420DD1026A41F211131A4208D1026A35
:10B0000040F244431A4202BF436C23F400434364BA
:10B01000026A41F211131A4208D1026A40F2444313
:10B020001A4202BF036823F00103036001238DB9B4
:10B0300084F83E300020BBE70268806AD36823F4BE
:10B040008063D360C4E70268C06AD36823F40063F6
:10B05000D360BDE70C2D13D007D8042D0AD0082DDE
:10B060000BD0012384F84330E4E7102DF9D184F8A4
:10B070004230DFE784F83F30DCE784F84030D9E73E
:10B0800084F84130D6E700BF002C0140FFF786BFAF
:10B0900070B590F83C30012B02464FF0020020D0F2
:10B0A00082F83D000F4D106843688468A84202BFD3
:10B0B0004E6823F4700333430E6823F07003334368
:10B0C000A842436002D0B0F1804F04D1896824F0D7
:10B0D00080030B4383600123002082F83D3082F817
:10B0E0003C0070BD002C014010B590F83C30012BA5
:10B0F00002463BD0CB6888681D4C23F44073034361
:10B10000486823F480630343086823F4006303431F
:10B11000086923F480530343486923F4005303432D
:10B12000086B23F480430343886923F4702343EAC4
:10B1300000431068A04214D1CC6923F0805323430C
:10B140008C6A23F4700343EA04530C6A23F080737F
:10B1500023434C6AC96A23F00073234323F000534E
:10B160000B434364002082F83C0010BD0220FCE742
:10B17000002C0140026852E8003F23F0C00342E87F
:10B18000003102680029F5D102F1080353E8003FBD
:10B1900023F4000302F1080C4CE800310029F3D13C
:10B1A0002023C0F88830704710B5026852E8003F8D
:10B1B00023F4907342E8003102680029F5D10F4C66
:10B1C00002F1080353E8003F234002F1080C4CE869
:10B1D00000310029F4D1C36E012B07D152E8003FA2
:10B1E00023F0100342E800310029F7D12023C0F8F2
:10B1F0008C300023C366436710BD00BFFEFFFFEF26
:10B20000F8B504461346D4F88850202D32D1F1B158
:10B21000EAB1E06FA4F85620A4F8542000262122B9
:10B22000C4F890602165C4F88820226888B1124F64
:10B23000C762124F0763124F2832C0E90D76FCF740
:10B24000F3FF30B11023C4F89030C4F888500120C7
:10B25000F8BD236840221A62226802F1080353E80D
:10B26000003F43F0800302F1080141E8003000286C
:10B27000F3D1EDE70220EBE785B20008CDB200087C
:10B28000D9B2000808B50346806A1B681B6813F032
:10B29000200317D1A0F85630026802F1080353E8E2
:10B2A000003F23F08003083242E8003102680029A1
:10B2B000F2D152E8003F43F0400342E80031002958
:10B2C000F7D108BDF9F72CF8FBE7704708B5806A9D
:10B2D000FFF7FBFF08BD7047806A38B50468D0F8F7
:10B2E0008830D0F88C50A268120606D5212B04D1E4
:10B2F0000023A0F85630FFF73DFFA3685B0606D594
:10B30000222D04D10023A0F85E30FFF74DFFD0F8C6
:10B31000903043F01003C0F89030FFF7DCFF38BDE9
:10B3200008B5806A0023A0F85E30A0F85630FFF719
:10B33000D2FF08BD704700000368D9691A682DE97B
:10B34000F04140F60F0631429D68044610D18E064A
:10B3500040F1978002F0200605F080573E4300F050
:10B360009080436F002B00F08580BDE8F0411847C6
:10B37000AB4EAC482E401040304300F08280CF07E7
:10B3800009D5D00507D501201862D4F8900040F007
:10B390000100C4F890008F0709D5E80707D50220FF
:10B3A0001862D4F8900040F00400C4F890004F07F1
:10B3B00009D5E80707D504201862D4F8900040F0BA
:10B3C0000200C4F890000F070BD502F020003043B4
:10B3D00007D008201862D4F8900040F00800C4F8A4
:10B3E00090000E050AD5500108D54FF40060186290
:10B3F000D4F8903043F02003C4F89030D4F8903063
:10B40000002B37D08B0609D502F0200205F08055BD
:10B410002A4303D0636F0BB1204698472668D4F8BF
:10B420009020B36802F0280203F0400353EA0205BB
:10B43000204621D0FFF7B8FEB3685F0617D5226813
:10B4400002F1080353E8003F23F04003083242E8CA
:10B4500000310029F3D1D4F8800040B1724B8363EE
:10B46000FCF75BFF30B1D4F88000836B7DE72046AA
:10B47000FFF731FFBDE8F081FFF72DFFC4F89050D2
:10B48000F8E7E06E012840F08980CE0640F1868022
:10B49000D00640F1838010221A629A6851064BD57B
:10B4A000D4F8802011684A6892B2002AE2D0B4F839
:10B4B0005C009042DED9A4F85E200A6892062FD480
:10B4C00053E8002F22F4807243E800210029F7D1CD
:10B4D00003F1080252E8002F22F0010203F10800F4
:10B4E00040E800210029F3D103F1080252E8002FBF
:10B4F00022F0400203F1080040E800210029F3D1C6
:10B500002022C4F88C20E16653E8002F22F01002BC
:10B5100043E800210029F7D1D4F88000FCF7C8FEE9
:10B5200002232367B4F85E30B4F85C10C91A89B2FC
:10B530002046FFF7FFFE9DE7B4F85E20B4F85E00FA
:10B54000B4F85C1080B292B2002893D0891A89B204
:10B5500000298FD053E8002F22F4907243E8002096
:10B560000028F7D1314D03F1080252E8002F2A409C
:10B5700003F1080646E800200028F4D12022C4F890
:10B580008C206067E06653E8002F22F0100243E849
:10B5900000200028F7D102232367C9E7CF0209D58D
:10B5A0006E0207D54FF4801220461A62BDE8F041C2
:10B5B00000F0A0BD08060BD502F0800005F40005E0
:10B5C000284305D0A36F002B3FF454AF2046CCE6B0
:10B5D0004F0611D556060FD553E8002F22F0400232
:10B5E00043E800210029F7D12023C4F88830A1675F
:10B5F0002046F8F795FE3DE70D0206D5500004D52C
:10B600002046BDE8F04100F077BDCB017FF532AFB9
:10B61000002ABFF62FAF2046BDE8F04100F06BBD19
:10B62000010000102001000421B30008FEFFFFEF1D
:10B63000D0F88C20B0F86010222A08B5036855D1E4
:10B640005B6A826D0B401370836D01338365B0F8C4
:10B650005E30013B9BB2A0F85E30B0F85E309BB22A
:10B66000002B42D1026852E8003F23F4907342E875
:10B67000003103680029F5D103F1080252E8002FD8
:10B6800022F0010203F1080C4CE800210029F3D15B
:10B690002022C0F88C20184A41679342016705D1E7
:10B6A000C26E012A0ED0F8F749FE1EE05A68110258
:10B6B000F6D553E8002F22F0806243E800210029EC
:10B6C000F7D1EDE70022C26653E8002F22F0100206
:10B6D00043E800210029F7D1DA69B0F85C10D206FE
:10B6E00044BF10221A62FFF725FE08BD9A6942F096
:10B6F00008029A61F9E700BF00800040D0F88C2072
:10B70000B0F86010222A08B5036852D15A6A114075
:10B71000826D22F8021B8265B0F85E20013A92B277
:10B72000A0F85E20B0F85E2092B2002A40D153E823
:10B73000002F22F4907243E800210029F7D103F191
:10B74000080252E8002F22F0010203F1080C4CE835
:10B7500000210029F3D12022C0F88C20174A41672C
:10B760009342016705D1C26E012A0ED0F8F7E6FDBB
:10B770001EE05A681102F6D553E8002F22F08062CD
:10B7800043E800210029F7D1EDE70022C26653E823
:10B79000002F22F0100243E800210029F7D1DA69D6
:10B7A000B0F85C10D20644BF10221A62FFF7C2FD47
:10B7B00008BD9A6942F008029A61F9E700800040EA
:10B7C0002DE9F84F0368B0F86060D3F81CB01F682B
:10B7D0009D68D0F88C20222A044640F0B980B0F849
:10B7E000683043B1DFF87491DFF874A14FF00008BE
:10B7F0001BF0200F20D1B4F85E309BB2D3B1B4F867
:10B8000068209A4216D9226802F1080353E8003FE3
:10B8100023F08053083242E8003122680029F2D137
:10B82000504B636752E8003F43F0200342E8003189
:10B830000029F7D1BDE8F88F2368A26D5B6A334019
:10B840001370A36D0133A365B4F85E30013B9BB266
:10B85000A4F85E302368D3F81CB01BF0070F2ED07D
:10B860001BF0010F09D0F90507D501221A62D4F89F
:10B87000902042F00102C4F890201BF0020F09D082
:10B88000EA0707D502221A62D4F8902042F0040297
:10B89000C4F890201BF0040F09D0E80707D5042254
:10B8A0001A62D4F8903043F00203C4F89030D4F810
:10B8B000903023B12046FFF70EFDC4F89080B4F815
:10B8C0005E309BB2002B93D1226852E8003F23F4F4
:10B8D000807342E8003123680029F5D103F10802A2
:10B8E00052E8002F02EA090203F1080040E80021B3
:10B8F0000029F3D120225345C4F88C2061672167C9
:10B900000AD05A68110207D553E8002F22F080624E
:10B9100043E800210029F7D1E26E012A14D1002268
:10B92000E26653E8002F22F0100243E800210029CC
:10B93000F7D1DA69B4F85C10D20644BF10221A625B
:10B940002046FFF7F7FC53E72046F8F7F7FC4FE7F0
:10B950009A6942F008029A616CE700BFFEFFFFEFB0
:10B960000080004031B600082DE9F84F0368B0F8B8
:10B970006060D3F81CB01F689D68D0F88C20222A24
:10B98000044640F0B780B0F8683043B1DFF87091FA
:10B99000DFF870A14FF000081BF0200F20D1B4F8A1
:10B9A0005E309BB2D3B1B4F868209A4216D92268AF
:10B9B00002F1080353E8003F23F08053083242E8C5
:10B9C000003122680029F2D14F4B636752E8003FF3
:10B9D00043F0200342E800310029F7D1BDE8F88F99
:10B9E0002368A26D596A314022F8021BA265B4F89F
:10B9F0005E20013A92B2A4F85E20D3F81CB01BF08E
:10BA0000070F2ED01BF0010F09D0F90507D5012231
:10BA10001A62D4F8902042F00102C4F890201BF082
:10BA2000020F09D0EA0707D502221A62D4F8902043
:10BA300042F00402C4F890201BF0040F09D0E8077C
:10BA400007D504221A62D4F8903043F00203C4F8F8
:10BA50009030D4F8903023B12046FFF73CFCC4F876
:10BA60009080B4F85E309BB2002B95D1226852E8EA
:10BA7000003F23F4807342E8003123680029F5D1A8
:10BA800003F1080252E8002F02EA090203F108005C
:10BA900040E800210029F3D120225345C4F88C202E
:10BAA000616721670AD05A68110207D553E8002F51
:10BAB00022F0806243E800210029F7D1E26E012ADA
:10BAC00014D10022E26653E8002F22F0100243E86E
:10BAD00000210029F7D1DA69B4F85C10D20644BF1E
:10BAE00010221A622046FFF725FC55E72046F8F79A
:10BAF00025FC51E79A6942F008029A616EE700BF9F
:10BB0000FEFFFFEF00800040FDB6000838B5044698
:10BB100003682169A2681D68C0690A4361690A4314
:10BB20007749024329400A431A605A68E16822F4BF
:10BB300040520A435A60734AA16993421CBF226A69
:10BB400011439A6822F06E4222F430620A439A60EE
:10BB5000DA6A616A22F00F020A43DA626A4A9342A1
:10BB600019D14FF0B043694AD3F8883003F003038A
:10BB700043F44033934200F0B480B3F1031F24D068
:10BB8000013A934240F0B580B0F5004F40F08F800D
:10BB9000FCF780FF6EE05E4A93421CD14FF0B04349
:10BBA0005C49D3F8883003F00C0343F440228A4206
:10BBB00000F0978006D8002B7CD0574B9A42E3D0F8
:10BBC000012026E0B2F10C1FFAD1B0F5004F53D09E
:10BBD0004FF4004075E04B4A9342F1D14FF0B0432F
:10BBE000D3F8883003F44063B3F5006F18D006D85B
:10BBF0005BB1B3F5806FE3D1FCF74CFF07E0B3F521
:10BC0000406FDDD14FF400400BE0FDF73BFB40B946
:10BC100000204FF00113A3660023C4E91D3338BD93
:10BC20003E4865683E4B626A05EB450133F81220D9
:10BC3000B0FBF2F39942C3D8B3EB053FC0D8002361
:10BC40001946F6F731FC090241EA10616B0800025F
:10BC5000C0182A464FF0000341F10001F6F724FC1A
:10BC6000304BA0F540729A42AAD82368D860CFE73B
:10BC7000FDF708FB0028CBD06168294B626A33F8D6
:10BC80001220B0FBF2F24B0803EB42034FF6EF72C7
:10BC9000B3FBF1F3A3F11001914291D823F00F020D
:10BCA000216892B2C3F342031343CB60B0E7FCF7C1
:10BCB000F1FE04E0B0F5004FDAD0FDF7E3FA00281A
:10BCC000A6D06368616A164A32F81120B0FBF2F020
:10BCD00000EB5300B0FBF3F04FF6EF73A0F110024E
:10BCE000C1E7B0F5004F0D48EBD1C5E7FDF7DAFA33
:10BCF000C0E7B0F5004FF9D0FDF7D4FADFE700BF99
:10BD0000F369FFCF008000400038014002000300CB
:10BD10000044004008000C0004000C000024F40063
:10BD200034800308FFFC0F00836ADA0710B506D5DC
:10BD30000168C46A4A6822F4003222434A609C07C0
:10BD400006D50168046B4A6822F4803222434A60B7
:10BD5000590706D50168446B4A6822F480222243C1
:10BD60004A601A0706D50168846B4A6822F40042CB
:10BD700022434A60DC0606D50168C46B8A6822F457
:10BD8000805222438A60990606D50168046C8A684D
:10BD900022F4005222438A605A060FD50168446C8F
:10BDA0004A6822F480122243B4F5801F4A6005D10C
:10BDB0004A68846C22F4C00222434A601B0606D5FE
:10BDC0000268C16C536823F400230B43536010BD19
:10BDD0002DE9F843DDF8209005460F4616469846B3
:10BDE0002A68D36937EA03030CBF01230023B34257
:10BDF00001D0002029E0B9F1FF3FF2D0F7F7C6FEED
:10BE0000A0EB080048452C6802D8B9F1000F1ED1FC
:10BE100054E8003F23F4D07344E80032002AF7D1FD
:10BE200004F1080353E8003F23F0010304F1080183
:10BE300041E80032002AF3D12023C5F88830C5F844
:10BE40008C30002385F884300320BDE8F883236814
:10BE50005A07C5D5E3691B05C2D54FF400632362B9
:10BE600054E8003F23F4D07344E80032002AF7D1AD
:10BE700004F1080353E8003F23F0010304F1080133
:10BE800041E80032002AF3D12023C5F88830C5F8F4
:10BE90008C30C5F89030D4E773B504460026C0F85E
:10BEA0009060F7F773FE23681B681A07054619D4DC
:10BEB00023681B685B070AD56FF07E43009300225E
:10BEC0002B464FF480012046FFF782FFB0B90020D7
:10BED0002023C4F8883084F88400C4F88C30E066ED
:10BEE00020670CE06FF07E430093324603464FF428
:10BEF00000112046FFF76CFF0028D9D0032002B0C4
:10BF000070BD10B5044650B3D0F888301BB980F826
:10BF10008430F8F713F922682423C4F888301368B2
:10BF200023F0010313602046FFF7F0FD012816D02F
:10BF3000A36A13B12046FFF7F7FE23685A6822F47C
:10BF400090425A609A6822F02A029A601A6842F077
:10BF5000010220461A60BDE81040FFF79DBF012096
:10BF600010BD000030B581658168A0F85C20002319
:10BF7000B1F5805FA0F85E20436735D10369002BDF
:10BF800040F2FF1318BFFF23A0F860300023C0F871
:10BF900090302223C0F88C30016801F1080353E887
:10BFA000003F43F00103083141E800340368002CEE
:10BFB000F2D1456E84680169B5F1005F32D1B0F805
:10BFC000685095422ED8B4F5805F244A03D1244CA2
:10BFD000002908BF22464267B1B153E8002F42F45E
:10BFE000807243E80021F7E729B90369002B14BFE9
:10BFF0007F23FF23C8E7B1F1805FC5D10369002B20
:10C0000014BF3F237F23BFE703F1080252E8002F4C
:10C0100042F0805203F1080040E800210029F3D1EA
:10C02000002030BDB4F5805F0E4A03D10E4C0029CC
:10C0300008BF2246426741B153E8002F42F4907294
:10C0400043E800210029F7D1EAE753E8002F42F046
:10C05000200243E800210029F7D1E1E7C1B7000839
:10C0600069B9000831B60008FDB60008D0F88C3078
:10C07000202B30B415D1B9B1B2B100230468C36626
:10C080000A4B9C420AD063681B0207D554E8003F64
:10C0900043F0806344E80035002DF7D130BCFFF752
:10C0A00061BF022030BC70470120FBE700800040E8
:10C0B000436E30B52BB90123A0F86A30A0F8683080
:10C0C00030BD0368094D9A689968094C490FC2F35D
:10C0D00042626B5C615CDB00B3FBF1F3A0F86A3099
:10C0E000AB5CA25CDB00B3FBF2F3E7E75480030830
:10C0F0004C8003087047704770471FB504AB03E9D5
:10C10000060090F88430012B04463AD0012380F8D1
:10C1100084302423C0F8883003681A6822F00102B2
:10C120001A609A6822F440120A439A6071B95A68F8
:10C13000BDF80C009DF80E1022F0100202435A6068
:10C140005A6822F07F4242EA01625A601A6842F05D
:10C1500001021A60F7F71AFD6FF07E420346009263
:10C160004FF4800100222046FFF732FE38B9202329
:10C17000C4F88830002384F8843004B010BD032054
:10C18000F8E70220F9E790F88430012B0FD0012363
:10C1900080F88430016851E8002F42F0020241E843
:10C1A0000023002BF6D180F8843018467047022017
:10C1B000704710B590F88430012B044617D0242323
:10C1C000C0F8883003681A68196821F00101196005
:10C1D00042F000524FF0005141661A60FFF768FFCD
:10C1E0002023C0F88830002084F8840010BD02208D
:10C1F000FCE770B590F88430012B044617D0056831
:10C200002423C0F888302E682B6823F001032B60AC
:10C21000AB6823F060431943A960FFF749FF20236F
:10C220002E60C0F88830002084F8840070BD0220A1
:10C23000FCE770B590F88430012B044617D00568F0
:10C240002423C0F888302E682B6823F001032B606C
:10C25000AB6823F060631943A960FFF729FF20232F
:10C260002E60C0F88830002084F8840070BD022061
:10C27000FCE7000038B5084D052455F8043B2BB900
:10C28000013C14F0FF04F8D1204638BDDB68984724
:10C290000028F5D0F9E700BFD0230020034BD87069
:10C2A000034B1B681B6C03B118477047B823002071
:10C2B000B4230020034B1874034B1B685B6C03B161
:10C2C00018477047B8230020B4230020F0B5314D43
:10C2D000314B95F90420314E91B00C46012795F968
:10C2E00005108DF8047002288DF809208DF80A10C9
:10C2F00010D18DF80800D8711C7203F075FB3378EB
:10C3000003B114B101A804F0A5F8254B059A1A60F1
:10C3100011B0F0BD59714FF480711A71D9801C723F
:10C3200033788DF8087053BB1F2306A88DF81C20A6
:10C330008DF8183003F036FD20238DF8183006A84C
:10C340002B798DF81C3003F02DFD22238DF8183049
:10C3500006A86B798DF81C3003F024FD21238DF89D
:10C36000183006A86B798DF81C3003F01BFD2923CB
:10C370008DF8183006A80B4B079303F013FD03F05C
:10C3800033FB012306A88DF818308DF81C3003F01C
:10C3900009FDB4E7B82300205C04002094220020AB
:10C3A00088230020000400017FB5092301A88DF82F
:10C3B000043004F04FF80038044B059A1A6018BF97
:10C3C0000120404207B05DF804FB00BF8823002035
:10C3D00070B504460B46144962784A700020A27872
:10C3E0000A7208701A884A729A788A72DB780B741B
:10C3F0006368CB600D4B1B68DA6A2AB1237803F0BF
:10C40000FB030A2B00D09047094E002556F8043B49
:10C410001BB15B6A0BB1204698470135EBB2052B87
:10C420006DB2F3D170BD00BF2C040020B4230020F6
:10C43000D023002070B504461148012303706378AF
:10C440004370A3788372E368C360E378037623695B
:10C450004376237943720B4B1B689B6A03B1984761
:10C46000094E002556F8043B1BB19B690BB12046D1
:10C4700098470135EBB2052B6DB2F3D170BD00BF0B
:10C4800040040020B4230020D0230020014B186872
:10C49000704700BF8823002000B58BB00123684699
:10C4A0008DF8003003F058FB38B99DF804000038CF
:10C4B00018BF01200BB05DF804FB0020FAE7000074
:10C4C00008B502F049FC40B9FFF7E6FF012806D0A5
:10C4D000054B197AD879FFF7F9FE012008BDBDE8B0
:10C4E0000840FFF7C7BE00BF5C0400202DE9F04103
:10C4F00086B005460E46174602F02EFC002873D182
:10C5000002F042FC044640B9FFF7C6FF01280AD0FA
:10C510003D4B197AD879FFF7D9FE6FF00204204617
:10C5200006B0BDE8F081DFF8E48088F80860003EDE
:10C5300018BF01268DF80460354E687833798DF880
:10C540001230694603F0A6FA00283FD08DF8044067
:10C550000394ADF810406FF0060495E803002D4BEE
:10C5600083E80300337988F80A30394601A804F0DB
:10C5700075F8294B059A1A6011283FD801A353F882
:10C5800020F000BFEFC50008E9C50008FDC50008A0
:10C59000FDC50008FDC50008FDC50008FDC5000873
:10C5A0001BC50008FDC50008FDC50008FDC5000845
:10C5B000E3C50008FDC50008FDC50008E9C5000881
:10C5C000E9C50008E9C5000803C600082B788DF806
:10C5D00008306B78ADF810306B6803934FF0FF3480
:10C5E000BBE76FF005049AE76FF0010497E70B4B88
:10C5F00000221A70E31D18BF144690E74FF0FF3475
:10C600008DE76FF004048AE75C04002040040020FA
:10C61000B823002050040020882300208723002016
:10C6200037B502F0BBFB134D052455F8043B4BB165
:10C630001A693AB19B682BB1984718B155F8043C78
:10C640001B699847013C14F0FF04EED1FFF712FE7E
:10C6500068B9094D2B7853B1084BADF80040D97833
:10C66000019422466846FFF741FF00B92C7003B0E1
:10C6700030BD00BFD023002087230020B823002036
:10C6800030B58BB0044602F067FB0546002835D173
:10C69000FFF702FF012834D168468DF8005003F0FF
:10C6A0005BFA40BB9DF80430A34204D0012C22D099
:10C6B000022C12D014B100200BB030BD002BFAD0E8
:10C6C00068468DF8044003F06DFBA0B90E4B1B6863
:10C6D0001B6B002BEFD09847EDE763B968468DF8E8
:10C6E000044003F05FFB30B9074B1B681B6B002B4A
:10C6F000E1D02046EFE74FF0FF30DDE76FF00100BB
:10C70000DAE76FF00200D7E7B423002010B5044643
:10C710008AB018B94FF0FF300AB010BD0023684648
:10C720008DF8003003F018FA0028F3D19DF804309A
:10C730002370F1E77FB500220B4620498DF80720D2
:10C7400001220A7042784A700446002A33D10279E5
:10C750000A721A884A729A788A72DB780B740369B3
:10C76000CB60C378164D8DF80830037B8DF8093007
:10C77000836803932B68DB6A0BB102A898472B6888
:10C780009B6B13B1227E02B198470E4E052556F8D9
:10C79000043B1BB1DB690BB120469847013D15F006
:10C7A000FF05F4D10DF10700FFF7B0FF637913B176
:10C7B000054B01221A7004B070BD00BF2C0400208C
:10C7C000B4230020D02300208723002010B5044686
:10C7D0008AB018B94FF0FF300AB010BD2023684668
:10C7E0008DF8003003F0B8F90028F3D1024A9DF922
:10C7F000043023701371EFE7B823002000B58BB02D
:10C800002323019068468DF8003003F0CBFA0038FE
:10C8100018BF012040420BB05DF804FB70B5654CB9
:10C8200001468EB01822204606F0BCFF624B002263
:10C830001A70FAF77FFE23784068012202FA03F1AA
:10C84000014004D15D4B084608F098FFFEE75C49C3
:10C850005C481A4602F00AFF18B14FF0FF300EB0E4
:10C8600070BD272304A88DF8103003F09BFA564EB4
:10C87000564D002870D1012333702B68DB690BB152
:10C8800000209847272304A88DF8103003F064F99E
:10C89000059B93F84820227093F8182193F81A31D9
:10C8A0006270A370464BD3E9020106F06BFE0546A9
:10C8B0000028D2D1464E062304A88DF8103003F08C
:10C8C0004BF9059B736104A803F06CFA022304A8DA
:10C8D0008DF81030059603F03FF90836032304A8BD
:10C8E0008DF81030059603F037F90F2606F010FF8B
:10C8F000012304A88DF814308DF8106003F052FA6B
:10C9000010230DEB03008DF810308DF8145003F058
:10C9100049FA04238DF8103004A8A3788DF8143058
:10C9200003F040FA3A238DF8103004A863690593A8
:10C9300003F038FA02A920788DF8086004F0CCFFE3
:10C94000003818BF0120E0711420FFF757FFE0798D
:10C9500004F046F8284682E728238DF810302B682B
:10C960001B6943B104A803F0F7F82B6805981B690D
:10C9700040F2C4519847272304A88DF8103003F0E3
:10C9800011FA50B9012304A88DF8103003F0E4F82F
:10C990009DF81430002B7FF46EAF3378002B7FF4BA
:10C9A0006CAF052204A88DF81020059303F0FAF966
:10C9B00078E700BFB8230020872300205C800308AD
:10C9C0008C230020A423002094220020B4230020E4
:10C9D000F423002037B500230D4601930446D0B957
:10C9E00000F07CFD0190019BD3B10F4A42F8243046
:10C9F0000E4A9A620E4A1268916B1963916C5963E0
:10CA000092690C49D9625A6128465B680A49F22248
:10CA10009847002006E001A900F076FD0028E2D04A
:10CA20004FF0FF3003B030BDD0230020CDC200084E
:10CA3000B4230020A9C3000895220020194B07B594
:10CA40001860194B194A1A60194A5A60194A9A60B3
:10CA5000194ADA60194B02681A6042685A608268A3
:10CA60009A60C268DA60164A1A6182695A61154B87
:10CA7000C26B5A60144A019119609A601946134AB0
:10CA8000DA600020FFF7A6FF48B901A800F02AFDF0
:10CA9000003818BF0120404203B05DF804FB4FF09E
:10CAA000FF30F9E7B4230020A423002035C4000898
:10CAB00035C7000875CB0008D1C300088C230020BF
:10CAC00089180108E42300209DC20008B5C20008AF
:10CAD00049B118B1012804D000207047034B0B6006
:10CAE000FAE7034BFBE74FF0FF307047000400010B
:10CAF0000100010208B503F08FFF002814BF6FF09A
:10CB00000100002008BD08B502F096FF002814BF00
:10CB10006FF00100002008BD20B1044BDB790370E9
:10CB2000002070474FF0FF30704700BFB82300204F
:10CB300008B5034BD87103F053FF002008BD00BFB8
:10CB4000B823002010B504468AB018B94FF0FF3062
:10CB50000AB010BD212368468DF8003002F0FCFFBA
:10CB60000028F3D1024A9DF9043023705371EFE796
:10CB7000B82300202DE9F0412F4D304F00232B70BA
:10CB800043786B703B689B6A8AB004460BB12846B9
:10CB90009847DFF8AC80002658F8043B1BB11B6AAD
:10CBA0000BB1204698470136F3B2052B76B2F3D18C
:10CBB0002378052B2FD00B2B35D0012B25D1214CE1
:10CBC000062368468DF8003002F0C6FF0199E0792F
:10CBD00006F01EFD10B91C4B019A5A611B48FFF765
:10CBE000F5FD1B48FFF7AEFF6B788BB9A371194BAE
:10CBF0005878FFF745FD3B685B6A0BB111489847D1
:10CC00006B7813B9E07906F095FD0AB0BDE8F081C4
:10CC1000FF23A371EFE7104B01225A74227A9A7412
:10CC2000627ADA74F1E76378002BEED00AB0BDE8DF
:10CC3000F041FFF7B9BB00BF40040020B42300203F
:10CC4000D02300205C040020F42300206004002096
:10CC500061040020B82300202C04002030B58BB0E4
:10CC6000FFF751FF0446F0B904F016FE831C1DD0F7
:10CC7000F8B9134D2B685B69DBB1272368468DF843
:10CC8000003002F069FF2B6801985B694FF4B961CD
:10CC9000984704F013FE78B92CB9094B1B68DB697F
:10CCA0000BB10120984720460BB030BD6FF0070450
:10CCB000EFE74FF0FF34ECE74FF0FF34F3E700BF4E
:10CCC000B4230020014B1878704700BF24240020B3
:10CCD000014B5878704700BF24240020064B0748BA
:10CCE00010B501225A7309F085F9054B5B6913B140
:10CCF000BDE81040184710BD242400200C2400205B
:10CD00006804002013B50A4C79B1A27001230022F7
:10CD1000616023700748084B00924FF0FF3109F023
:10CD2000BDF80023637002B010BD2170F9E700BFA9
:10CD3000242400200C240020DDCC00082DE9FF472E
:10CD4000C378CA2B804600F0BE8004B0BDE8F087EF
:10CD5000D8F808305A5D6E1CF6B2032A0FD8DFE807
:10CD600002F0022E6CAB7A6800231355611CA31CE1
:10CD7000DBB2C9B2012050540334D054E4B235467A
:10CD800098F80C30AB42E3D8002CDED0CA238DF8E3
:10CD90000830504B8DF809405B6803930DF1070094
:10CDA000FFF7BAFE0020FFF7C3FE0122002102A810
:10CDB000FFF79CFB9DF80700FFF7BAFEC5E70022CE
:10CDC0007A7398F818204AB96A1DD2B2397A9A5CF7
:10CDD00001F00F0102F00F02914202D0AE1DF6B237
:10CDE000CDE7AA1CD2B29E5D9A5C06EB0226EA1C35
:10CDF000D2B20DF1080A9A5C06EB02462A1DD2B2A5
:10CE000050469B5C06EB036608F022FF029B33440E
:10CE100002939AE8030008F0F3FE3B7AC3F303029F
:10CE2000013262F303033B722B4B1B6B002BD5D0FB
:10CE30000136022ED2D89847D0E7EE1C0235EDB26B
:10CE40001E215B5D002003F00F0380259D4006F04E
:10CE50008DFC7A680223135504EB030A631CDBB2D2
:10CE60000021D154054402A808F0F2FE029B7A6822
:10CE70004B4504F1030188BFA3EB09035FFA8AFA6B
:10CE8000C9B2180A02F80A305054611D201DC9B2F7
:10CE9000C0B24FEA134C1B0E02F800C053544FF4BB
:10CEA0007A7169430D4809F0DFF806340B48F6B291
:10CEB000E4B209F09FF862E79B5D023503F00703D7
:10CEC0007B73EEB25BE70024024FDFF81490254637
:10CED00056E700BF24240020680400200C24002012
:10CEE000803DD51210B5114C637A8AB0E3B10423AA
:10CEF0008DF800306846A37A8DF8043002F052FFB6
:10CF000018238DF800306846E37A8DF8043002F07B
:10CF100049FF20238DF800306846237B8DF80430CC
:10CF200002F040FF002363720AB010BD24240020E9
:10CF3000004870476804002030B58FB0FFF7C0FA92
:10CF4000002861D1324C657A4DBB042304A88DF8CA
:10CF5000103002F001FE9DF81430A37204A88DF881
:10CF6000145002F01FFF182304A88DF8103002F0AF
:10CF7000F3FD9DF81430E37204A801238DF81430FA
:10CF800002F010FF202304A88DF8103002F0E4FD19
:10CF90009DF8143023731F4BDB6A03B1984702A836
:10CFA00008F056FE029A1C4B1C4913448B4288BF62
:10CFB0001B4B616888BF9B181A0A4B708A701A0C49
:10CFC0001B0E0B71237ACA7001256FF304134B718A
:10CFD0000D7023720DF1070040F2CA63ADF81030F6
:10CFE00005916572FFF798FD0020FFF7A1FD2A4625
:10CFF000002104A8FFF77AFA04469DF80700FFF71E
:10D0000097FD20460FB030BD4FF0FF34F9E700BF69
:10D01000242400206804002080C22AED803DD5121F
:10D02000008555DA10B5054C637B2BB1FFF784FF03
:10D0300010B9637B013B637310BD00BF2424002043
:10D04000014B1878704700BF50240020014B5878DE
:10D05000704700BF5024002070470000044B9A7AAC
:10D060000AB101225A70034B5B6903B1184770473C
:10D0700050240020A004002073B5224C6378002BBC
:10D0800033D008F025FF66680546FFF7FFF9064430
:10D09000AE4214D2A37A93B1E0228DF800208DF82D
:10D0A0000130217AE368019301226846FFF71EFAF6
:10D0B00008B1073010D100236370A372656094F843
:10D0C0003430EBB1002384F834300F4B5B6BBBB1D1
:10D0D00002B0BDE87040184740F2DC510B4808F040
:10D0E000C3FF0A4808F086FFE8E794F83520002AD5
:10D0F000E5D094F8360084F83530FFF7C1FADEE762
:10D1000002B070BD50240020A00400203424002070
:10D1100037B5104D104CC8B1C1B162720123002265
:10D120002860E16023700D480D4B00924FF0FF31F5
:10D1300008F0B4FE00250B4825822022294606F07F
:10D1400045FB6570A574A58603B030BD00232B6038
:10D150002370EFE74C2400205024002034240020CA
:10D160005DD00008642400202DE9F0478E4C237820
:10D170008CB0002B56D0C2780AB9837B13B1238AB6
:10D1800001332382437B002B4CD0E02A4AD1002379
:10D19000A372876897F80080B8F1220F27D8B8F1FA
:10D1A000220F30D8DFE818F04100FB0052005A008F
:10D1B00061006E0075008E009D00B400C7002F0056
:10D1C0002F002F002F002F002F002F002F002F00E7
:10D1D0002F002F002F002F002F002F002F002F00D7
:10D1E0002F002F002F002F00C900D000D400B8F16D
:10D1F0007E0F00F0CC80B8F17F0F00F0DF80B8F137
:10D200007D0F00F0AB80A57A002D00F05B81674CAC
:10D21000637A3BB94FF47A71204608F025FF204627
:10D2200008F0E8FE0CB0BDE8F087E36801220021B9
:10D23000A2721970A37AE1689818A0720620C854E7
:10D24000A37AE1689818A072CA54DCE7584B9B6A2D
:10D25000002BD8D0012102209847D4E77B7884F8AE
:10D260003630012384F83530CDE704238DF80430BF
:10D270007B78003B18BF012301A88DF8083002F02D
:10D2800091FDC0E77878003818BF012003F0A8FBB3
:10D29000B9E7484E0FCE01AD0FC50FCE0FC596E8CA
:10D2A000070085E807007B780A2BACD8424A126851
:10D2B0005268002AA7D00CA901EB830353F82C0C69
:10D2C0009047A0E77878431E012B9CD83A4B013851
:10D2D0001B6818BF012020729B68002B93D09847D1
:10D2E00091E7E26801230821A3721170627A057B3D
:10D2F000A17AAA4228BF2A46934284D285685A1C42
:10D30000EB5CE56801334E1CA6726B54D3B2EDE7BB
:10D31000E3680122A27209221A70A37AE268218AC4
:10D32000581CA072D154A27A238AE1681B0A501CAF
:10D33000A0728B5467E7238265E705238DF80430DC
:10D3400001A803F087F85EE7194BDB6A98475AE7B4
:10D35000194B78781B686075DB68BEE7037B072B89
:10D360007FF451AF06238DF80430B7F80130ADF8E3
:10D3700008307B793A791B0443EA0223FA78134395
:10D38000642253430393BB798DF81030D8E73B22D6
:10D3900001A88DF804208DF8083002F003FD012368
:10D3A00084F834302FE700BF5024002034240020BC
:10D3B000A0040020C42B03084C2400202A2301A829
:10D3C0008DF8043002F0C8FB94F80A90E6689DF8E6
:10D3D00008009DF809509DF80A709DF80BC09DF853
:10D3E0000D309DF80E209DF80F109DF80CE009F10E
:10D3F000010A84F80AA006F80980354E94F80A90CC
:10D400003668D4F80C8009F1010A84F80AA096F86D
:10D4100003A008F809A094F80A90D4F80C8009F148
:10D42000010A84F80AA096F802A008F809A094F866
:10D430000A90D4F80C8009F1010A84F80AA096F841
:10D4400001A008F809A094F80A9009F1010A84F8EB
:10D450000AA096F80080E66806F8098094F80A8029
:10D46000E66808F1010984F80A9006F808C094F803
:10D470000AC0E6680CF1010884F80A8006F80C700E
:10D48000A77AE66807F1010C84F80AC0F555A57A79
:10D49000E6686F1CA7727055A07AE568461CA672F4
:10D4A0002954A17AE0684D1CA5724254A27AE16821
:10D4B000501CA0728B54A37AE268591CA17202F826
:10D4C00003E0A0E6034808F047FD6570AAE600BF48
:10D4D0004C2400203424002070470000004870478E
:10D4E000A0040020002108B50120FFF773FA0146CF
:10D4F00038B90220FFF76EFA003818BF0120404209
:10D5000008BD4FF0FF30FBE710B50C4661B10128B4
:10D5100003D0022805D0002010BDFFF709FD2060D0
:10D52000F9E700F01FFCFAE74FF0FF30F4E70000E6
:10D53000014B1878704700BF10050020014B587848
:10D54000704700BF10050020F7B500208DF80700D8
:10D55000EFF3108272B62A4FBB78FD7882F3108801
:10D56000012B08D0022B04D1264B93F82030012B3D
:10D570003CD103B0F0BD234E0DF10700FFF7C6F814
:10D58000382303FB056393F82C00012806D19DF88E
:10D590000730022B08D10023BB70EAE7022803D131
:10D5A0009DF80730012BF5E7FFF76AF805EB450416
:10D5B000E400B0B9144BB8701C44382303FB056673
:10D5C0004FF47A7196F82830994096F82C30012B58
:10D5D00000D1C901204608F047FD204608F00AFDA9
:10D5E000C7E70A4B1C444FF47A71F3E7FFF748F89A
:10D5F0000028D0D0044C05EB450504EBC504F2E748
:10D6000010050020B824002088240020A024002039
:10D6100037B50F4CD1B100250123A16022712370D1
:10D620002A460C4B0C4800954FF0FF3108F036FCB1
:10D630000A4B0B4800952A464FF0FF3108F02EFCAC
:10D64000084A00236370137003B030BD2170F7E700
:10D65000100500209DD60008A024002069D60008EF
:10D6600088240020B824002010B5084808F074FC75
:10D67000074B002283F82020064B02225A80064BDB
:10D680005B6913B1BDE81040184710BD8824002025
:10D69000B824002010050020D804002010B5084848
:10D6A00008F05AFC074A012382F82030064A5380CA
:10D6B000064B5B6913B1BDE81040184710BD00BFB1
:10D6C000A0240020B824002010050020D804002049
:10D6D0002DE9F04FC378C82B8FB0824600F0298324
:10D6E0000FB0BDE8F08FDAF80820D05C591CC9B241
:10D6F000052816D8DFE810F00600AA00F000AE01F9
:10D70000E1018B02BA680023601C1355C0B2A31C50
:10D71000DBB24FF0020C02F800C001200334D054F9
:10D72000E4B20B469AF80C209A42DCD8002CD7D0F1
:10D73000C8238DF81430B74B8DF815409B680693BD
:10D740000DF11300FFF7E8F90020FFF7F1F90122CE
:10D75000002105A8FEF7CAFE9DF81300FFF7E8F9BF
:10D76000002DBDD1AC4CAD4F637803F003032A46C6
:10D77000294600930220AA4B08F000F82646636869
:10D7800000932A462946A74B022007F0F7FF16F818
:10D79000083F00932A462946A34B022007F0EEFFDC
:10D7A000012516F8013F009300223B461146022056
:10D7B000013507F0E3FF102DF3D1002211469B4BFA
:10D7C000022007F0DBFFA369009300221146984B6B
:10D7D000022007F0D3FFE369009300221146954B26
:10D7E000022007F0CBFF636A009300221146924BA0
:10D7F000022007F0C3FF94F8282001239340002261
:10D800001146009302208D4B07F0B8FF94F82C309E
:10D810000022012B236B00931146894B4FF002002D
:10D8200040F08D8207F0AAFF94F934300093002273
:10D83000844B1146022007F0A1FFE38E0093824B38
:10D8400000221146022007F099FF49E7BD6812F84F
:10D8500001C001222A55023300220234DBB2E4B2B5
:10D86000114696460CF0010C96F80080BEF1000FB0
:10D8700007D0120102F07002114369700546194683
:10D880004FE7B8F1000FF4D0BCF1000F21D005F83C
:10D8900004E004F1010E5FFA8EFE716805F80E10C7
:10D8A00004F1020E71685FFA8EFE090A05F80E1087
:10D8B00004F1030E5FFA8EFEB6F8068005F80E80BE
:10D8C000211DC9B296F807E005F801E00534E4B27D
:10D8D000614601328646C7E7555C382105F00305ED
:10D8E00001FB056103F1020B5FFA8BFB4D70002D0C
:10D8F00040F08E80D81C12F80B107160C0B203F19A
:10D90000050C105C01EB0021181DC0B27160105CA9
:10D910005FFA8CFC01EB0041716012F80CC0981D9D
:10D9200001EB0C6903F11601DFF820C1C6F8049081
:10D93000C0B2C9B286460130C0B212F80EE00CF88F
:10D9400001EF8842F6D1115CB16103F11700C0B25A
:10D9500003F11E0B105C01EB002103F11800C0B2B3
:10D96000B161105C01EB004103F11900C0B2B1617B
:10D97000105C01EB006803F11A01C9B2C6F8188007
:10D9800003F11B00515CF161C0B25FFA8BFB105CCC
:10D9900001EB002103F11C00C0B2F161105C1D33EA
:10D9A00001EB0041DBB2F161D35C0DF1170001EB3B
:10D9B000036321220021F361039321F001FE40F271
:10D9C0000112ADF814207278039B0A93C2F301028E
:10D9D0008DF8162005A81E4ACDF818900792CDF8AC
:10D9E000248002F065FC012390B93370B9680223EA
:10D9F0000B55621C1C44382303FB0563D2B25B78D1
:10DA0000C3F3010343EA80008854E4B2594688E630
:10DA10000120EBE710050020B8240020FB8003085C
:10DA2000C0800308D3800308E8800308BA7D030898
:10DA30000181030814810308278103083A81030840
:10DA40004F8103086281030878810308BF24002006
:10DA5000C0240020555C382005F00305023300FB8C
:10DA600005FB5FFA83F906EB0B034FF0000818463D
:10DA700010224146083083F80180C3F804800393E4
:10DA800005F0A4FE039BC3E90688BB68032204F1EA
:10DA900001081A5528465FFA88F802F051FC40B197
:10DAA00045F00403BA68023402F80830E4B249468B
:10DAB00037E606F80B002B46F4E74FF0000B8DF825
:10DAC00013B0555C03F1020815F003055FFA88F8FE
:10DAD00040F09680DFF874B24FF002098BF82C907A
:10DAE000D81C12F80810CBF82410C0B203F10B08B0
:10DAF000105C01EB0021181DC0B2CBF82410105CA3
:10DB000001EB0041581DC0B2CBF82410105C01EBB2
:10DB100000618F480844991DC9B2CBF82400515CBC
:10DB200001F00F018BF82810D91DC9B203F10800CC
:10DB3000515CCBF83010C0B25FFA88F8105C41EA53
:10DB4000002103F10900C0B2CBF83010105C0A3399
:10DB500041EA004164204143DBB2CBF83010D35C92
:10DB60008BF834300DF113020BF12C01284602F032
:10DB700013FC002849D105A808F06AF8DBF8242036
:10DB8000059BA2EB030BBBF1000F31DD4FF47A7163
:10DB900001FB0BF16F48039108F066FA6D4808F03D
:10DBA00029FA039900916C4B29462A46484607F00A
:10DBB000E5FD0121BA6804231355601CC0B29DF82D
:10DBC00013C002F800C0A31CDBB271B102F803B0AD
:10DBD000E31CDBB24FEA2B21D154631D0434E4B2C1
:10DBE0004FEA2B4B02F804B0DBB21C46414698E5E5
:10DBF0009DF8133043F010038DF813302946D9E710
:10DC000010238DF813305946D4E7AB46F6E74FF0B2
:10DC1000000B8DF813B0555C03F1020815F00305F5
:10DC20005FFA88F87ED1DFF824B14FF001098BF854
:10DC30002C90D81C12F80810CBF82410C0B203F1B5
:10DC40000B08105C01EB0021181DC0B2CBF82410AA
:10DC5000105C01EB0041581DC0B2CBF82410105CE1
:10DC600001EB00613A480844991DC9B2CBF8240081
:10DC7000505CC0F30210ABF83600515C01F00F01AC
:10DC80008BF82810D91DC9B203F10800515CCBF8FC
:10DC90003010C0B25FFA88F8105C41EA002103F14D
:10DCA0000900C0B2CBF83010105C0A3341EA0041E1
:10DCB00064204143DBB2CBF83010D35C8BF83430B6
:10DCC0000DF113020BF12C01284602F065FB70BB2D
:10DCD00005A807F0BDFFDBF82420059BA2EB030B92
:10DCE000BBF1000F16DD4FF47A7101FB0BF11948FF
:10DCF000039108F0B9F9174808F07CF903990091ED
:10DD0000154B29462A46022007F038FD4946BA68D5
:10DD1000052351E79DF8133043F010038DF81330BD
:10DD20002946F4E710238DF813305946EFE7AB4648
:10DD3000F6E70024094F054EFF252346F2E407F0DD
:10DD40001DFD94F934300093054B79E5B82400208B
:10DD5000803DD512A0240020A580030810050020D6
:10DD60006281030800487047D8040020044B054A2C
:10DD700093F81831022B18BF062382F890347047AD
:10DD80005C2B002020310020034BD3F8483313B123
:10DD90005B6903B11847704720310020034A1378AC
:10DDA00043F004031370FFF7EFBF00BF042500200A
:10DDB0001FB50A4B8DF8090093F87C208DF80A20D6
:10DDC00093F88C2093F848000D3202A98DF80820B2
:10DDD00003F082FDC0B205B05DF804FB5C2B0020AF
:10DDE00008B5074808F0B8F8064B93F81A2412B1A2
:10DDF000012283F81924BDE80840FFF7C5BF00BF22
:10DE0000203500202031002010B50C4CD4F84033D0
:10DE100043F08003C4F8403394F81A3413B100205F
:10DE2000FFF7DEFF94F8913423F0120343F012035E
:10DE300084F89134BDE81040FFF798BF20310020EE
:10DE40002DE9F041DFF8AC8098F81831022B064636
:10DE50000D4602D0284BDB6A984702F078FE044654
:10DE600028B1022002F069FE002002F06BFE98F853
:10DE70001831012B17D102F06CFE074630B100209B
:10DE800002F05CFE002002F05EFE3C4602F063FE03
:10DE900048B1002002F053FE002002F055FEBDE81C
:10DEA000F041FFF763BF002CF9D1144C94F8902493
:10DEB00094F81A34BAB90BB184F84164304602F0D0
:10DEC000EBFFD8F82C0008F00DF8D4F8B4339842E2
:10DED000E5D30B4808F040F894F8913443F0100370
:10DEE00084F89134DBE70BB184F84154284602F002
:10DEF000D3FFF1E75C2B0020B88803082031002015
:10DF0000B8340020074A10B5137843F002031370A9
:10DF1000FFF73AFFBDE81040034B01220021022029
:10DF200007F02CBC042500208B810308074A10B59C
:10DF3000137843F008031370FFF726FFBDE8104085
:10DF4000034B01220021022007F018BC0425002009
:10DF50009B8103082DE9F0410F4616461D46804679
:10DF600007F0B6FF0B4A0C4C1378278123F01103FE
:10DF700043F01103C4E90008137066812573FFF7AD
:10DF800003FFBDE8F041054B01220021022007F00C
:10DF9000F5BB00BF04250020F0240020AB8103085E
:10DFA00013B507F095FF0D4B6C461860204607F03F
:10DFB0004FFE94E803000A4A0A4B83E803001378F3
:10DFC00043F020031370FFF7DFFE074B012200210F
:10DFD000022002B0BDE8104007F0D0BB00250020B1
:10DFE0000425002058340020B88103082DE9F041B1
:10DFF00092B0064602F0ABFD002840F05881AD4DCE
:10E0000095F81831012B09D02B6BAB4C93B194F8D8
:10E010000431BBB1042B6FD0032003E002F099FD63
:10E0200018B10F2012B0BDE8F08102F094FD002875
:10E03000EAD0F6E7B5F82031D4F81C24013B53436D
:10E040002B63E4E79D4803F07EFB002840F012813B
:10E0500094F80C3123802B6B0C930DF1180895F874
:10E0600039308DF83830404695F81C318DF83A300B
:10E0700007F014FED5F82831009302AF98E80600A7
:10E08000D5F82431384607F09FFD97E803000FAB21
:10E0900083E80300EB6A0D9300238DF84430238856
:10E0A000ADF8463095F8303101228DF839201BB992
:10E0B0008DF844208DF83930814B0093814B95F8D1
:10E0C0004800A3F179020CA903F07BFCC0B10B2836
:10E0D000A8D1D4F8941499B1002EA3D0D4F8403329
:10E0E000794843F02003C4F8403307F0BDFF764879
:10E0F00007F080FF002095E7704803F058FBA4E785
:10E1000095F8487095F9693095F9392095F87D10A2
:10E110006E4E384603F062FC009641B2EB6C95F807
:10E1200050203846183603F0FDFB0096EB6C95F84E
:10E13000502095F9701095F8480003F0F3FBD4F8DF
:10E14000C413AB6DD4F8DC230B44C4F8B033EB6DCF
:10E150001344C4F8B43394F80431042B07D02B6E65
:10E160000B44C4F8B0336B6E1344C4F8B4330023CB
:10E17000089395F83031002B40D100238DF81330EF
:10E1800095F839308DF8213095F838308DF82230F7
:10E19000D5F880300993D5F884300A932388ADF8F8
:10E1A0002C3095F8303194F81B648DF82E3095F8AA
:10E1B0004800474B8DF820600DF1130208A903F0C9
:10E1C000C5FB012384F8413495F8393084F8423492
:10E1D0009DF8133084F84334D4F81C34C4F85064E8
:10E1E000C4F84834C4F8583402F0B7FCC8B1D4F8C5
:10E1F0001C0402F0C4FCA0B1102013E708A802F030
:10E200007BFD60B995F9390094F837629DF820706C
:10E21000FFF7CEFD3E44B042AFD2082002E7132004
:10E2200000E795F81831012B01D102F0AAFC02F0A9
:10E2300097FC0023059394F8043195F9395094F82C
:10E240001B649BB1042B7FF4E7AE05A802F088FFA6
:10E2500058BB94F8183413B1059B013B0593174B39
:10E2600005983246E9B202F0E1FF02E0134802F0FD
:10E27000B1FF08B11120D5E6D4F8403394F80C1161
:10E28000218043F00203C4F8403394F81834114855
:10E290000133DBB284F8183484F845340E4B002582
:10E2A0009B6AC4F89854984724E71220BAE60E20D7
:10E2B000B8E600BF5C2B002020310020283200206F
:10E2C0008C2B0020B435002088340020D834002066
:10E2D0003C35002022310020B888030873B5134D67
:10E2E000134E0096EB6C95F8502095F9781095F840
:10E2F000480003F017FB95F83031337595F8480066
:10E3000040F2012306F13C023146738203F016FB12
:10E3100050B196F83C3086F88230064B00205B6B9B
:10E320009847F37C86F8A83002B070BD5C2B0020C3
:10E3300008350020B8880308F8B5324C94F8183135
:10E34000012B05460ED0022B4ED0002B57D138B9E9
:10E35000D4E91B0104F1740383E803000020F8BD35
:10E36000012806D102F0FEFB0028F8D184F81851EC
:10E37000F5E7022843D1244E84F8180106F5747C91
:10E38000BCE80F0006F57A770FC79CE8030094F805
:10E39000E92094F8003187E8030086F8FB53D2B1F6
:10E3A000022B18D1D4F804316367C6F8EC3394F823
:10E3B0007D3094F8082186F8F83394F88C3084F88E
:10E3C000782086F8F93396F81B2486F8E82340F283
:10E3D0000133A6F8FA33002386F81A340B4BDB6AB4
:10E3E0009847FFF77BFFB9E748B9074B84F8180156
:10E3F000062283F89024054BDB6A9847AEE703209A
:10E40000ADE700BF5C2B002020310020B888030856
:10E41000F0B5504C504EB4F8DC202287D4E92D01E1
:10E4200094F8B12084F8692004F16C0282E80300BA
:10E43000D4E92F0104F1740282E80300B4F8C42087
:10E44000A4F87C2091B0D4F8CC20D4F8C810C4F83B
:10E4500084200025D4F8D020C4F888200123A4F813
:10E460002031C4F8801084F83051A56284F81B5123
:10E4700084F83A5084F81D5184F81E51C4F8345180
:10E48000C6F89854A6F8185486F81A54A4F83851C7
:10E490008DF8183004F50973039304F50A7394F8A2
:10E4A0004800049303A92D4B84F84551C4E94F5506
:10E4B000A4F84651059303F01DFAE36EC6F8D43371
:10E4C00094F87D3086F8E03394F88C3086F8E133A8
:10E4D0004FF48073A6F8E23386F8D05394F83031C5
:10E4E00086F8E43306F574770FCF06F57A740FC417
:10E4F00097E8030040F2012384E80300A6F8FA330A
:10E50000D6F8483386F81B54CDE901551BB15A683B
:10E510005B6901920293124B0793A3F148020892A0
:10E52000A3F1140209920F4A0B9229330A93A2F124
:10E530009C030C93A2F198030D93131D0E9301A954
:10E5400002F14C0307A802F599620F9302F0F4FA66
:10E5500011B0F0BD5C2B00202031002008250020E8
:10E5600088350020402C0020F8B50D4F0D4E0C468C
:10E5700007F0F2FC3B6B98470B4A96F8480021469F
:10E5800003F0DCF950B1094D706D95F8243485F82D
:10E590006A347B6B9847E37C85F89034F8BD00BF04
:10E5A000B88803085C2B002044350020203100206F
:10E5B0000F4890F81B3480F8B8330E4B93F869205D
:10E5C00080F8BB2393F87D2080F8C82393F88C2033
:10E5D00080F8C92393F8303180F8CC330022A0F8BA
:10E5E000CA2300F56E7100F56070FFF7BDBF00BF74
:10E5F000203100205C2B0020114890F89034EBB1C2
:10E6000090F81B3480F8D0330E4BDA6EC0F8D42368
:10E6100093F87D2080F8E02393F88C2080F8E123A4
:10E6200093F8303180F8E4334FF48072A0F8E2239D
:10E6300000F5747100F56670FFF796BF704700BF74
:10E64000203100205C2B002070B5344C2421204662
:10E6500005F0BEF8636A984218BF60624FF01C0173
:10E660002F4814BF0125002505F0B2F8636C9842CD
:10E6700018BF60644FF480712A4818BF45F0020546
:10E6800005F0A6F8D4F84831984218BFC4F84801FC
:10E690004FF0D401244818BF45F0040505F098F860
:10E6A000D4F82032984218BFC4F820024FF000017D
:10E6B0001E4818BF45F0080505F08AF8D4F8243242
:10E6C000984218BFC4F824024FF46071184818BF6C
:10E6D00045F0100505F07CF8D4F8A835984218BF2D
:10E6E000C4F8A8054FF01401124818BF45F02005E2
:10E6F00005F06EF8D4F8C03598420F4B18BFC4F837
:10E70000C005D3F8483318BF45F040052BB11B694D
:10E710001BB12846BDE87040184770BD5C2B002037
:10E72000842B0020A42B0020A82C0020802D00206A
:10E73000842D002008310020203100202DE9F04FE9
:10E740008FB04FF00009012B06460F4690468DF81A
:10E750000D90ADF8109002D84C46BC4202D30FB0D9
:10E76000BDE8F08F305D02F007FB2044B842F6DCD4
:10E77000335D651C023BEDB2112BF0D801A252F8BB
:10E7800023F000BFCDE70008F7E70008F5E8000830
:10E790001DE900089BE90008C1E9000827EA000814
:10E7A0004FEA0008D5EA00085FE700085FE70008C5
:10E7B00029EB00085FE700085FE70008D1EB0008DD
:10E7C000F9EB000831EC000865EC0008052002F0C8
:10E7D0007BFB70B10521002002F03CFB725DBA4B5F
:10E7E000E51C0234E4B283F85C24325D83F85D24D6
:10E7F000EDB22C46B1E700238DF80E308DF80F30C6
:10E800008DF814308DF81830B9F1000F6DD1AF4C80
:10E810004FF0050994F87C208DF831206B1E94F898
:10E8200039208DF83320334494F838200B938DF839
:10E83000342094F81A3194F868208DF83520D4F8F3
:10E840002C218DF832300A9273B37B1C5B1BDBB238
:10E850008DF8303006AB019305AB009394F8480077
:10E860000DF10F030DF10E020AA903F07BF88DF8EC
:10E870000D0000F00700072813D194F939209DF905
:10E880000E3084F839309A429DF80F3084F83830D1
:10E89000B8BF01229DF81430B8BF84F81D2184F858
:10E8A00068304FF0000A09E00523D1E701220DF19D
:10E8B0000D01032002F078F90AF1010A5FFA8AF2E9
:10E8C0009DF81830B3FBF9F19142EFD82B44DDB23B
:10E8D0006B1EDBB29F420BD9F25C032A9AD0AF4287
:10E8E00088BF1D464FF0010983E70534E5B2F9E71B
:10E8F0001D46F7E7735D754903F00F03012281F8A8
:10E900001B31023402FA03F3A1F82031E4B20022F1
:10E9100004A9042002F048F925466AE707238DF888
:10E920000D30735DC3F3021203F00F038DF828302E
:10E93000E31CDBB28DF82920F25C231DDBB2651DE0
:10E94000F35C0234E4B21B0443EA0223325D5F4C01
:10E9500013436422534394F848000B930AA903F02D
:10E9600010F800F00703072BEDB28DF80D000CD165
:10E970009DF8283084F8703084F878300B9BE3667B
:10E9800063679DF8293084F869308DF81000012202
:10E9900004A9052002F008F92BE74B4BD3F84833C4
:10E9A00063B11B6853B1984708F03F038DF810001E
:10E9B0008DF81130022204A90620EBE7FF20F3E7CF
:10E9C00003238DF80D30735D8DF81C300AAB069370
:10E9D000E31CDBB2A51DF25C231DDBB206A9F35CD0
:10E9E0001B0443EA0223A21CD2B20534B25C1343D7
:10E9F00064225343E4B20A9300230B93335D8DF8F2
:10EA00003030324B93F8480002F0C1FFC3B2002807
:10EA1000EDB28DF80D30FFF6ECAE8DF8103001221E
:10EA200004A90720B6E7735D03F00F03012B4FF431
:10EA30007A7238BF01235343244A0234936503F5A5
:10EA40007A73D365E4B2002204A9082062E7735DFB
:10EA50001E4DC3F340128DF8152095F84800C3F3FE
:10EA6000001205A903F00F038DF814208DF816305D
:10EA700002F093FF02340130E4B23FF44DAFBDF831
:10EA80001430134AA5F87C309DF816309DF814A078
:10EA9000D05CF3F78FFA0223C5F880000AA995F835
:10EAA00048008DF828308DF82AA002F015FF95F95E
:10EAB0003930069040B29842B8BF184685F8390000
:10EAC000002204A9092025E7203100205C2B00202A
:10EAD000C581030803238DF80D30735D8DF8283050
:10EAE000E31CDBB2651DF25C231DDBB20234F35C78
:10EAF000E4B21B0443EA0223325D1343642253430E
:10EB00000B93644B0AA993F8480002F04CFFC3B280
:10EB10000028EDB28DF80D30FFF66BAE8DF8103099
:10EB2000012204A90A2035E7092002F0CDF9DFF817
:10EB300068B1002849D00921002002F08BF9002398
:10EB4000ADF81E30A31CDBB2F25CE31CDBB216F89E
:10EB500003A0735D4FEA0A4A4AEA022A4AEA030A14
:10EB6000231DDBB2A51D0534F35CE4B24AEA036A57
:10EB7000335D4FF47A7253430AAC1B122046ADF852
:10EB80001C3007F065F8454B53440693DBF83C33E3
:10EB900000930DF1180A9AE80600DBF8383308A84C
:10EBA00007F012F8099B009394E80600089B504672
:10EBB00006F0EFFF9AE8030007F022F801F0DCFF0F
:10EBC0000123EDB28BF8383413E68BF8380410E6E5
:10EBD0000C2002F079F900283FF40BAE0C21002044
:10EBE00002F038F92C4B93F89034043B012B7FF65C
:10EBF00000AE01F0BDFFFCE5A31CDBB2725DF15C71
:10EC0000E31CDBB2651DF35C0434E4B21B04305D2D
:10EC100043EA012313436421594300F00F0001F03C
:10EC2000A8FFEDB28DF81000012204A91120B1E671
:10EC30000D2002F049F900283FF4DBAD0D21002042
:10EC400002F008F9A31CDBB2154AF05C735D126890
:10EC5000251D0334E4B243EA0020315DEDB201F03A
:10EC60008AFFC6E5725DA31C251D0334DBB2E4B246
:10EC7000F15C335D1B0443EA0123134364205843D2
:10EC800001F07BFFEDB28DF81000012204A91320E2
:10EC900080E600BF5C2B002020310020803DD51293
:10ECA000F02400200E4B93F89124920703D593F89B
:10ECB0008F24012A08D90B4991F81A2122B18A6AB6
:10ECC000501C18BF01328A620022A3F8182483F86E
:10ECD0001A24D3F8402322F00202C3F840237047DD
:10ECE000203100205C2B002070B5184C1848194DBD
:10ECF00007F032F9D4F84033D4F89804D5F890608E
:10ED000023F02003C4F8403338B107F0EBF8864213
:10ED100003D2002385F83A3070BD0120FFF766F971
:10ED20000028F9D00B28F7D095F8393084F8423410
:10ED3000092094F8183484F8453484F8410402F02A
:10ED4000ABF8BDE87040FFF7ADBF00BF2031002039
:10ED5000883400205C2B0020094BD3F84023012A83
:10ED60000AD008490978C90708D43AB993F8920437
:10ED7000013818BF012070470020704701207047FC
:10ED80002031002004250020034BD3F84003431E0C
:10ED900058425841704700BF203100202DE9F04F04
:10EDA000A9B0EFF3108272B6DFF8F0B20021DBF801
:10EDB0000030CBF8001082F31088B94C002B00F023
:10EDC000E180DAB29B06039264D5B64D95F818310E
:10EDD000022B02D0B44BDB6A9847EFF3108872B66F
:10EDE000B24F07F075F83E68D4F8B013361A3144C4
:10EDF000AF4807F039F9AE4807F0FCF8D4F8B4137F
:10EE0000AC48314407F030F9AA4807F0F3F888F32A
:10EE1000108894F81A34002B00F06B81152312A986
:10EE200095F848008DF8483002F056FDD4F8B41338
:10EE30000F900144A04807F017F99F4807F0DAF84F
:10EE40003B6894F81B24EB620DAF38468DF87020B8
:10EE50001D9306F023FFD5F82831009306AE97E8FE
:10EE60000600D5F82431304606F0AEFE96E80300E1
:10EE70001FAB83E80300D4F81C341E9395F830319F
:10EE800095F84800003B18BF01231CA98DF871308C
:10EE900002F02BFD039BDF0648D5824DDFF81CA254
:10EEA000D5F8E42004929BF80020BAF90A809AF978
:10EEB0000C90A4F88C84002363F300020A9384F876
:10EEC0004434A4F8223484F82534C4F82834A4F84F
:10EED0002C3484F82E34C4F8303484F82034C4F848
:10EEE000343484F83834C4F83C346F4B8BF8002049
:10EEF00094F89024DB6A84F88E9484F88F24DAF8EE
:10EF00000470BAF80860984794F88F3413B96948C8
:10EF100007F022F83146384601F017FE83460028F4
:10EF200000F0EA80A4F87E8484F88094039B19079B
:10EF30001AD55C4B93F81831022B02D05A4BDB6A7E
:10EF400098470220FEF712FF84F8410401F0A4FF65
:10EF500094F81A3413B1012384F8193494F89134D5
:10EF600043F0100384F89134039B5A0703D506211C
:10EF70000520FEF765FF039B9B0703D504210320B3
:10EF8000FEF75EFF01F000FE94F89124D7065FD5EE
:10EF9000002384F89234D4F840331E0644BF23F093
:10EFA0008203C4F8403312F0050F00F0FB820B20FF
:10EFB00001F08AFF002800F0F58294F89134DD0713
:10EFC00000F1F082580740F10783D4F8403323F072
:10EFD0000203C4F84033D4F8402382BB94F8915420
:10EFE00015F001011EBF2B4662F3000384F8913433
:10EFF00094F891345E0744BF6FF3820384F8913430
:10F00000012384F8923421B1D4F844332C481B688E
:10F0100098476D070BD52B4801F062FF01F090FF78
:10F0200028B194F8913443F0040384F8913401F04A
:10F0300098FD94F891346FF3041384F8913401230C
:10F0400084F8923494F8913443F0200384F8913496
:10F0500094F8913418070AD56FF3C3031A4984F85A
:10F060009134D4F84433A1F12400DB68984794F834
:10F07000913499070AD56FF34103134984F8913409
:10F08000D4F84433A1F16C005B68984794F890344D
:10F09000022B1BD1FFF722F918E000BF0425002046
:10F0A000203100205C2B0020B888030800250020B8
:10F0B000A0340020B834002020350020F0240020A7
:10F0C0006035002074350020AC35002094F8913470
:10F0D0009A0640F1C4826FF3451384F89134D4F852
:10F0E0004033002B40F0BB8229B0BDE8F04FFFF762
:10F0F000ABBA84F84134A3E695F81831012B0CD152
:10F1000001F027FD804668B1584601F017FD5846CA
:10F1100001F019FD042384F88F347EB9012384F8AB
:10F1200021344FE101F017FD0028F6D0404601F0F0
:10F1300006FD404601F008FD0523ECE73B7805930A
:10F140005B09013B062B00F21782DFE813F0070092
:10F15000150295001502920015020602102EDDD947
:10F1600095F830311297F6B28DF84C60002BD5D15E
:10F170001CA804F03FFA12AA1CA9FF2002F072F9A1
:10F180009DF85830C3F3030307468DF82C3095F8EB
:10F19000480095F87D308DF82D3007220BA902F03C
:10F1A000AEFB002F5DD100285BD09DF853309DF859
:10F1B00052201599C5F8E4101B0443EA02239DF878
:10F1C000512002201343C5F8E03004F021FA9DF8E5
:10F1D000583095F8480085F82E71C3F30212C3F336
:10F1E000030385F8703085F878309DF8593085F83C
:10F1F0006920012B38BF01234FF47A725343AB656A
:10F200001344EB650DF15A034FF001081093113EC2
:10F2100094F81B348DF83C300FA985F868808DF880
:10F22000446002F074FB0223404685F8303101F05F
:10F230004BFE18B14146384601F00CFE94F88F346D
:10F24000012B00F2A78194F81A34002B40F09A8128
:10F2500094F8913443F0100384F89134FEF786FD5E
:10F2600064E6012001F030FE0028E7D001210720EC
:10F27000E2E7012384F8203495F87D308DF82E30B4
:10F2800094F824348DF82D3095F88C3095F848009A
:10F290000D330BA98DF82C3002F01EFBA6F10D03E7
:10F2A0001BB2099023EAE37300B283423FF736AF03
:10F2B0000B2E7FF633AFBA4B25931CA8FF231C9768
:10F2C0008DF874608DF8983002F0E2F90746002856
:10F2D0007FF424AF95F81831012B13D101F039FCDC
:10F2E000002872D0384601F029FC384601F02BFC8A
:10F2F00004239DF87C101E9884F88F34C1F300110C
:10F3000001F041FC9DF87C301E99C4F8341413F0D0
:10F310000F0203D09DF89000002862D19DF898005C
:10F32000002861D0002A7FF4F9AE9DF89020002AD1
:10F3300014BF4FF003084FF0020800220A92D5F8DC
:10F34000EC2095F8E900914251D100284FD0D5F832
:10F350000C1195F8EAB009680A9195F8181102297C
:10F3600002D1032184F88F14B8F1030F7FF4D6AED5
:10F3700013F0600F7FF4D2AE0492012795F82E317E
:10F38000BBF1000F36D0BBF1010F13D1012B33D1EC
:10F390006FF0090646FA08F606F00106C6F1020605
:10F3A000F6B2BDF87E100AAA304601F0E5FE38B389
:10F3B000072823D0012384F821340A9BC4F8303471
:10F3C000C4F86C34FEF720FDB0E501F0C4FB002862
:10F3D00098D0384601F0B3FB384601F0B5FB052361
:10F3E00087E74FF00008A8E74FF00108A5E74FF0C6
:10F3F000010BC3E70426D4E70326D2E70823DAE7A4
:10F400001CAB009304990A9B3246584601F076FFE4
:10F4100020B1022814BF0B230A2380E60A9BC4F8FC
:10F420003034C4F86C349DF87C3084F82104C3F384
:10F43000401384F82E3484F8443494F88F3484F8DC
:10F440002274012B9EBF0122A86285F81E21012F84
:10F45000C4F8280484F82C0484F8410438D102222A
:10F4600084F8202495F83A20002A4AD19DF87C207F
:10F47000D60646D4012B94F840149DF87C2005D87C
:10F48000012901D1900601D501F020FCB8F1020F4D
:10F4900094F88F3443D0B8F1030F0AD09DF87C1054
:10F4A000B8F1010F4A4601F00F0120A83BD0FFF749
:10F4B00045F99DF8903084F82334259BC4F828340E
:10F4C0009DF8983084F82C34012384F82D3430E0F2
:10F4D000059A02F0E002A02A1BD195F82E11012214
:10F4E00085F83A2009B927996963012B84F820240B
:10F4F00007D9D5F89020C4F83C24DAF80020C4F8E5
:10F50000982495F81821002AB4D1012284F82524E2
:10F51000B0E7002285F83A2084F82024A6E79DF879
:10F52000981025984A46FFF709F99DF8903084F81D
:10F5300023349DF89020E02A08D195F81F312BB98B
:10F5400084F82324C4F82834A4F82C3494F8913493
:10F5500043F0020384F8913470E6114D013EB2B2DB
:10F56000791C284604F01EF90323A4F82034C4F8BB
:10F57000285484F82C64E9E7012384F82134FEF749
:10F5800043FC5BE694F84434002B3FF461AE00206A
:10F59000FEF726FC94F88F34022B3FF45FAE57E65B
:10F5A0005833002094F89134590715D5012001F003
:10F5B0008BFC60B1012001F05FFC08B984F81804ED
:10F5C000D4F8403323F00203C4F8403304E00620AB
:10F5D00001F07AFC0028F3D194F89134DA077FF532
:10F5E000FAAC94F840240AB1032A18D11D4A94F8C1
:10F5F000181492F86820914205D29B0723D594F8FD
:10F600008F34012B1FD8184806F0A6FCD4F84033DD
:10F6100023F02003C4F84033FFF744FBDBE4012A66
:10F6200011D194F81924002A3FF4D5AC0D4A94F86E
:10F63000181492F868209142E5D29F0703D594F8F8
:10F640004434002BDFD194F8913400206FF304137D
:10F6500084F8913484F81904FFF746FBBBE429B021
:10F66000BDE8F08F5C2B0020883400202DE9F04F9E
:10F6700089468DB090460746002800F08F8100290A
:10F6800000F08C810368002B00F088814368002B18
:10F6900000F084818368002B00F08081C368002B18
:10F6A00000F07C81104602F013F9002800F0788108
:10F6B000BD4CBE4D384601F083FB40F2C4520021E0
:10F6C000204604F083F840F21C520021284604F042
:10F6D0007DF8B74BC4F82C3104F50973089304F591
:10F6E0000A7300264046099308A9B24B84F8488063
:10F6F0000A9384F8186184F88C608DF82C6002F00D
:10F70000F9F80F2306A994F848008DF8183002F094
:10F71000E3F8801B18BF01204FF00A0B84F81C018E
:10F7200006A994F848008DF818B002F0D5F84FF00B
:10F73000060A84F8DC0006A994F848008DF818A0A1
:10F7400002F0CAF8102384F8DD0006A994F84800F6
:10F750008DF8183002F0C0F81123C4F89C0006A9F7
:10F7600094F848008DF8183002F0B6F81223C4F867
:10F77000A00006A994F848008DF8183002F0ACF803
:10F780001323C4F8A40006A994F848008DF8183093
:10F7900002F0A2F81423C4F8A80006A994F84800BF
:10F7A0008DF8183002F098F81623C4F8AC0006A9BA
:10F7B00094F848008DF8183002F08EF8172384F87A
:10F7C000B10006A994F848008DF8183002F084F8CA
:10F7D00018230DEB0301C4F8B400C4F8BC0094F87E
:10F7E00048008DF8183002F077F8C0B21D2384F875
:10F7F000B80084F8C00006A994F848008DF81830C5
:10F8000002F06AF81E2384F8C40006A994F84800A0
:10F810008DF8183002F060F81F2384F8C50006A99F
:10F8200094F848008DF8183002F056F82023C4F8F8
:10F83000C80006A994F848008DF8183002F04CF87A
:10F840000B23C4F8CC0006A994F848008DF81830B2
:10F8500002F042F80C2306A9A4F8D00094F848005E
:10F860008DF8183002F038F8D4F89C306365D4F87D
:10F87000A030A365D4F8A430E365D4F8A83023669B
:10F880004FF00108D4F8AC300590A4F8D2006366BC
:10F8900084F8B080C4F894B084F898A0C4F84CB050
:10F8A00084F850A084F8688084F81F81C5F84893D4
:10F8B000FEF7AEFDC5F84473C4E90B663E4B84F811
:10F8C000198185F89164C5F8408332464FF0FF31C5
:10F8D000009605F55A7006F0E1FA384B009632466C
:10F8E0004FF0FF3105F5607006F0D8FA344B009602
:10F8F00032464FF0FF3105F5667006F0CFFA02AFE1
:10F90000304B009632464FF0FF3105F5806006F02F
:10F91000C5FA384606F0C2F997E8030004F5927379
:10F9200083E80300284B294F1E60294BC5F84C3350
:10F93000284BC5F85433284BC5F85C33274BC5F822
:10F940005033274BC5F8583305F553703B6898473B
:10F9500004F5A67003F06AFC20B1112630460DB004
:10F96000BDE8F08F204601F0D7FB0028F5D101F06B
:10F970000DF9B8B91B4801F021FC06460028ECD16E
:10F980007B69984703F0ECFEBB6D94F8190198472A
:10F99000FB6A9847012385F89234DFE70326DDE709
:10F9A0000926DBE71326D9E75C2B00202031002055
:10F9B0000004000108250020E9EC0008B1E500087A
:10F9C000F9E50008E1DD000804250020B8880308F7
:10F9D000A1DF000855DF00089DDD00082DDF0008CD
:10F9E00005DF0008442C002008B5034B0020C3F8B5
:10F9F0004003FEF7BBF908BD2031002010B5FFF72A
:10FA0000ABF90A4C60B90A4B93F81831022B02D1BA
:10FA1000084BDB6A98470123C4F84033002010BD2F
:10FA2000D4F84003013818BF0120F8E72031002046
:10FA30005C2B0020B888030838B5124C204606F02D
:10FA40008BFA04F1180006F087FA04F1300006F092
:10FA500083FA04F1980006F07FFA01F081F80A4B6E
:10FA60000025DB6A984744F8285CFEF7EDFD07495E
:10FA7000074840F2C45203F095FE012344F8283CA5
:10FA8000284638BD88340020B88803085C2B002045
:10FA90009825002070B52E4B8AB0054693F8DD00FE
:10FAA0008DF8090093F8DC008DF80A0029489A6A5D
:10FAB00090F81804039200268DF80B0004960C466B
:10FAC000002940D00692D3F8882007921A8F93F825
:10FAD0001A118DF8151052BAADF8202093F87C2039
:10FAE00093F848308DF8243003AB8DF822008DF860
:10FAF000232000930DF10A020DF10B030DF1090112
:10FB000005A88DF8146000F0A9FF9DF90900FEF723
:10FB10004FF9607004A801F0EFF8B0B9049A0F2A09
:10FB20000DD863789A420AD81544AB42A3EB020180
:10FB30002CBF002001202170C0000AB070BD00233E
:10FB400023700820F9E70320F7E71320F5E700BF4B
:10FB50005C2B0020203100201FB50446002800F057
:10FB600010810378412B00F20781DFE813F0420097
:10FB700049004D005100550059005E000501050186
:10FB80000501050105010501050105016500690083
:10FB90006D0078007F00820085008A0088008C005C
:10FBA00090009300960099009C009F00AE00B20068
:10FBB000BA00B600BE00C100C500CE00CA00CC002D
:10FBC0000501D20005010501050105010501050139
:10FBD00005010501050105010501050105010501F5
:10FBE0000501DA00DE00E200E700EB00EF00F300C1
:10FBF000FC00664B93F818312371002004B010BD4F
:10FC0000624B93F83031F7E7406803F0ADFCF4E75E
:10FC1000406803F0EFFCF0E75C4B93F81A31EBE738
:10FC20005A4BD3F8E0306360E7E7584B011D93F877
:10FC3000300103F0F7FCE0E7544B93F81931DBE7B0
:10FC4000524B93F88C30D7E71C238DF808304F4B7C
:10FC500002A993F8480001F03FFE6060CDE74C4BED
:10FC6000043493E8030084E80300C6E7494B0434F6
:10FC7000F7E7494B0434F4E7484B0434F1E71A231F
:10FC8000E3E71923E1E7414B93F86830B4E73F4BD2
:10FC90005B6DC8E73D4B9B6DC5E73C4BDB6DC2E739
:10FCA0003A4B1B6EBFE7394B5B6EBCE702238DF806
:10FCB0000830364B02A993F87C2093F848008DF861
:10FCC0000A2001F009FE207197E7304B93F8DD30F0
:10FCD00092E72E4B93F839308EE72C4B93F8DC30BB
:10FCE0008AE72A4B93F8383086E7284BDB6C9AE793
:10FCF000264B93F850307FE7244BD3F88430636071
:10FD00007BE7224B8FE7264B8DE7204BD3F8CC3097
:10FD1000F5E71E4BD3F82C31436001F06BFEA06079
:10FD20006BE71A4BD3F890307DE7184B93F81F31EF
:10FD300062E7164BB3F88830A3805EE7134BB3F845
:10FD40008A30F9E7114BB3F8D030F5E70F4BB3F831
:10FD5000D230F1E70D4B93F848200AB1062A12D1B0
:10FD6000B3F8A035E8E7094B93F848200AB1062A12
:10FD700009D1D3F8A43556E704B0BDE8104000F02F
:10FD8000F3BE03203AE7182038E700BF5C2B0020C1
:10FD9000C82B0020102C0020D02B0020182C002075
:10FDA000982500207FB5044610B9032004B070BD2B
:10FDB000A34DD5F840339A0700F16F820278412AAB
:10FDC00000F26882DFE812F04200470055005B0055
:10FDD0005F00640069007600810087008D00930059
:10FDE00099009F00A500AB00B5006602BA00DC00D8
:10FDF000EF0016013801290142014B014F01530167
:10FE000057015B0166025F01710199018701AB0136
:10FE1000B101B801BD01C201660228026602660294
:10FE20006602660266026602660266026602660292
:10FE300066026602660266026602660234023902E1
:10FE40003E02430248024D0252025C020079FEF774
:10FE500073FA30B1AAE70379022BA6D0794A82F867
:10FE6000303195F8913443F0200385F89134002027
:10FE70009CE7406803F06AFB0028F2D095E74068F1
:10FE800003F0A8FBF8E76F4B027983F81A21E8E743
:10FE90006C4B4268C3F8E020E3E76A4E416896F88D
:10FEA000300103F0B5FB00287FF47FAF6368C6F82C
:10FEB000E430D6E7416800293FF477AF002001F035
:10FEC000B1FA0028CDD0112070E7416800293FF435
:10FED0006CAF0120F3E7416800293FF466AF0820CA
:10FEE000EDE7416800293FF460AF0920E7E741688A
:10FEF00000293FF45AAF0C20E1E7416800293FF4A4
:10FF000054AF0D20DBE7416800293FF44EAF0E20CF
:10FF1000D5E7416800293FF448AF0F20CFE74A4CAE
:10FF2000484B007983F81901A36D9847E36A984715
:10FF300097E7444B027983F88C2092E7414E037A8D
:10FF40008DF8043096F8480096F87D308DF805302D
:10FF5000072201A901F0D3FC00283FF426AF636813
:10FF600096F848000193002201A901F0C8FC00287E
:10FF70003FF41BAF6C36D4E9010186E8030070E75B
:10FF8000304E037A8DF8043096F8480096F87D30AC
:10FF90008DF80530072201A901F0B1FC00283FF4DB
:10FFA00004AFB436E7E7274E037A8DF8043096F8AD
:10FFB000480096F87D308DF80530072201A901F040
:10FFC0009EFC00283FF4F1AED4E9010106F1740370
:10FFD00083E8030096F81831022B7FF442AF96F8BD
:10FFE0003031002B3FF43DAF174BDB6A9847FEF7EB
:10FFF00075F936E7134E037A8DF8043096F8480009
:020000040801F1
:1000000096F87D308DF80530072201A901F077FCC4
:1000100000283FF4CAAEBC36ADE743680293012323
:100020008DF80C30074B02A993F8480001F074FCDE
:1000300000287FF416AFB8E6436802930023EFE789
:10004000203100205C2B0020B888030803795A1E59
:100050000E2A3FF6AAAE934A82F8683001E7914B28
:1000600042685A65FDE68F4B42689A65F9E68D4B0A
:100070004268DA65F5E68B4B42681A66F1E6894B11
:1000800042685A66EDE6874C037994F848008DF88B
:100090000430062201A901F032FC00283FF485AEAD
:1000A0009DF8043084F8DD30DBE67E4C03798DF872
:1000B000043094F8480094F87C308DF8063005221E
:1000C00001A901F01CFC00283FF46FAE9DF804303C
:1000D00084F83930C5E6734C037994F848008DF8FC
:1000E00004300A2201A901F00AFC00283FF45DAEA9
:1000F0009DF8043084F8DC30B3E66A4C037994F858
:1001000048008DF80430092201A901F0F8FB00280D
:100110003FF44BAE9DF8043084F83830A1E6614BD3
:100120004268C3F89420DA649BE65E4B027983F858
:10013000982083F8502094E65A4B4268C3F88420F4
:100140008FE6584B4268C3F8CC208AE6012B40F07A
:10015000A480554C2421204603F03AFB636A984260
:1001600001D0172022E61C2104F1280003F030FB07
:10017000636C9842F5D14FF4807104F1480003F0AC
:1001800027FBD4F848319842EBD1D42104F5A6706E
:1001900003F01EFBD4F820329842E2D1002104F58E
:1001A000097003F015FBD4F824329842D9D14FF4EA
:1001B000607104F50A7003F00BFBD4F8A83598427F
:1001C000CFD1142104F2AC5003F002FBD4F8C035B7
:1001D0009842C6D1334E2146304640F2C45203F015
:1001E000E1FA204640F2C452002103F0EFFA95F8FC
:1001F0001B3485F8E833736FC5F8EC3396F87D301F
:1002000085F8F83340F20123A5F8FA33274B96F826
:1002100019019B6D984724E68379012B3FF6C5AD04
:10022000204B42684068C3F82C2100F091FF48E65B
:100230001C4B4268C3F8902013E61A4B027983F8EE
:100240001F210EE6174B8288A3F8882009E6154B7C
:100250008288A3F88A2004E6124B8288A3F8D02073
:10026000FFE5104B8288A3F8D220FAE50D4B93F8F6
:1002700048200AB1062A12D1A288A3F8A025F0E5E9
:10028000084B93F848200AB1062A08D16268C3F8DF
:10029000A425E6E500F06AFCDBE5012086E51820F0
:1002A00084E500BF5C2B002098250020B888030857
:1002B000DFF880C0F8B5DCF840339B07064635D43C
:1002C0008778002F34D105460FCD1B4C0FC40FCDBE
:1002D0000FC42B6823609CF89134B16843F020036D
:1002E0008CF891343378BBB10D2001F09BF810B13C
:1002F00011273846F8BD7168B07801F031F900284F
:10030000F6D1B2780D4B302101FB02334FF0FF32B2
:10031000D3F80C311A60ECE70E2001F083F80028C6
:10032000E6D1F1680F2001F07DF8E8E70127E0E76A
:100330001627DEE720310020442C00205C2B002013
:10034000F0B5134FD7F840339B078BB006461AD44D
:10035000D8B9104C94F8E930BBB10146242201A869
:1003600001AD03F033FA0FCDE8340FC40FCD0FC445
:100370002B68236097F8913443F0200387F8913479
:1003800030460BB0F0BD0126FAE71626F8E700BFAD
:10039000203100205C2B002000F00303F7B51C3354
:1003A000294F13701546D7F8402392070C4647D4BF
:1003B0000A78013A012A03D90325284603B0F0BD83
:1003C00000283FD1214E96F8E920002A3AD003F0C8
:1003D0000F032B7091F908308DF8043096F848001F
:1003E00096F87D308DF80530072201A901F087FAD3
:1003F00018B12B7823F004032B70636896F848003B
:100400000193002201A901F07AFA18B12B7823F0A8
:1004100008032B702D78002DCED194E807000C4BEB
:1004200083E8070097F8912442F0200287F891248E
:100430002278012AC1D1A3F1180000F0A3FBBCE788
:100440000125BAE71625B8E7203100205C2B0020F3
:100450005C2C00202DE9F04387B00023ADF800307C
:100460000646002800F0EE800361FEF775FC20B11F
:100470000124204607B0BDE8F08300F067FD0028A6
:10048000F6D100F05DFD014618B96F48142203F063
:100490009DF96E4D95F89134012243F0040385F8DF
:1004A000552485F8913433788DF804300021013BD0
:1004B0008DF80520ADF806100C2B00F2BB80DFE8AC
:1004C00003F007B9B9B97982B9B990B9AD9AA90061
:1004D000D5F8407317F02007CAD196F80480B8F118
:1004E000020F46D1DFF868815A4CFDF791FF96F96B
:1004F000051098F848003A4601F05BFA88F8390090
:10050000B37988F83830384607238DF80530FDF781
:1005100013FFFF2304F58670A5F80C31C5F80841D8
:1005200085F8047103F066F804F58A7003F01CF88E
:100530003846FDF75BFD0446002839D096F90510D2
:1005400098F84800012201F034FA88F83900D5F80B
:1005500094343361002C71D000F0F2FC002888D173
:1005600095F8913485F81A0460F3820385F8913484
:100570007FE7B8F1010F4FF00204E8D1DFF8D09027
:100580008DF8144099F8480089F81D7102A901F00E
:10059000B1F9337989F830318DF805708DF806801E
:1005A000FDF7F2FB95F8913443F0100385F8913490
:1005B0000024CCE700226946022000F0F5FA00286A
:1005C000F6D01324C3E7244BB288DB6B96F90C10EA
:1005D000B0689847D5F8403343F00203C5F840337C
:1005E000E6E702A90D2000F055FB0028E0D000222C
:1005F00069460D20E1E7164B93F81831D3B93479E9
:1006000004F0070000F0ABFA8DF8004001226946C3
:100610001020D2E7002269461220CEE78DF807208D
:1006200000F08EFA044638B900F087FA204600F050
:1006300089FABDE702248AE7012488E701A800F0CF
:10064000D3FB16E7032414E7743500202031002083
:100650005C2B002022310020B88803082DE9F04FE0
:1006600099B08046059118B9032019B0BDE8F08F04
:1006700000230361FEF770FB0446002840F0A580CC
:1006800046460FCE0EAD0FC51422524898F800A072
:10069000B8F80C7098F90EB04F4E214603F096F85A
:1006A0004E4B012283F8412496F83021022A254638
:1006B0000BD196F81821022A07D196F81E2122B9EB
:1006C000BAF1010F38BF4FF0010ABAF1010F2BD078
:1006D000BAF1030F2AD0BAF1000F33D102229DF8EC
:1006E0003C30DDF84090029362F34715012496F800
:1006F0007C108DF8321002220CA996F848008DF873
:10070000302001F0E9F896F81A3196F830C196F8E1
:100710001D1140B2002B63D0BCF1010F57D100294D
:1007200055D1002C61D153E00422D8E70023DDF835
:100730003C90BDF840709DF942B0029365F01F05F2
:100740000124D4E74FF0000BD946CDF808B0CEE72E
:100750004FF0010084F81A04D2E005F29A420BA986
:1007600000F0D6FA002800F015811320049B33878F
:100770001A4B002283F81A2423E105F29A452A46EF
:100780000BA900F0C5FA0028EFD10B9B84F82801D3
:10079000C4F82C5184F83031FCE0B9F1000F00F0BE
:1007A000F980002A00F0F6804946E01C02F0FAFFCA
:1007B00094F8373201332380ECE01220D6E7022090
:1007C000D4E70720D4E71320D2E701204DE7FCB996
:1007D0000220F6E0603500205C2B00202031002054
:1007E000002CF5D05845B8BF584696F87C308DF8A7
:1007F0002000052296F848008DF8223008A901F063
:100800007EF800283FF430AF9DF8203086F839306C
:100810006F4A704BD2F89804D3F8904038B105F085
:1008200061FB6C4B84423CBF002283F83A20198F55
:100830001A8F93F830010491996A099152BA0028ED
:10084000BFD093F81B0100B9186393F81801ADF8F5
:100850005820013893F87C2093F81A411491D0F174
:10086000000BD3F888108DF85B204BEB000B93F84E
:10087000482093F83A0093F868308DF85A3009AB65
:100880000093554B03904FF001008DF84C001591EB
:100890008DF85C20A3F12F01A3F1300213A88DF88D
:1008A0004D4000F0DBF8039B4FEA0B1B4BEA431B68
:1008B00000264BEA801B4BEAC413B145444C03931A
:1008C00008BF37463A46494604F59C70CDE90A66AA
:1008D0009B46268084F81A6402F064FFE9B2A57092
:1008E000C5F34215FAB2042D3A4E039B84F8372221
:1008F0003FF42EAF072D3FF450AF022D7FF45FAFD2
:10090000364D84F80D110420029984F80401FF206B
:1009100084F80C0184F8281184F81431D6F8E41016
:10092000C4F8085105F59B730AA8C4F8101184F89F
:100930003021C4F82C3100F013FC00287FF43DAFC7
:100940000A9BA4F844040BA8A4F81631C4F84C344C
:1009500000F0D2F900287FF408AF0B9BD3B196F9D1
:100960003900FDF725FA94F83732002B3FF405AF34
:100970000B9B0F2B3FF6F1AE05F58B720BA90F20E9
:1009800000F0C6F900287FF4F0AE0B9B63F3030B75
:1009900084F814B10598FDF729FB00287FF4E6AE32
:1009A000099B86F83A00B36200F082F900287FF4D0
:1009B0000AAF94F8913484F840A443F0010384F81A
:1009C0009134034BD3F89434C8F810304DE600BF8F
:1009D000203100205C2B0020C42B0020223100207D
:1009E00037B50B4D8DF8040004460F2295F84800EA
:1009F00001A900F084FF40B1064A85F81C4192F835
:100A0000913443F0200382F8913403B030BD00BF2D
:100A10005C2B00202031002010B5FEF7EFFF0446CC
:100A200088B90A4805F098FA094805F095FA094886
:100A300005F092FA00F094F8FDF7EAFC064BDB6A49
:100A40009847204610BD0124FBE700BF88340020F2
:100A5000A0340020B8340020B88803082DE9F04FF6
:100A60008BB047780093149B90F90C8090F90D603F
:100A700090F80EB08A464168196004469146002FEE
:100A800058D002238DF8103004A9C37B007C8DF868
:100A9000123000F021FFB4F808C0618943B26068E9
:100AA000984545466144B8BF1D46604534BF0027A0
:100AB0000127884209D30A218DF81010207C019368
:100AC00004A900F009FF019B46B2B4F808C0608990
:100AD00061680CEB400E714519D3A1EB0C01B1FB21
:100AE000F0FC00FB1C1191B9984503DC2378CBB9CD
:100AF0004FF0010B21238DF81030207CE37B8DF823
:100B0000115004A98DF8123000F0E6FE45B2009BAA
:100B10008AF80050384689F8006083F800B00BB0BE
:100B2000BDE8F08F0223207C8DF8243006A900F068
:100B3000E1FEDDE74546EAE77047704770477047DA
:100B400000207047704770477047002070470020B2
:100B500070470020704700207047002070477047A2
:100B6000704770470220704702207047022070478C
:100B70007047002070477047704700207047002082
:100B800070477047704770477047000010B5054CBC
:100B90004FF403722046002102F018FE0020C4E941
:100BA000000010BD3C3600202DE9F84381469046F8
:100BB00000293CD01F4C2023224604F1100012F8DB
:100BC000017F6FBB8242FAD11B4E3368013403B9F7
:100BD0003460736803B11C6000252560C4F8088088
:100BE00074601FFA88F284F80490601D02F0DAFD48
:100BF000B9F1110F4FF0000398BF104D6373D6F891
:100C0000083298BF25FA09F503F1010398BF05F0F2
:100C1000010543442573C6F808323846BDE8F88319
:100C2000013B13F0FF030446C6D10227F5E7012775
:100C3000F3E700BF433600203C36002020070200C7
:100C400010B518B3124A1368984204D103681360B0
:100C5000002305E00B46002BFAD019688842F9D131
:100C60005168884208BF53600BB101681960D2F81F
:100C700008328168013B00245B1A04602146C2F8F7
:100C80000832102202F0A2FD204610BD0120FCE730
:100C90003C360020054B1B6813B11A798242FAD109
:100CA000002B0B600CBF0320002070473C36002057
:100CB00010B5054B186800B910BD037B04680BB96B
:100CC000FFF7BEFF2046F6E73C36002038B5084B5C
:100CD000084C186800B938BD03790568112B05D890
:100CE00024FA03F3DB0701D5FFF7AAFF2846F1E753
:100CF0003C3600202007020028B1044BD3F808320C
:100D00000360002070470120704700BF3C36002080
:100D10002DE9F04107460E46154642B339B3154B4F
:100D20001C6800232CB93046FFF7E6FF0020BDE821
:100D3000F081A268F91A0132914215D32279EA545E
:100D4000581C22895FFA80F8611D55FA80F002F084
:100D500029FDA368246898445FFA88F3E2E72046F7
:100D60002568FFF76DFF2C46002CF8D1DBE701204A
:100D7000DDE700BF3C3600200238C0B211289ABF20
:100D8000014B185C00207047D581030830B50B4B30
:100D900093F820200446084672B100211C330578E0
:100DA000A54208D001319842CDB214BF04301038AA
:100DB000AA42F4D8002030BD1046FCE74838002095
:100DC00010B5084C00232060142204F10C00FF2110
:100DD00084F82030C4E9010002F0F8FC012384F813
:100DE000213010BD4838002010B50E4A92F820106E
:100DF000042915D8936804781C7044785C70C47812
:100E0000807898700131DC7082F8201002F11C01AA
:100E10008B4214BF043302F10C039360012010BD18
:100E20000020FCE748380020094B93F8200068B107
:100E30005A6803F11C018A4200F1FF3014BF0432EA
:100E400003F10C0283F820005A600120704700BFB4
:100E50004838002010B5074B93F820200446084678
:100E600032B15968FFF792FF10B1012344708370CB
:100E700010BD00BF4838002008B5064B93F820206D
:100E80002AB15968FFF782FF08B1407808BD0120F8
:100E9000FCE700BF4838002030B50A4A92F820101D
:100EA000536882F8210061B1916801241C32DD7819
:100EB000587005B99C70934214BF0433103B99429B
:100EC000F5D130BD4838002008B5044B5968FFF70C
:100ED0005DFF003818BF012008BD00BF4838002062
:100EE000F7B50422154E044600210DEB020096F8DA
:100EF000207002F06BFC0025EBB29F4201D803B0DA
:100F0000F0BD7368197821705A786270987838B19A
:100F1000336820469B689847FFF786FF0135EBE76B
:100F2000DB788DF804108DF805208DF80730FFF779
:100F30007BFF01A8FFF758FFF0E700BF483800200B
:100F4000014B93F82000704748380020034B93F87A
:100F50002000042894BF002001207047483800205A
:100F60001FB50024CDE90244C41F8DF800408DF860
:100F700001100C0AADF80420090C120C8DF80310B6
:100F80008DF806208DF8073002461B0A01216846BD
:100F90008DF802408DF8083002F073FA002818BF6F
:100FA0000E2004B010BD2DE9F04188B090460D46EA
:100FB0000F9A0746002847D000240121CDE90444B8
:100FC0008DF810109DF838108DF81510ADF816300A
:100FD000190CCDE900441B0ECDE902448DF81930FF
:100FE000ADF81A20130C120E07948DF818108DF816
:100FF0001C308DF81D20E3B21E01002DF6B203DC7B
:10100000002008B0BDE8F081013310218DF81F30B9
:1010100042466B460DEB010002F0C9F90346A8B940
:10102000102D28463E44A8BF10206946327811F89A
:1010300001CB013382EA0C02984206F8012BF5DC61
:10104000103D2DB20134D6E70920DAE70E20D8E7AB
:101050000138032815D8DFE800F002080C100A4B0D
:101060001B681B690B6000207047074B1B685B699E
:10107000F8E7054B1B689B69F4E7034B1B68DB69CA
:10108000F0E70520704700BF6C3800202DE9F041E3
:10109000C4B00C464A9E17461D468046B8B3B1F50B
:1010A000807F36D84FF488720021684602F08EFBAC
:1010B000492300934FF48073ADF804302B0C8DF866
:1010C0000830330CADF80650ADF80A608DF80C30DE
:1010D00022460023414604A82D0E360E8DF80E3010
:1010E0008DF809508DF80D608DF80F4002F05AFB15
:1010F00004F110014B9A3B4689B2684602F041F96F
:1011000010B1012818BF0E2044B0BDE8F0810920BD
:10111000FAE70D20F8E7000010B590B10A4C28223C
:101120000021206002F052FB2368084A1A60002068
:101130004FF0FF32C3E90302C3E90522C3E90722E6
:1011400010BD0820FCE700BF6C3800200001010141
:10115000024B1B6818600020704700BF6C380020ED
:1011600030B1044B1B68DB6801330360002070471B
:10117000092070476C38002013B500230C460193FA
:10118000CAB101A9FFF764FF18B9019B591C02D12C
:10119000146002B010BD99B2611A002901DD5C181B
:1011A000F6E702D113600720F3E71B0C1B0403F5DD
:1011B00080331C44ECE70920EBE7000028B1044B26
:1011C0001B681C334362002070470920704700BF32
:1011D0006C3800201FB5044600B3002303A8039316
:1011E00002F0A6F9104ABDF80C3012682046938030
:1011F000E38200F0A8FA98B904F11803009321687B
:101200000123132202F0B2F860B9204600F09BFAE5
:10121000003818BF0120000104B010BD0920FBE711
:101220001020F9E70E20F7E76C380020F0B50546EE
:1012300087B01C4613B9092007B0F0BD2E4E3368A5
:10124000DB68834255D894F82020002A0CBF08227E
:101250000922834205D3204600F0A9FA68B1102084
:10126000EAE7002301900093A36894F82810606ACD
:10127000FFF799FE0028EED0DEE723792168B4F865
:1012800008C0A768043B9AB20029D4D0B2F5807F89
:101290002DD8ADF80EC08DF817304FEA174C04F179
:1012A0002C033F0E8DF8117000932F0C08234FF084
:1012B000490EADF80C008DF814708DF816002F0E45
:1012C0000DEB0300CDF808E08DF810C0ADF812501A
:1012D0008DF8157002F04AF808B10E20ACE72046F0
:1012E00000F065FA0028BAD13368DD60A4E70D206C
:1012F000A2E70620A0E700BF6C3800202DE9FF41DF
:101300000A9D80460F4616461C46002D5AD00023E3
:1013100003A910460393FFF79BFE18B1062004B003
:10132000BDE8F081039B9C4201D80133F6D12846E9
:1013300000F0AEF9002847D1264B1A78424503D079
:101340001A79424542D10120AA68BA4240D103EB42
:101350008002EB6A92F801802979CDE900430439D3
:10136000927828683B4689B2FFF790FE0028D6D1D4
:1013700095F820300194002B4FF00103009314BF27
:101380004246082295F82810686A3B46FFF70BFE94
:101390000028C4D1013E032EC1D8DFE806F00207C1
:1013A0000B0F0D4B1B681C611C62B8E70A4B1B68D6
:1013B0005C61F9E7084B1B689C61F5E7064B1B680D
:1013C000DC61ACE70920AAE70F20A8E70B20A6E71D
:1013D0000220A4E71C0500206C3800201FB50B2953
:1013E0004FF00003CDE90033CDE902330A4607D0C0
:1013F0000C2914D00A2910D00A2005B05DF804FB8E
:10140000012802D120238DF800300021684602F027
:1014100038F8002818BF0E20EFE73023F3E70B2140
:10142000F4E7000038B5054602F026F8044610B18E
:101430000E24204638BD002DFBD1094B1B680B2123
:101440009878FFF7CBFF0028F2D10C21FFF7C6FFF9
:101450000028EDD10A21FFF7C1FF0028E9D0E7E716
:101460006C3800202DE9F04380468FB00C461746BB
:10147000002A6BD0002969D0002529461D2206A824
:1014800005951EF09DF88DF81350344D2B680DF125
:1014900014099E88CDF804900DF1130302933B7953
:1014A00000933B6832462146404602F006F8002889
:1014B0004ED138683A79494602F074F9384600F05E
:1014C00099F8002846D13C7AFA79BB79240444EA99
:1014D00002241C432B689A6894423DD99C609DF875
:1014E00013000B21FFF77AFF034658BB0C21FFF7CF
:1014F00075FF034630BB0A21FFF770FF034608BBA8
:101500007B7ABA7AFF7A3F0447EA02271F433A46BA
:10151000334621460920FFF723FD034690B93346A1
:101520003A4621460820FFF71BFD034650B92A68BA
:101530009DF8131091700021D1604FF0FF31C2E986
:101540000411916118460FB0BDE8F0830923F9E753
:101550000E23F7E70F23F5E70323F3E76C380020AA
:1015600070B588B000293FD0214C2378834231D018
:10157000237983423AD101220023CDE90133CDE919
:10158000053304EB8204039307930123C1F307207F
:10159000CDB28DF80030C1F30743090E8DF802007B
:1015A0008DF8041002268DF812008DF81410627860
:1015B000E1788DF8015068468DF803308DF81060A1
:1015C0008DF811508DF8133001F05BFF20B10E2023
:1015D00008B070BD0022CFE7A278E17804A801F03E
:1015E00050FF0028F4D0F2E70920F1E70B20EFE7E5
:1015F0001C05002010B50446002845D001680029CC
:1016000042D011F8013B43710322063002F0CAF8C0
:101610002046032250F8091B043102F0C3F8216868
:10162000CB79E3600A7A43EA0223E3604A7A43EA29
:101630000243E3608A7A43EA0263E360CB7A23746D
:101640000B7B63742379212B1AD110220D3104F105
:10165000120002F0A7F81D222168501C8B5C636207
:10166000085C43EA0023901C6362085C033243EA8F
:10167000004363628A5C43EA02636362002010BD38
:10168000112B03DC0D22E7E70220F8E70120F6E743
:1016900010B50446002854D00168002951D00B78B9
:1016A00043714B7883608A7843EA02238360CA7867
:1016B00043EA024383600A7943EA026383604B7919
:1016C00003738B79C381CA7943EA0223027BC38106
:1016D00002F00F020831103002F064F8237B002280
:1016E00003F00F0384F8202084F82820227903F1E6
:1016F0000800111A04290DDD21680933043AD21AB1
:10170000085C84F82000D2B2606A84F8282019446A
:1017100002F048F8237922681A44002012F8043CA9
:10172000E36212F8031C43EA0123E36212F8021C8D
:1017300043EA0143E36212F8012C43EA0263E362E5
:1017400010BD0220FCE710B5044660B3036853B334
:101750000279162A29D942791A700146082251F8CD
:10176000060B013002F028F82146082251F80E0B32
:10177000093002F021F82368E28A5A74E38A226869
:101780001B0A93742368A269DA74A36922681B0A8E
:1017900013752368628B5A752368E27E9A75172346
:1017A0002371002010BD0120FCE70220FAE738B5C4
:1017B0000446002863D00168002960D0037B90F8BC
:1017C000282003F00F03002A57D108332079043270
:1017D0001344984255D363790B702368A2685A70FA
:1017E000A36822681B0A937023686289DA702368F1
:1017F000E27A1A712368227B5A712368E2899A710E
:10180000E38922681B0A2146D371227B51F8100B11
:1018100002F00F02083001F0C5FF237B94F8282066
:1018200003F00F0303F108052AB1226894F8201091
:10183000515503F10905206894F82820616A28446D
:1018400001F0B0FF94F828302268E16A2B44D154AB
:101850005A1CE16A206892B2090A81549A1C2168D4
:10186000E08D92B28854DA1C216894F82F0092B26D
:10187000043388542371002038BD0933A6E70120C2
:10188000FAE70220F8E70000024B1A88104318809C
:10189000704700BF7038002008B5074B1B883BB16C
:1018A000FEF7ACF8002814BF6FF00200002008BD5E
:1018B0006FF00100FBE700BF7038002010B5034B4C
:1018C00000241C80FEF790F8204610BD70380020E0
:1018D000B0FA80F04009704782B018B9084602B0EB
:1018E00000F0CAB8002002B0704710B9084600F0F6
:1018F00079B9704710B9084600F090B970470346AF
:10190000084611460BB900F0DDB90020704710B948
:10191000084600F039BD704710B9084600F0FEB91E
:101920000020704710B40446084611461A46019B31
:1019300014B910BC00F00CBA10BC7047034608463E
:1019400011460BB900F036BA0020704710B40446B7
:10195000084611461A4614B910BC00F0A3BA00207C
:1019600010BC704730B40546084611461A46DDE9FA
:1019700002341DB9029430BC00F022BB002030BC00
:10198000704710B9084600F0D3BB0020704710B96B
:10199000084600F037BD0020704710B9084600F037
:1019A000E2BB0020704710B9084600F0DFBB002002
:1019B00070470346084611460BB900F0F9BB0020FA
:1019C000704710B40446084611461A46019B14B9E4
:1019D00010BC00F0EFBB092010BC704710B40446E7
:1019E000084611461A4614B910BC00F02DBDC8B205
:1019F00010BC70470048704701000102064B10B54B
:101A00001B6A0446984730B10448054B204498426D
:101A10008CBF0020012010BDB8880308403576C96E
:101A2000405DC600F0B5114B85B00C4610491F56FD
:101A3000054601F017F80F4BE4B25E6A072D4FF030
:101A40000103CDE9024301460AD105220023CDE975
:101A500000234FF47A727A431846B04705B0F0BDC0
:101A600008220020CDE900203A46F5E7A0820308CD
:101A700080820308B88803081FB500230093037809
:101A8000013B372B21D8DFE803F01C242020201E47
:101A9000202020204143454E2055585B5E61642044
:101AA0006C1E6E73787A7D207F8326202020202074
:101AB000202020202020202085878C2020858C201D
:101AC0008E92C3780BB102230093009805B05DF8A5
:101AD00004FB8378F6E743788DF8043007238DF80C
:101AE00005308378003B18BF01235B008DF806307A
:101AF00010238DF80730314B1B6801A803F558728D
:101B0000CDE9022300F08EFF0090DEE74023DBE703
:101B10002023D9E7827890F9013012B9284AD35CA2
:101B2000D2E7284AFBE7827890F90130002AF8D101
:101B3000254AF4E740F6B833C6E74FF47A73C3E7B3
:101B40004FF4FA63C0E741F28833BDE741F27073A6
:101B5000BAE71E484FF47A7101F008FE00F5FA600A
:101B6000D2E71B4BB0E7154B1B6803F55873ABE787
:101B7000124B1B6803F55B73A6E71023A4E70F4B1A
:101B80001B68A1E701239FE74FF0834300939CE785
:101B9000104BFBE7104B97E740F21113ADF8003004
:101BA00093E7032390E790F901300C4AB7E70C491B
:101BB00090F9010000F056FFA6E700BF783800203A
:101BC00077820308678203086F82030818FCFFFF0F
:101BD00000EA06379A99094040F70937A0820308BE
:101BE0008082030837B50B4B02781B680C2101FB80
:101BF00002335B7A03EB4304074B1D6803690093D0
:101C0000C3684278816805EBC40000F0A7FC03B00C
